:020000040800F2
:10800000A8DA0020D1B700080D90000817900008EA
:1080100029900008339000083D90000800000000FF
:108020000000000000000000000000005D82000869
:10803000519000080000000091820008EFF5000850
:10804000EBB70008EBB70008EBB70008EBB7000888
:10805000EBB70008EBB7000805E900082FE90008B6
:1080600055E900087BE90008EBB70008EBB700080A
:10807000EBB70008EBB70008EBB70008EBB7000858
:10808000EBB70008EBB70008EBB70008EBB7000848
:10809000EBB70008EBB70008EBB70008A1E9000850
:1080A000EBB70008EBB70008EBB70008EBB7000828
:1080B000EBB7000865D90008EBB70008EBB700087C
:1080C000EBB70008EBB70008EBB70008EBB7000808
:1080D000EBB70008A52B0108EBB70008EBB70008C9
:1080E0000FEA0008EBB70008EBB70008EBB7000891
:1080F000EBB70008EBB70008EBB70008EBB70008D8
:10810000EBB70008EBB70008EBB70008EBB70008C7
:1081100057970108EBB70008D3D90008EBB7000860
:10812000EBB70008EBB70008EBB70008EBB70008A7
:1081300000F002F800F082F80AA090E8000C8244F7
:108140008344AAF10107DA4501D100F077F8AFF2D4
:10815000090EBAE80F0013F0010F18BFFB1A43F025
:108160000103184738D7010058D701000A444FF0DF
:10817000000C10F8013B13F0070408BF10F8014B86
:108180001D1108BF10F8015B641E05D010F8016BCB
:10819000641E01F8016BF9D113F0080F1EBF10F82F
:1081A000014BAD1C0C1B09D16D1E58BF01F801CB52
:1081B000FAD505E014F8016B01F8016B6D1EF9D5D5
:1081C0009142D6D3704700000023002400250026EA
:1081D000103A28BF78C1FBD8520728BF30C148BF2A
:1081E0000B607047642919F0EB87752919F0E8874F
:1081F00078291AF0218073291AF0738400207047BF
:1082000054656D636F5049443533202000000047AA
:10821000003530001FB51AF00EFA1AF063FD0400A5
:10822000002000211CF04EF9401C6060002000215D
:108230001CF05EF9E0601FBD10B510BD1AF090FF94
:108240001146FFF7E7FF00F02EFE1BF02BFA03B4F8
:10825000FFF7F2FF03BC07F06BFA00001A4B196836
:108260000868B0E8F00F80F309884FF0000080F351
:1082700011884EF00D0E70470000000003480068A2
:10828000006880F3088862B600DF00BF08ED00E0F8
:10829000EFF309800C4B1A6820E9F00F106008B565
:1082A0004FF0BF0080F3118806F0DCFE4FF00000B5
:1082B00080F31188BDE8084019680868B0E8F00F3D
:1082C00080F30988704700BFB800002001B44FF068
:1082D000BF0080F3118801BC704701B44FF000006B
:1082E00080F3118801BC70470B49D1F800C04A687F
:1082F0005CF8043B1068184442F8040B8C4528BF16
:10830000A1F1DC0C8A4228BFA1F1DC02C1F800C057
:108310004A6020F00040704740C8002010B501219D
:108320000D2001F059FF0121FA4801F04AFD10BD6E
:1083300010B512F07BFDF848006812F07EFD12F0D7
:108340003FF84FF0FF300EF0A4FA2020F3490870F8
:10835000F34908703420F34908800EF05CF910BD31
:1083600086B00024FFF7E4FF002013F0F9F90020A5
:1083700014F0AAF800BFEC48807C80B900200346C6
:108380004FF41672E949009001A812F022FD04464C
:108390002CB100232246E54901A814F058F8052025
:1083A00007F093FAE7E738B5E148007860B90120B3
:1083B000DF4908704FF4FA71DE4807F0A9FA42F27B
:1083C0001071DD4807F0A4FA09F040FADB49088093
:1083D00008460088002835DD0220D949087080024F
:1083E00007F011FBD7498989884217D1012007F08E
:1083F00004FDD248008800286DDD09F006F809F078
:108400002DFA0220D0490870D0480068006800901A
:10841000CE490968C88807F0F6FA5CE040F6060025
:1084200007F0F1FAC7498989884254D108F081FFE1
:10843000C248008800284EDD09F010FA0220C24927
:10844000087048E0BB4807F076FA002843D0B948E6
:1084500007F066FA002418E000BF04EB8400BC4972
:1084600001EBC000BB490860022007F0C6FC00BF5A
:10847000B2480088002806DD08F0C7FF09F0EEF9D1
:108480000220B1490870601CC4B21E2CE4DB002439
:1084900016E000BFB04800EB8410AC49086005202E
:1084A00007F0ABFC00BFA5480088002806DD08F0F7
:1084B000ACFF09F0D3F90220A3490870601CC4B2D4
:1084C0000A2CE6DB9C4807F036FA20B19A4807F000
:1084D00027FA08F080FE38BD002405E0322007F0BE
:1084E000F4F99EA019F022FE09F06AF80028F5D1EF
:1084F00000BFFFF758FFA0480078012803D09F482D
:108500000078012809D1601CC4B20A2C05D10024CE
:108510000020994908700AF079FC01F0D8FC02208B
:1085200007F0D3F9E5E710B595480068012805D1B3
:1085300094480088401C9349088002E0002091493B
:10854000088090480088642804DD00208D49088058
:108550000AF020FB10BD0AF04EFC00BFFFF7E3FF5E
:108560008948007850B188480078401E86490870D4
:1085700008460078012801D10CF0A1FE834800785C
:10858000002809DD81480078401E804908700846AF
:10859000007808B90AF0FEFA052007F096F9DDE741
:1085A00003F036F900207A4908707A49088000BF44
:1085B00079480078401C78490870084600780228FD
:1085C00003DB0020087003F095F974488088401C94
:1085D000724988800A2007F078F971480078401CB9
:1085E0006F490870084600786428E1DB0DF0F2FF5F
:1085F00007F09DFA00206A490870D9E700BF0024FF
:1086000031E0684830F8140001282AD1464A403247
:1086100012F83410A20002F1BE0004F07DFE424ABE
:10862000403202EBC4025178A20002F1BF0004F014
:1086300073FE3D4A403202EBC4029178A20002F17F
:10864000C00004F069FE384A403202EBC402D1781F
:10865000A20002F1C10004F05FFE0020514921F8A0
:108660001400601CC4B2202CCBDB40F6B83007F0FD
:108670002CF9C4E705F032FD00BFFFF727FE4A489A
:10868000046805F0CDFF48480068051B681D0521FA
:10869000B0FBF1F045490988084444490880084680
:1086A0000088C82801DB0EF033FD40480088B0F593
:1086B0007A7F04DB00203D4908800EF08DFE052006
:1086C00007F003F935480089401C34490881FFF759
:1086D000FDFDD2E77CB504F0EFFD1D2004F0F0FDB8
:1086E0008DF80000202004F0EBFD8DF801009DF8CE
:1086F00000109DF8010001EB00202D4908800DF0CD
:10870000A3FE94285AD10A202449888229A00CF07B
:108710003BFE7DE00004300004000020F301002057
:10872000F5010020F40100205860002048040020DA
:1087300024000020140000201C0000203C01002028
:108740005B000020984800205C00002048010020C9
:108750009C50002044010020885500207461706402
:1087600065765F696E69742829206661696C656445
:10877000202E2E2E0D0A0000820100200000002075
:10878000A0012142100000208A0100208801002061
:108790000A0000200C0000200E0000206865002068
:1087A0000F000020A016002064000020120000200E
:1087B000C001002054335F33324149000DF044FEC4
:1087C00040F2CA51884203D11420FE4988821FE03A
:1087D0001E20FC4988821422FB4940F2BA2004F092
:1087E0000FFEF9480078FF2812D1F7484078FF289B
:1087F0000ED1F5488078FF280AD1F348C078FF28C9
:1088000006D1F1480079FF2802D1F0A00CF0BCFDA0
:10881000002004F055FDF0490870012004F050FDDF
:10882000ED494870022004F04BFDEB4988700320AD
:1088300004F046FDE849C87008460078FF2811D1C9
:1088400008464078FF280DD108468078FF2809D1D6
:108850000846C078FF2805D1012008704870022022
:108860008870C870002407E004F1160004F028FDA9
:108870000DF80400601CC4B2042CF5DB9DF8000068
:108880009DF8011000EB01209DF8021000EB014063
:108890009DF8031000EB0160D049086008460068AD
:1088A000401C70B10846008880B24FF6FF718842C4
:1088B00007D0CA48006820B1C8480068B0F5800FEA
:1088C0000FD3C5480078C449497800EB0120C2495C
:1088D000897800EB0140C049C97800EB0160BF49CD
:1088E0000860042004F0ECFC8DF80000052004F082
:1088F000E7FC8DF801009DF800109DF8010001EBE8
:10890000002085B24721042004F006FD0021052047
:1089100004F002FD3F2D02DA04200EF039FE06209D
:1089200004F0CEFCAC49087108460079FF2802D05B
:108930000846007938B9FE20A74908710846017930
:10894000062004F0E9FC3520A3498873122004F0C6
:10895000B7FCA349087008460078FF2803D00846F2
:108960000078012807DCFE209D4908700846017840
:10897000122004F0D1FC984800799A4908701B2015
:1089800004F09EFC8DF800001C2004F099FC8DF88A
:1089900001009DF80000FF2801D1012000E0002027
:1089A0009DF80110FF2901D1012100E000210840BC
:1089B00020B14BF6C0208849888707E09DF8010068
:1089C0009DF8001040EA012083498887082004F0C0
:1089D00077FC8149C8730846C07BFF2802D008464F
:1089E000C07B10B903207C49C873102004F068FCD8
:1089F00079494873112004F063FC77490874132007
:108A000004F05EFC74490873152004F059FC8DF8DD
:108A100000007148007B052802DD01206E490873C3
:108A20009DF800006C49097B884204D06A48017BAC
:108A3000152004F071FC6848007B062834D2DFE87A
:108A400000F0030B131B232B4FF416506249886070
:108A500006206549087028E04FF496405E4988601A
:108A600003206149087020E04FF416405A4988609D
:108A700002205D49087018E04FF461405649886053
:108A800001205949087010E04FF4E13052498860E4
:108A900001205549087008E04FF496304E4988602F
:108AA00001205149087000E000BF00BF4A498868B2
:108AB00006F057FE142004F003FC4749887408466A
:108AC000807C032804D00846807C08B10320887489
:108AD000002407E004F1280004F0F2FB0DF8040084
:108AE000601CC4B2062CF5DB9DF80000FF2825D1E0
:108AF0009DF80100FF2821D19DF80200FF281DD11B
:108B00009DF80300FF2819D19DF80400FF2815D116
:108B10009DF80500FF2811D104208DF800000220E7
:108B20008DF8010035208DF80200AF208DF803008C
:108B300000208DF8040001208DF80500002406E0D7
:108B40001DF80410244814300155601CC4B2062CD2
:108B5000F6DB002407E004F12F0004F0B1FB0DF870
:108B60000400601CC4B2042CF5DB9DF80000FF2853
:108B700041D19DF80100FF283DD19DF80200FF285A
:108B800039D19DF80300FF2835D1C0208DF80000B1
:108B9000A8208DF8010000208DF8020003208DF838
:108BA00003009DF800102F2004F0B6FB9DF8011083
:108BB000302004F0B1FB9DF80210312004F0ACFB32
:108BC00014E0000068650020C46200203372642055
:108BD00070726F6475637400586000200400002098
:108BE0008F0100208E010020890100209DF80310D4
:108BF000322004F091FB002408E01DF80410E8483E
:108C00000155015D11300155601CC4B2042CF4DB28
:108C10002E2004F055FB8DF800009DF8000001287F
:108C200007DD00208DF800009DF800102E2004F0D4
:108C300073FB9DF80000DA491A3988770846807F6F
:108C400081F82F00002407E004F1330004F038FB22
:108C50000DF80400601CC4B2042CF5DB9DF8000084
:108C6000FF2828D19DF80100FF2824D19DF802009B
:108C7000FF2820D19DF80300FF281CD18DF80000AB
:108C80008DF801008DF8020000208DF803009DF89A
:108C90000010332004F040FB9DF80110342004F054
:108CA0003BFB9DF80210352004F036FB9DF80310C5
:108CB000362004F031FB002409E01DF80410B84808
:108CC000401D0155015D11300155601CC4B2042CDA
:108CD000F3DB002407E004F1370004F0F1FA0DF8AB
:108CE0000400601CC4B2042CF5DB9DF80000FF28D2
:108CF0002BD19DF80100FF2827D19DF80200FF2805
:108D000023D19DF80300FF281FD1C0208DF800005B
:108D1000A8208DF8010000208DF8020004208DF8B5
:108D200003009DF80010372004F0F6FA9DF80110BA
:108D3000382004F0F1FA9DF80210392004F0ECFA22
:108D40009DF803103A2004F0E7FA002409E01DF82A
:108D50000410934809300155015D11300155601C24
:108D6000C4B2042CF3DB3B2004F0AAFA8DF8000017
:108D70009DF80000FF2807D100208DF800009DF825
:108D800000103B2004F0C8FA9DF8000084491A390D
:108D900081F82700084690F8270081F838003C2029
:108DA00004F08EFA8DF800003D2004F089FA8DF869
:108DB00001009DF80000FF2812D19DF80100FF2856
:108DC0000ED14FF4FB7076491A3908850846008D9C
:108DD000000A8DF80000084690F828008DF8010080
:108DE0009DF801009DF8001040EA01206C491A39F5
:108DF00008850846008D4887002081F83E00C87429
:108E00000C2004F05DFA67490870002448E0A100D6
:108E100001F1BE0004F054FA6149263101F8340032
:108E2000A10001F1BF0004F04BFA5D49263101EBCE
:108E3000C4014870A10001F1C00004F041FA584992
:108E4000263101EBC4018870A10001F1C10004F0DA
:108E500037FA5349263101EBC401C8705048263017
:108E600010F83400FF2819D14D48263000EBC4001B
:108E70004078FF2812D14A48263000EBC4008078A1
:108E8000FF280BD14648263000EBC400C078FF28ED
:108E900004D100214248263040F83410601CC4B28E
:108EA000202CB4DB7CBD1FB53F49080300F041FA1C
:108EB000FFF734FA4FF4A06000F004FA01212020FB
:108EC00001F08AF9482006F0B1FCFFF703FC0EF030
:108ED00091FB04F0F7FA04F07DFB0EF09BFD33A04C
:108EE00019F024F900200323CDE900300290034655
:108EF000802231A10390324805F046FE0020012374
:108F0000CDE900300290034680222EA10390AFF6F7
:108F1000131005F039FE00200423CDE90030029043
:108F200003464FF41D722AA103902C4805F02CFE35
:108F300000200223CDE9003002900346802228A1C0
:108F40000390294805F020FE00200423CDE90030DD
:108F500002900346802225A10390264805F014FEC6
:108F600000200123CDE90030029003464FF4207227
:108F700021A10390214805F007FE00200423CDE93C
:108F80000030029003464FF420721DA103901E484A
:108F900005F0FAFD06F080F9002004B010BD0000D5
:108FA00072600020090000200080000854335F73C5
:108FB00065726965730A0D00494E5055545300009F
:108FC0007586000853544F52454545500000000037
:108FD000576966697461736B00000000E57B0108E6
:108FE0004C45443000000000A1850008434F4D4D22
:108FF00000000000578500084E455400D984000841
:109000004D535450000000006183000810B518A0B3
:1090100019F08CF810BD06E0184883884288018852
:1090200017A019F083F8F7E702E01BA019F07EF80B
:10903000FBE702E01BA019F079F8FBE702E01CA0B7
:1090400019F074F8FBE710B51DA019F06FF810BD0A
:1090500010B51DA019F06AF810BD10B51CA019F0CC
:1090600065F810BD10B51CA019F060F810BD000027
:109070004E4D49206661756C7400000068650020E3
:1090800048617264204661756C742025642C2564E7
:109090002C256420000000004D656D204661756C34
:1090A00074200000427573204661756C74200000C6
:1090B0005573616765204661756C7420000000007F
:1090C000535643200000000044656275672000008D
:1090D00050656E20000000005379735469636B2063
:1090E000000000000CB50020019000906C48006862
:1090F00040F480306A49086000BF6948006800F4A5
:10910000003000900198401C0190009818B9019817
:10911000B0F5A06FF1D16248006800F4003010B1E2
:109120000120009001E0002000900098012843D128
:109130005C48006840F010005A4908600846006822
:1091400020F0030008600846006840F00200086054
:10915000534840685249486008464068486008469D
:10916000406840F4806048600846406820F47C1005
:1091700048600846406840F4E810486008460068C7
:1091800040F08070086000BF4548006800F0007043
:109190000028F9D04248406820F003004049486068
:1091A0000846406840F00200486000BF3C48406804
:1091B00000F00C000828F9D10CBD10B5FFF792FFA4
:1091C00010BD10B53648006840F001003449086011
:1091D00008464068344908403149486008460068FC
:1091E000324908402E4908600846006820F4802073
:1091F00008600846406820F4FE0048604FF41F00F5
:109200008860FFF7DAFF4FF000602949086010BD61
:1092100010B5002100200022214B5B6803F00C01F7
:1092200021B1042906D0082928D107E0214B224C7E
:10923000236027E01F4B204C236023E0184B5B6822
:1092400003F47010164B5B6803F48032022303EBC7
:10925000904022B9194B4343174C23600DE0104B4B
:109260005B6803F4003323B1144B4343124C236077
:1092700003E0104B4343104C236003E00D4B0E4CB6
:10928000236000BF00BF064B5B68C3F303130C4CA5
:10929000E15C094B1B68CB40074C236010BD00000C
:1092A00000100240002002400000FFF8FFFFF6FE21
:1092B00008ED00E000127A002800002000093D00BF
:1092C0002C00002031490143314A1160704770B5CC
:1092D000002100230F22C47804B32D4C246804F429
:1092E000E064C4F5E064210AC1F10403CA40447893
:1092F00004FA03F18478144021430901254C0678CF
:10930000A155047804F01F050124AC4005786D11C7
:10931000AD0005F1E025C5F8004109E0047804F04E
:109320001F050124AC401C4D0678761145F82640F7
:1093300070BD1A4A0A400243154B1B1F1A60704742
:1093400039B1134A121D12680243114B1B1D1A60DA
:1093500006E00F4A121D126882430D4B1B1D1A6056
:109360007047042808D14FF0E021096941F0040159
:109370004FF0E022116107E04FF0E021096921F090
:1093800004014FF0E0221161704700000000FA056F
:109390000CED00E000E400E080E100E080FFFF1F52
:1093A00010B50446FA48844208D10121401500F066
:1093B0002DFF0021601500F029FF17E0F5488442D9
:1093C00008D10121001500F021FF0021201500F037
:1093D0001DFF0BE0F048844208D10121C80300F0D2
:1093E00015FF00214FF4004000F010FF10BD30B514
:1093F0000246002000235068E84C20400D790C689C
:1094000044EA0524204350609068E54C2040D1E9AF
:1094100002542C434D7944EA450420439060D06ABD
:1094200020F470000C7C641EE4B2234340EA035035
:10943000D06230BD00210160017141718160C16065
:1094400001210174704721B1826842F001028260FB
:1094500003E0826822F001028260704721B18268D5
:1094600042F48072826003E0826822F4807282603B
:10947000704710B50023CBB21AB144681C43446056
:1094800002E044689C43446010BD816841F00801DB
:1094900081607047014600208A6802F008020AB124
:1094A000012000E000207047816841F004018160E4
:1094B0007047014600208A6802F004020AB10120C8
:1094C00000E00020704721B1826842F4A00282606F
:1094D00003E0826822F4A002826070470146002007
:1094E0008A6802F480020AB1012000E0002070477F
:1094F00010B50A4600210023416821F46041531E43
:1095000041EA4331416010BD21B1426842F400623A
:10951000426003E0426822F4006242607047F0B5A6
:1095200004460D4600200021092D11DDE068A5F15B
:109530000A0606EB4607072606FA07F18843A5F157
:109540000A0606EB460603FA06F10843E0600CE063
:10955000206905EB4507072606FA07F1884305EB66
:10956000450603FA06F108432061072A0FDA606B0B
:10957000561E06EB86071F2606FA07F18843561E7D
:1095800006EB860605FA06F10843606322E00D2A21
:109590000FDA206BD61F06EB86071F2606FA07F1A7
:1095A0008843D61F06EB860605FA06F108432063BA
:1095B00010E0E06AA2F10D0606EB86071F2606FA08
:1095C00007F18843A2F10D0606EB860605FA06F1BF
:1095D0000843E062F0BD21B1826842F480128260EB
:1095E00003E0826822F48012826070470146C86CF2
:1095F00080B2704766484C300068704721B14268BD
:1096000042F48062426003E0426822F48062426079
:10961000704721B1426842F48052426003E04268E0
:1096200022F48052426070470A460021816821F48A
:10963000E04111438160704721B1826842F40042E9
:10964000826003E0826822F400428260704721B1A8
:10965000826842F40212826003E0826822F40212FD
:1096600082607047014600208A6802F400120AB145
:10967000012000E000207047F0B5044615460020A8
:1096800000220026092911DDE068A1F10A0707EB95
:10969000470C072707FA0CF29043A1F10A0707EBE2
:1096A000470703FA07F21043E0600CE0206901EB82
:1096B000410C072707FA0CF2904301EB410703FA2C
:1096C00007F210432061A06BC0F30156EF1C06F1B6
:1096D000010CA7EB0C0707EB870C1F2707FA0CF20E
:1096E0009043EF1C06F1010CA7EB0C0707EB870773
:1096F00001FA07F21043A063F0BD10B50A4600213D
:109700000023816B21F44011531E41EA0351816310
:1097100010BD08B5002300930090009B0B440093FC
:10972000009B1A6008BD08B5024600200090009218
:1097300001F12800009B184400900098006880B256
:1097400008BD0A4600214168164B1940114341608B
:1097500070474162826270470A460021416821F0E9
:109760001F0111434160704740B109490831096840
:1097700041F40001064A0832116007E0044908314B
:10978000096821F40001024A0832116070470000A4
:109790000024014000280140003C0140FFFEF0FF92
:1097A000FDF7F1FFFFFD3FFF0246002013680B406D
:1097B0000BB1012000E000207047CA4302607047EF
:1097C00070B502460020002300240B125568CEB26B
:1097D00005EA060415681D4015B10CB1012000E032
:1097E000002070BD00220A12D343036070470000BE
:1097F00001684FF6FE721140016000210160416076
:109800008160C1608D49884208D18C490839496816
:1098100041F00F01894A083A51608AE087491431C2
:10982000884208D185490839496841F0F001834AE6
:10983000083A51607DE081492831884208D17F494A
:109840000839496841F470617C4A083A516070E017
:109850007A493C31884208D178490839496841F44D
:109860007041764A083A516063E074495031884249
:1098700008D172490839496841F470216F4A083AA1
:10988000516056E06D496431884208D16B4908390E
:10989000496841F47001694A083A516049E06749F2
:1098A0007831884208D165490839496841F07061CA
:1098B000624A083A51603CE06149884206D1011F82
:1098C000096841F00F01021F116032E05C49143158
:1098D000884208D15A49091F096841F0F001584AE5
:1098E000121F116025E056492831884208D1544999
:1098F000091F096841F47061514A121F116018E094
:109900004F493C31884208D14D49091F096841F44B
:1099100070414B4A121F11600BE049495031884297
:1099200007D14749091F096841F47021444A121FB1
:109930001160704710B50022026847F6F0739A4331
:109940000C6A8B6823430C6923434C6923438C695D
:109950002343CC6923434C6A23438C6A23431A4331
:109960000260CB6843600B6883604B68C36010BDC6
:109970000021016041608160C160016141618161DC
:10998000C161016241628162704721B1026842F0A7
:109990000102026004E002684FF6FE731A400260A2
:1099A00070471AB103680B43036002E003688B43FE
:1099B00003607047416070470146486880B2704755
:1099C00001460020002201F080531BB11C4B083BD4
:1099D0001A6802E0194B083B1A6802EA01030BB14E
:1099E000012000E00020704700F0805119B11449B7
:1099F000091F086002E011490839486070470146B4
:109A00000020002201F080531BB10D4B083B1A6867
:109A100002E00A4B083B1A6802EA01030BB101207D
:109A200000E00020704700F0805119B10449091F7F
:109A3000086002E0014908394860704708000240A8
:109A400008040240002044490860091D0860091DFF
:109A50000860091D086041483F491431086070479B
:109A600000213D498279002A3AD00A4612680368EB
:109A70009A430B461A600A1D126803689A430B1D2D
:109A80001A60027911440A6803681A430A60324A6C
:109A90000832126803689A432F4B08331A601A1D64
:109AA000126803689A432C4B0C331A604279102ACF
:109AB0000ED11A1F126803681A43274B08331A6025
:109AC0001A1D126803681A43234B0C331A600DE009
:109AD0002149427911440A6803681A430A6005E083
:109AE000027911440A6803689A430A6070470021AA
:109AF000016001710C21417100218171704716498B
:109B0000103109680143144A103211607047014650
:109B10000020114A143212680A400AB1012000E004
:109B2000002070470C49143108607047014600203E
:109B30000022094B1B6803EA0102074B14331B6820
:109B40000B4013B10AB1012000E000207047024928
:109B5000143108607047000000040140FFFF0F004F
:109B600010B50446CC48844208D10121042000F0FD
:109B70004DFB0021042000F049FB46E0C748844229
:109B800008D10121082000F041FB0021082000F04D
:109B90003DFB3AE0C248844208D10121102000F088
:109BA00035FB0021102000F031FB2EE0BD4884423F
:109BB00008D10121202000F029FB0021202000F005
:109BC00025FB22E0B848844208D10121402000F062
:109BD0001DFB0021402000F019FB16E0B348844231
:109BE00008D10121802000F011FB0021802000F02D
:109BF0000DFB0AE0AE48844207D10121801500F038
:109C000005FB0021A01500F001FB10BD10B50121DE
:109C1000084600F0FBFA0021012000F0F7FA10BD21
:109C20002DE9F041024600250026002000230024F3
:109C3000002791F803C00CF00F0591F803C00CF059
:109C4000100CBCF1000F03D091F802C04CEA0505DE
:109C500091F800C0BCF1000F31D0146800202BE057
:109C60004FF0010C0CFA00F3B1F800C00CEA030647
:109C70009E4220D183004FF00F0C0CFA03F7BC4337
:109C800005FA03FC4CEA040491F803C0BCF1280F68
:109C900006D14FF0010C0CFA00FCC2F814C00AE027
:109CA00091F803C0BCF1480F05D14FF0010C0CFA3C
:109CB00000FCC2F810C0401C0828D1D31460B1F8D1
:109CC00000C0BCF1FF0F34DD546800202EE000F12D
:109CD000080C4FF0010808FA0CF3B1F800C00CEAC8
:109CE00003069E4221D183004FF00F0C0CFA03F7BC
:109CF000BC4305FA03FC4CEA040491F803C0BCF130
:109D0000280F05D100F1080C08FA0CF8C2F81480ED
:109D100091F803C0BCF1480F07D100F1080C4FF0D7
:109D2000010808FA0CF8C2F81080401C0828CED3AD
:109D30005460BDE8F0814FF6FF710180022181700F
:109D40000421C17070470246002093680B400BB19C
:109D5000012000E0002070470146886880B270470B
:109D600002460020D3680B400BB1012000E0002028
:109D700070470146C86880B2704701617047416111
:109D800070470AB1016100E041617047C1607047EE
:109D90004FF480320A438261816182618269826903
:109DA000704702460020434B18684FF680731840F6
:109DB00040EA021008433F4B186070473E49C861B3
:109DC0007047F0B50A46002300240021002500F06A
:109DD0000046B6F1004F02D1364EF16901E0354E32
:109DE0007168C0F3034583B200F44016B6F5401F16
:109DF00008D121F070612F4E766826F070662D4FE5
:109E00007E6012E000F48016B6F5801F06D10326AE
:109E100006FA05F4A14341F0706106E0460D3601F3
:109E200003FA06F6B14341F0706122B1460D3601E6
:109E300003FA06F6314300F00046B6F1004F02D1B6
:109E40001C4EF16101E01B4E7160F0BD30B5002287
:109E50008B071C0F0F2303FA04F2164B08338C10E8
:109E600053F824309343134C08348D1044F82530B4
:109E700023468C1053F824308C07240F00FA04F486
:109E800023430C4C08348D1044F8253030BD0A496A
:109E9000DC3108607047000000080140000C014000
:109EA000001001400014014000180140001C014056
:109EB0000020014000000140000020420E490860DF
:109EC00070470D49486070470B49886070474AF6F3
:109ED000AA200949086070474CF6CC400649086042
:109EE000704701460020044AD2680A400AB10120A6
:109EF00000E000207047000000300040DF480068AC
:109F000040F00100DD49086008464068DC4908402F
:109F1000DA49486008460068DA490840D7490860CD
:109F20000846006820F4802008600846406820F455
:109F3000FE0048604FF41F0088607047CF490968F1
:109F400021F48031CD4A11601146096821F4802145
:109F50001160B0F5803F03D0B0F5802F0ED106E040
:109F6000C649096841F48031C44A116007E0C34919
:109F7000096841F4A021C14A116000E000BF00BFA0
:109F8000704710B501460022002300204A11012A23
:109F900002D1BA4C236806E0022A02D1B74C236AE8
:109FA00001E0B64C636A01F01F02012494401C409A
:109FB0000CB1012000E0002010BD38B50020009059
:109FC0000024002500BF3120FFF7DBFF0546009885
:109FD000401C00900098B0F5A06F01D0002DF2D089
:109FE0003120FFF7CEFF08B1012400E00024204615
:109FF00038BD01460020A14A106820F0F80040EA70
:10A00000C10010607047A0490860704702460020F8
:10A010009A4B586820F47C1042EA01031843974B8E
:10A020005860704798490866704701460020934A77
:10A03000506820F003000843506070478F48406824
:10A0400000F00C007047014600208C4A506820F058
:10A05000F00008435060704701460020874A50686E
:10A0600020F4E06008435060704701460020834AB6
:10A07000506820F4605040EAC1005060704729B138
:10A080007E4A527A02437D4B5A7204E07B4A527AEE
:10A0900082437A4B5A7270477B49D83108607047C7
:10A0A00001460020754A506820F440400843506043
:10A0B00070470021714A20321170704A82F82010D6
:10A0C000012802D004280AD104E001216B4A203281
:10A0D000117005E00521694A2032117000E000BFCF
:10A0E00000BF70476949086070476449096A0143C5
:10A0F000624A11627047654944390860704730B55B
:10A1000000210022002400235C4D6D6805F00C0145
:10A1100021B1042905D0082923D105E05C4D056053
:10A1200022E05B4D05601FE0544D6D6805F4701230
:10A13000524D6D6805F48034022505EB92421CB93E
:10A14000544D554305600BE04C4D6D6805F40035EA
:10A150001DB1504D5543056002E04D4D554305601E
:10A1600002E04B4D056000BF00BF444D6D6805F037
:10A17000F0010909484D6B5C0568DD4045603F4DC5
:10A180006D6805F4E061090A434D6B5C4568DD408C
:10A1900085603A4D6D6805F46051C90A3E4D6B5CAF
:10A1A0004568DD40C560354D6D6805F44041890B5B
:10A1B0003A4D6B5CC568B5FBF3F5056130BD29B15F
:10A1C0002E4A526902432D4B5A6104E02B4A5269D0
:10A1D00082432A4B5A61704729B1284A9269024347
:10A1E000264B9A6104E0254A92698243234B9A6187
:10A1F000704729B1214AD2690243204BDA6104E059
:10A200001E4AD26982431D4BDA61704729B11B4A4D
:10A21000D2680243194BDA6004E0184AD2688243DC
:10A22000164BDA60704729B1144A12690243134B86
:10A230001A6104E0114A12698243104B1A61704797
:10A2400012494039086070470F49C86470470B498C
:10A25000C87170470948406A40F0807007494862F9
:10A26000704701460020054A92680A400AB1012061
:10A2700000E00020704701498872704700100240DA
:10A280000000FFF8FFFFF6FE000042428004424259
:10A2900000127A0000093D003C0000204C00002024
:10A2A00010B50446BE48844208D101218014FFF74E
:10A2B000ADFF0021A014FFF7A9FF16E0B9488442C2
:10A2C00008D101210014FFF7AEFF00212014FFF791
:10A2D000AAFF0AE0B448844207D10121C013FFF766
:10A2E000A2FF0021E013FFF79EFF10BD10B5002272
:10A2F000028802F441520B884C8823438C88234304
:10A30000CC8823430C8923434C8923438C892343E2
:10A31000CC8923431A430280838B4FF2FF7423407E
:10A3200083830B8A038210BD2DE9F04F85B005466B
:10A330000C464FF0000902274FF000084FF0010BC8
:10A340000026B246A88B4FF240010840A8830220A5
:10A350002884B5F81C90A068022801D100BF38E01D
:10A36000A08810B94FF0010B01E04FF0020B8D48AF
:10A37000854200D100E000BF6846FFF7C0FEDDF86F
:10A3800000A0E088B0F5007F0AD14FEA1A2000EB68
:10A3900080004000A168B0FBF1F0401D86B20BE0E8
:10A3A0004FEA4B10BAFBF0F000EB80004000A168D0
:10A3B000B0FBF1F0401D86B20A20B6FBF0F606F0C5
:10A3C0000108A6EB0800C0F34F074FF6FF7000EA44
:10A3D0000828022F01DBFF2F02DD02274FF00008C3
:10A3E000E08840EA080038432884A088A18908430F
:10A3F000618808432188084340F4006040EA090965
:10A40000A5F81C9005B0BDE8F08F002101804180C7
:10A410008180C180018141818181C18107210182C7
:10A4200070470021018041808180C18002218160CC
:10A4300000218181704721B1028842F040020280F0
:10A4400004E002884FF6BF731A400280704721B1C2
:10A45000828B42F48062828304E0828B4FF6FF336A
:10A460001A408283704730B5002400230C11012567
:10A47000A540ABB21AB185881D43858002E085886E
:10A480009D43858030BD1AB183880B43838002E0F1
:10A4900083888B4383807047818170470146888918
:10A4A00070474FF6FF62914204D0028842F48072F6
:10A4B000028004E002884FF6FF631A400280704772
:10A4C00021B1828842F00402828004E082884FF643
:10A4D000FB731A408280704702884FF2FF731A4064
:10A4E000028002880A4302807047018841F480514B
:10A4F0000180704721B1028842F40052028004E0DA
:10A5000002884DF6FF731A40028070470246002011
:10A51000012901D0108B00E0908A70470146088A1B
:10A520007047B1F5804F04D1028842F48042028026
:10A5300004E002884BF6FF731A400280704702461F
:10A54000002013890B400BB1012000E00020704770
:10A55000CA4302817047F0B5024600200024002360
:10A56000002501F00F070126BE40B4B20B110126F1
:10A570009E40B3B2968806EA03051689264016B1B6
:10A580000DB1012000E00020F0BD10B5002201F067
:10A590000F040123A3409AB2D343038110BD0000EE
:10A5A0000030014000380040003C004010B5044637
:10A5B000FE48844208D10121C014FFF727FE002184
:10A5C000E014FFF723FEC4E0B4F1804F08D101216D
:10A5D0000846FFF728FE00210120FFF724FEB8E01F
:10A5E000F348844208D101210220FFF71CFE00211C
:10A5F0000220FFF718FEACE0EE48844208D10121AA
:10A600000420FFF710FE00210420FFF70CFEA0E05D
:10A61000E948844208D101210820FFF704FE002107
:10A620000820FFF700FE94E0E448844208D10121AD
:10A630001020FFF7F8FD00211020FFF7F4FD88E05F
:10A64000DF48844208D101212020FFF7ECFD0021E2
:10A650002020FFF7E8FD7CE0DA48844208D10121A0
:10A660004014FFF7D3FD00216014FFF7CFFD70E029
:10A67000D548844209D10121C804FFF7C7FD002154
:10A680004FF40020FFF7C2FD63E0D048844209D1B7
:10A6900001210805FFF7BAFD00214FF48010FFF7F4
:10A6A000B5FD56E0CA48844209D101214805FFF7AB
:10A6B000ADFD00214FF40010FFF7A8FD49E0C548AB
:10A6C000844208D101214020FFF7ADFD0021402048
:10A6D000FFF7A9FD3DE0C048844208D10121802058
:10A6E000FFF7A1FD00218020FFF79DFD31E0BB4871
:10A6F000844208D101218015FFF795FD0021A015A6
:10A70000FFF791FD25E0B648844209D101210804F4
:10A71000FFF77CFD00214FF48030FFF777FD18E054
:10A72000B048844209D101214804FFF76FFD0021A0
:10A730004FF40030FFF76AFD0BE0AB48844208D1CC
:10A7400001218804FFF762FD00214FF48020FFF70C
:10A750005DFD10BD00220288944B98420ED0994BAB
:10A7600098420BD0B0F1804F08D0914B984205D061
:10A77000904B984202D0904B984204D14FF68F7381
:10A780001A404B881A438D4B984207D08C4B984205
:10A7900004D04FF6FF431A40CB881A4302808B88BF
:10A7A00083850B880385814B98420BD0854B98425B
:10A7B00008D08B4B984205D08A4B984202D08A4BE6
:10A7C000984201D10B7A038601238382704770B5CA
:10A7D000002400220023058C4FF6FE7635400584C8
:10A7E000028C8388048B4FF68F752C40B51E2C404D
:10A7F0000D882C43751E2A400D892A434D882A4313
:10A800006A4DA8420BD06F4DA84208D0744DA842A3
:10A8100005D0744DA84202D0734DA84213D14FF613
:10A82000F7752A404D892A434FF6FB752A408D88DB
:10A830002A434FF6FF652B404FF6FF552B408D897D
:10A840002B43CD892B4383800483CD888586028466
:10A8500070BD70B5002400220023058C4FF6EF7602
:10A8600035400584028C8388048B48F6FF752C40A4
:10A870004FF6FF452C400D884FF6FF7606EA05257A
:10A880002C434FF6DF752A400D8906EA05152A4349
:10A890004D8806EA05152A43444DA84202D0494D89
:10A8A000A8421DD14FF67F752A404D894FF6FF769D
:10A8B00006EA05152A434FF6BF752A408D8806EA39
:10A8C00005152A434FF6FF352B404FF2FF752B40FD
:10A8D0008D8906EA85052B43CD8906EA85052B433C
:10A8E00083800483CD880587028470BD70B5002401
:10A8F00000220023058C4FF6FF6635400584028C4C
:10A900008388848B4FF68F752C404FF6FC752C4056
:10A910000D882C434FF6FF552A400D894FF6FF76E0
:10A9200006EA05252A434D8806EA05252A431F4DD8
:10A93000A84202D0234DA8421DD14FF2FF752A40F4
:10A940004D894FF6FF7606EA05252A434FF6FF3577
:10A950002A408D8806EA05252A434EF6FF752B40CE
:10A960004DF6FF752B408D8906EA05152B43CD89E1
:10A9700006EA05152B4383808483CD88858702846E
:10A9800070BD70B5002200230024058C4EF6FF76C2
:10A9900035400584038C8488828B48F6FF752A40F5
:10A9A0004FF6FF452A400D8820E00000002C0140B2
:10A9B0000004004000080040000C0040001000406F
:10A9C0000014004000340140004C014000500140A0
:10A9D0000054014000180040001C004000200040CE
:10A9E0000040014000440140004801404FF6FF761E
:10A9F00006EA05252A434DF6FF752B400D8906EA28
:10AA000005352B434D8806EA05352B43FA4DA84200
:10AA100002D0FA4DA84208D14BF6FF752C408D8923
:10AA20004FF6FF7606EA85152C4384808283CD8815
:10AA3000A0F84050038470BD828B4FF2FF331A4060
:10AA40008283828B4FF6FF7303EA01231A438283CA
:10AA50007047F0B50C461546002200210026078CF1
:10AA60004EF6FF7C07EA0C070784828B018C4FF6B9
:10AA7000FF7707EA043640F6FF473A404FF6FF7784
:10AA800007EA05273A434FF6FF7707EA03373A43C9
:10AA9000D94FB8420ED0D94FB8420BD0B0F1804F49
:10AAA00008D0D74FB84205D0D64FB84202D0D64FC3
:10AAB000B84206D14DF6FF77394046F48057394306
:10AAC00005E047F6FF57394044F480573943828305
:10AAD0000184F0BD828B4FF6F3731A408283828B20
:10AAE0000A4382837047F0B50C46154600220021C8
:10AAF0000026078C4FF6FF6C07EA0C070784828B51
:10AB0000018C4FF6FF7707EA04264FF60C773A40A0
:10AB10004FF6FF7707EA03172F433A43B64FB84281
:10AB20000ED0B64FB8420BD0B0F1804F08D0B44F22
:10AB3000B84205D0B34FB84202D0B34FB84206D1A5
:10AB40004FF6FF57394046F48077394305E04FF21E
:10AB5000FF57394044F48077394382830184F0BD44
:10AB6000028B4FF2FF331A400283028B4FF6FF73C2
:10AB700003EA01231A4302837047F0B50C461546D9
:10AB8000002200210026078C4FF6EF7C07EA0C0715
:10AB90000784028B018C4FF6FF7707EA041640F614
:10ABA000FF473A404FF6FF7707EA03373A434FF63D
:10ABB000FF7707EA05273A438F4FB8420ED08F4FF1
:10ABC000B8420BD0B0F1804F08D08D4FB84205D0BD
:10ABD0008C4FB84202D08C4FB84206D14FF6DF7787
:10ABE000394046F01007394305E04FF65F773940AA
:10ABF00044F01007394302830184F0BD028B4FF605
:10AC0000F3731A400283028B0A4302837047F0B544
:10AC10000C46154600220021068C4FF6FE773E407A
:10AC20000684028B018C4FF60C7632407E1C06EABD
:10AC300003162E433243704EB0420ED06F4EB042D8
:10AC40000BD0B0F1804F08D06D4EB04205D06D4EA4
:10AC5000B04202D06C4EB04206D14FF6FD76314084
:10AC600044F00106314305E04FF6F576314044F0FB
:10AC70000106314302830184F0BD70B505460C46E0
:10AC80005D4885420ED05D4885420BD0B5F1804FBE
:10AC900008D05B48854205D05A48854202D05A48C0
:10ACA000854200D100E000BF208850B92389A288E6
:10ACB00061882846FFF7ABFFE1882846FFF79EFF33
:10ACC00025E0208804280AD12389A28861882846A3
:10ACD000FFF753FFE1882846FFF742FF17E020887F
:10ACE00008280AD12389A28861882846FFF7FBFE3D
:10ACF000E1882846FFF7EEFE09E02389A2886188F3
:10AD00002846FFF7A6FEE1882846FFF795FE70BDAE
:10AD10002DE9F04105460C4600260127608808B958
:10AD2000022600E00026A088012801D1022700E0C9
:10AD300001272088A0B92389A28861882846FFF7C7
:10AD400066FFE1882846FFF759FF23893A463146D6
:10AD50002846FFF712FFE1882846FFF701FF13E0BE
:10AD60002389A28861882846FFF707FFE1882846E3
:10AD7000FFF7F6FE23893A4631462846FFF747FF9C
:10AD8000E1882846FFF73AFFBDE8F0810A884B8842
:10AD90001A438B881A43CB881A430B891A434B8971
:10ADA0001A438B891A43A0F8442070474FF6FF716D
:10ADB000818000210180C1804180017270470021A3
:10ADC000018041808180C180018141818181C18177
:10ADD0007047002101804180012181800021C180D4
:10ADE000018170470021018041808180C180018103
:10ADF0004181818170470000002C014000340140F6
:10AE00000004004000080040000C004021B102880E
:10AE100042F00102028004E002884FF6FE731A40FD
:10AE20000280704731B1B0F8442042F40042A0F8EB
:10AE3000442005E0B0F84420C2F30E02A0F84420FC
:10AE400070471AB183890B43838102E083898B4366
:10AE5000838170478182704741EA0203A0F848303D
:10AE600070471AB183890B43838102E083898B4346
:10AE70008381704701894FF6F87211400181704754
:10AE80000A46002101894FF68F7319401143018151
:10AE9000704730B504460D4629462046FFF7F0FFBF
:10AEA000208940F00700208130BD2DE9F0410446A3
:10AEB0000D4616461F46602D06D13B4601223146FF
:10AEC0002046FFF75AFE05E03B4601223146204668
:10AED000FFF79DFE29462046FFF7D2FF208940F06C
:10AEE00007002081BDE8F08130B50C4600210189C2
:10AEF000C9B24FF6FF7505EA0325154325432943DB
:10AF0000018130BD2DE9F04105460E4617469846B1
:10AF1000002443463A4631462846FFF7E5FF2C8990
:10AF20004FF6F870044044F007044FF68F70044069
:10AF300044F070042C81BDE8F081F0B504460D4664
:10AF400016461F463B46324629462046FFF7CCFFB1
:10AF5000208940F480402081F0BD018582827047C5
:10AF60000A46002101884FF68F7319401143018072
:10AF70007047F0B50C4615461E46002100220023FE
:10AF80000189028B038C4FF6F877394021434FF645
:10AF9000FC473A4040F201173A434FF6DD773B4019
:10AFA0004FF6FF7707EA06172F433B4301810283E1
:10AFB0000384F0BD0A460021018B4FF68F731940C0
:10AFC0001143018370470A460021018B48F6FF7345
:10AFD00019404FF6FF7303EA0223194301837047B8
:10AFE0000A460021818B4FF68F73194011438183EC
:10AFF00070470A460021818B48F6FF7319404FF6CF
:10B00000FF7303EA022319438183704721B1028849
:10B0100042F08002028004E002884FF67F731A40FB
:10B020000280704721B1828842F00402828004E0ED
:10B0300082884FF6FB731A408280704721B1828864
:10B0400042F00802828004E082884FF6F7731A40CB
:10B050008280704721B1828842F00102828004E040
:10B0600082884FF6FE731A40828070470A4600219C
:10B07000018B4FF6F77319401143018370470A465D
:10B080000021018B4FF2FF7319404FF6FF7303EA63
:10B0900002231943018370470A460021818B4FF632
:10B0A000F77319401143818370470A460021818B51
:10B0B0004FF2FF7319404FF6FF7303EA022319435F
:10B0C000818370470A460021018B4FF6FB731940BC
:10B0D0001143018370470A460021018B4FF6FF336D
:10B0E00019404FF6FF7303EA0223194301837047A7
:10B0F0000A460021818B4FF6FB731940114381836F
:10B1000070470A460021818B4FF6FF3319404FF6F6
:10B11000FF7303EA02231943818370470A46002123
:10B12000018B4FF67F7319401143018370470A4624
:10B130000021018BC1F30E014FF6FF7303EA0223D6
:10B140001943018370470A460021818B4FF67F73B4
:10B1500019401143818370470A460021818BC1F356
:10B160000E014FF6FF7303EA0223194381837047F0
:10B170000A460021018C4FF6FD73194011430184EA
:10B1800070470A460021018C4FF6F77319401143AE
:10B19000018470470A460021018C4FF6DF73194085
:10B1A0004FF6FF7303EA02131943018470470A46FE
:10B1B0000021018C4FF67F7319404FF6FF7303EAAD
:10B1C00002131943018470470A460021018C4FF68F
:10B1D000FF5319404FF6FF7303EA0223194301841A
:10B1E00070470A460021018C4FF2FF7319404FF659
:10B1F000FF7303EA02231943018470470A460021C2
:10B20000018C4DF6FF7319404FF6FF7303EA0233CA
:10B2100019430184704730B5002301248C40A3B248
:10B22000048C9C430484048C02FA01F5ADB22C43D7
:10B23000048430BD30B5002304248C40A3B2048CB8
:10B240009C430484048C02FA01F5ADB22C430484BF
:10B2500030BD70B503460020002418461830012583
:10B260008D40ACB21D8CA5431D8409B1082909D1BC
:10B2700000EB6100056825F0700505600568154361
:10B2800005600EE00D1FC5F34E052844056825F442
:10B29000E045056005684FF6FF7606EA022635436D
:10B2A000056070BD21B1028842F00202028004E014
:10B2B00002884FF6FD731A400280704721B1028860
:10B2C00042F00402028004E002884FF6FB731A4049
:10B2D0000280704721B1828842F08002828004E0BF
:10B2E00082884FF67F731A408280704702884FF63B
:10B2F000F7731A40028002880A43028070478288EE
:10B300004FF68F731A40828082880A43828070478A
:10B3100002894FF6F8731A40028102890A430281BA
:10B32000704702894FF67F731A40028102890A43EF
:10B33000028170478184704781857047818670479C
:10B340000187704781877047A0F8401070470288D6
:10B350004FF6FF431A40028002880A43028070477A
:10B360000146888E70470146088F70470146888FD6
:10B3700070470146B1F8400070470146888C70471D
:10B380000146088D704702460020138A0B400BB11E
:10B39000012000E000207047CA430282704730B5A8
:10B3A0000246002000230024158A05EA010395893E
:10B3B00005EA010413B10CB1012000E0002030BD0A
:10B3C000CA4302827047000010B50446FB4884421D
:10B3D00009D101218803FEF719FF00214FF48040B5
:10B3E000FEF714FF32E0F648844209D101214804F7
:10B3F000FEF719FF00214FF40030FEF714FF25E09F
:10B40000F048844209D101218804FEF70CFF002195
:10B410004FF48020FEF707FF18E0EB48844209D183
:10B420000121C804FEF7FFFE00214FF40020FEF7C3
:10B43000FAFE0BE0E548844208D101210805FEF739
:10B44000F2FE00214FF48010FEF7EDFE10BD2DE955
:10B45000F04786B005460E460024A24600BFA1462E
:10B460000027B08900B100BF2F462C8A4CF6FF7030
:10B470000440F08804432C82AC894EF6F31004405B
:10B48000B08831890843718908430443AC81AC8A90
:10B490004FF6FF400440B0890443AC8201A8FEF798
:10B4A0002EFEC648874202D1DDF810A001E0DDF88B
:10B4B0000CA0A88900F4004040B10AEBCA0000EBE0
:10B4C0000A1031684900B0FBF1F807E00AEBCA0046
:10B4D00000EB0A1031688900B0FBF1F86420B8FB7A
:10B4E000F0F004012009642101FB1089A88900F40F
:10B4F000004040B1322000EBC900B0FBF1F000F099
:10B500000700044308E0322000EB09106421B0FB7F
:10B51000F1F000F00F0004432C8106B0BDE8F08785
:10B520004FF41651016000218180C18001810C21FE
:10B53000418100218181704710B502460020108AA8
:10B540004FF2FF0318400B884C8823438C88234319
:10B55000CC8823431843108210BD00210180418014
:10B560008180C180704721B1828942F4005282817A
:10B5700004E082894DF6FF731A4082817047F0B56E
:10B580000346002400260025002040F66A17B94231
:10B5900000D100BF1846C1F3421401F01F06012775
:10B5A00007FA06F5012C01D10C3004E0022C01D180
:10B5B000103000E014301AB107682F43076002E032
:10B5C0000768AF430760F0BD1AB1838A0B438382DB
:10B5D00002E0838A8B4383827047028A4FF6F073BE
:10B5E0001A400282028A0A430282704782894FF21D
:10B5F000FF731A40828182890A438281704721B198
:10B60000828942F00202828104E082894FF6FD7352
:10B610001A4082817047028A4FF6DF731A40028215
:10B62000028A0A430282704721B1028A42F48042B0
:10B63000028204E0028A4BF6FF731A4002827047CE
:10B64000C1F308028280704701468888C0F3080071
:10B650007047818941F0010181817047028BD2B22C
:10B660000283028B42EA012202837047028B02F4BA
:10B670007F420283028B0A430283704721B1828A90
:10B6800042F02002828204E0828A4FF6DF731A4081
:10B690008282704721B1828A42F01002828204E0E5
:10B6A000828A4FF6EF731A408282704721B1828AF4
:10B6B00042F00802828204E0828A4FF6F7731A4051
:10B6C0008282704721B1828942F40042828103E084
:10B6D0008289C2F30E028281704721B1828A42F4CC
:10B6E0000062828204E0828A4FF2FF731A408282F3
:10B6F0007047828A4FF6FB731A408282828A0A431D
:10B700008282704721B1828A42F00202828204E082
:10B71000828A4FF6FD731A408282704702460020EB
:10B72000B1F5007F00D100BF13880B400BB10120A1
:10B7300000E00020704701F40072B2F5007F00D1F4
:10B7400000BFCA430280704770B502460024002340
:10B750000025002040F66A16B14200D100BFC1F3B7
:10B76000421501F01F03012606FA03F3012D02D151
:10B770009689334006E0022D02D1168A334001E05B
:10B78000968A33400C12012606FA04F416883440D7
:10B7900013B10CB1012000E0002070BD10B50022F3
:10B7A000002340F66A14A14200D100BF0A1201240E
:10B7B0009440A3B2DC43048010BD00000038014077
:10B7C0000044004000480040004C00400050004051
:10B7D0000948804709480047FEE7FEE7FEE7FEE725
:10B7E000FEE7FEE7FEE7FEE7FEE7FEE70448054961
:10B7F000054A064B70470000C391000831810008DC
:10B80000A8C80020A8DA0020A8CA0020A8CA0020E2
:10B8100008B5FE48C07B002817DC01214020FEF758
:10B82000DBFC4FF6FF70ADF8000010208DF8030030
:10B8300003208DF802006946F548FEF7F1F9BDF8DE
:10B840000010F348FEF79BFA53E001214420FEF775
:10B85000C3FC49F6FF70ADF8000010208DF803001E
:10B8600003208DF802006946E948FEF7D9F9BDF8D2
:10B870000010E748FEF783FA4FF44050ADF800009F
:10B8800010208DF8030003208DF802006946E1487E
:10B89000FEF7C6F9BDF80010DE48FEF770FA012188
:10B8A0003020FEF799FC40F69B70ADF800001020A8
:10B8B0008DF8030003208DF802006946D648FEF794
:10B8C000AFF9BDF80010D448FEF759FA4FF4005014
:10B8D000ADF8000010208DF8030003208DF8020061
:10B8E0006946CE48FEF79CF9BDF80010CB48FEF73C
:10B8F00046FA08BDCA480088401CC9490880084665
:10B90000008819281BDB00200880C648007818B979
:10B910000120C449087002E00020C2490870C148F3
:10B92000007830B9C048006820F40050BE49086073
:10B9300005E0BD48006840F40050BB4908600020A5
:10B94000BA490870FEE3B9480078C0EBC00101EBCA
:10B950000010B74901EB400090F82D0048B9B348FA
:10B96000017801208840B04909680843AE49086061
:10B9700016E2AE480078C0EBC00101EB0010AC4904
:10B9800001EB400090F82800002859D1A748007822
:10B99000C0EBC00101EB0010A54901EB400090F89D
:10B9A0002D0001282CDBA1480078C0EBC00101EB81
:10B9B00000109F4901EB400090F82D000B281FDC80
:10B9C0009A480078C0EBC00101EB0010984901EBE8
:10B9D000400090F8260048B1944801780120884042
:10B9E00091490968814390480160D9E18F48017805
:10B9F000012088408C49096808438B490860CFE1E1
:10BA00008A480078C0EBC00101EB0010884901EBC7
:10BA1000400090F8260048B1844801780120884011
:10BA200081490968084380490860B9E17F48017885
:10BA3000012088407C49096881437B480160AFE16F
:10BA40007A480078C0EBC00101EB0010784901EBA7
:10BA5000400090F82D000F280CD074480078C0EBFF
:10BA6000C00101EB0010724901EB400090F82D007D
:10BA700019281ED16F486D490978405C01280ED104
:10BA80006A4801780120884067490968814366480F
:10BA9000016000206749654A1278885480E1634854
:10BAA0000178012088406049096808435E490860C0
:10BAB00076E15E480078C0EBC00101EB00105C4904
:10BAC00001EB400090F82D0001282DDB574800784D
:10BAD000C0EBC00101EB0010554901EB400090F8AC
:10BAE0002D000A2820DC51480078C0EBC00101EB92
:10BAF00000104F4901EB4000D0F81E00002809DB80
:10BB00004A480178012088404749096881434648EE
:10BB1000016045E1454801780120884042490968B3
:10BB20000843414908603BE140480078C0EBC00150
:10BB300001EB00103E4901EB400090F82D00132866
:10BB400022D13A480078C0EBC00101EB001038491F
:10BB500001EB4000D0F81E0041F28831884209DB39
:10BB600032480178012088402F49096881432E48D6
:10BB7000016015E12D480178012088402A490968B3
:10BB80000843294908600BE128480078C0EBC00150
:10BB900001EB0010264901EB400090F82D000B2826
:10BBA00022D122480078C0EBC00101EB00102049EF
:10BBB00001EB4000D0F81E0040F6C411884209DBBA
:10BBC0001A480178012088401749096881431648BE
:10BBD0000160E5E0154801780120884012490968B4
:10BBE000084311490860DBE010480078C0EBC00151
:10BBF00001EB00100E4901EB400090F82D000B28DE
:10BC000039D10A480078C0EBC00115E05860002027
:10BC100000180140000801400014014000100140DC
:10BC20005E0000205800002054000020600000202A
:10BC3000E76C00202017002001EB0010FE4901EB0B
:10BC40004000D0F81E0040F6C411884209DBFB48D2
:10BC5000017801208840FA4909688143F848016069
:10BC60009EE0F648017801208840F54909680843BC
:10BC7000F349086094E0F1480078C0EBC00101EBA3
:10BC80000010ED4901EB400090F82D000D2822D165
:10BC9000EA480078C0EBC00101EB0010E64901EB77
:10BCA0004000D0F81E0042F21071884209DBE348E0
:10BCB000017801208840E24909688143E048016039
:10BCC0006EE0DE48017801208840DD4909680843BC
:10BCD000DB49086064E0D9480078C0EBC00101EBA3
:10BCE0000010D54901EB400090F82D00102819D024
:10BCF000D2480078C0EBC00101EB0010CE4901EB47
:10BD0000400090F82D0012280CD0CC480078C0EBF1
:10BD1000C00101EB0010C84901EB400090F82D0074
:10BD2000112822D1C5480078C0EBC00101EB0010FA
:10BD3000C14901EB4000D0F81E004CF2503188425E
:10BD400009DBBE48017801208840BD49096881436C
:10BD5000BB48016024E0B948017801208840B84917
:10BD600009680843B64908601AE0B648B34909783B
:10BD700030F81100B0F5006F09DDB04801780120FE
:10BD80008840AF4909688143AD48016008E0AB488D
:10BD9000017801208840AA4909680843A849086039
:10BDA000A64800780B30C0EBC00101EB0010A2499F
:10BDB00001EB400090F82D0048B9A048017801201F
:10BDC0008840A149096808439F490860EFE19B4802
:10BDD00000780B30C0EBC00101EB0010964901EB7D
:10BDE000400090F8280090BB944800780B30C0EBDE
:10BDF000C00101EB0010904901EB400090F82D00CC
:10BE000001282FDB8D4800780B30C0EBC00101EB1F
:10BE10000010894901EB400090F82D000B2821DC2F
:10BE2000864800780B30C0EBC00101EB001082495E
:10BE300001EB400090F8260050B1804801780120C5
:10BE400088408149096881437F480160AFE12AE069
:10BE50007A480178012088407B49096808437A497B
:10BE60000860A4E1754800780B30C0EBC00101EB1D
:10BE70000010714901EB400090F8260048B16F486E
:10BE80000178012088407049096808436E490860BC
:10BE90008DE16A480178012088406B490968814337
:10BEA0006948016083E1654800780B30C0EBC00150
:10BEB00001EB0010604901EB400090F82D000F28C5
:10BEC0000DD05E4800780B30C0EBC00101EB0010D4
:10BED000594901EB400090F82D0019281CD159490F
:10BEE000564800780B3031F81000B0F5006F09DAD1
:10BEF00052480178012088405349096881435248DB
:10BF0000016054E14D480178012088404E4909689C
:10BF100008434D4908604AE1484800780B30C0EBBF
:10BF2000C00101EB0010444901EB400090F82D00E6
:10BF300001282FDB414800780B30C0EBC00101EB3A
:10BF400000103D4901EB400090F82D000A2821DC4B
:10BF50003A4800780B30C0EBC00101EB00103649C5
:10BF600001EB4000D0F81E00002809DB33480178BF
:10BF7000012088403449096881433348016016E153
:10BF80002E480178012088402F49096808432E492E
:10BF900008600CE1294800780B30C0EBC00101EBD0
:10BFA0000010254901EB400090F82D00132823D103
:10BFB000224800780B30C0EBC00101EB00101E4995
:10BFC00001EB4000D0F81E0041F28831884209DBC5
:10BFD0001A480178012088401B49096881431A48A2
:10BFE0000160E4E01548017801208840164909689D
:10BFF000084315490860DAE0104800780B30C0EBC0
:10C00000C00101EB00100C4901EB400090F82D003D
:10C010000B282ED1094800780B30C0EBC00101EB92
:10C020000010054901EB4000D0F81E0040F6C41195
:10C03000884214DB014809E0E76C00206000002022
:10C0400054000020E016002050000020017801205C
:10C050008840F74909688143F5480160A7E0F54841
:10C06000017801208840F24909680843F0490860D6
:10C070009DE0F04800780B30C0EBC00101EB0010F0
:10C08000ED4901EB400090F82D000D2823D1E9483F
:10C0900000780B30C0EBC00101EB0010E64901EB6A
:10C0A0004000D0F81E0042F21071884209DBE148DE
:10C0B000017801208840DE4909688143DC4801603D
:10C0C00075E0DC48017801208840D94909680843B7
:10C0D000D74908606BE0D74800780B30C0EBC0014F
:10C0E00001EB0010D44901EB400090F82D0010281E
:10C0F0001BD0D04800780B30C0EBC00101EB001022
:10C10000CD4901EB400090F82D0012280DD0C94810
:10C1100000780B30C0EBC00101EB0010C64901EB09
:10C12000400090F82D00112825D1C24800780B302E
:10C13000C0EBC00101EB0010BF4901EB4000D0F89B
:10C140001E0000E038E04CF25031884209DBB9486B
:10C15000017801208840B64909688143B4480160EC
:10C1600025E0B448017801208840B14909680843B6
:10C17000AF4908601BE0B149AE4800780B3031F898
:10C180001000B0F5006F09DDAA4801780120884051
:10C19000A74909688143A648016008E0A5480178DD
:10C1A00001208840A24909680843A1490860A148C4
:10C1B0000078401C9F4908709E4800780B28FFF6C5
:10C1C000C2AB16209B49087028E29A480078C0EB61
:10C1D000C00101EB0010984901EB400090F82D00E0
:10C1E00058B9944800780838012101FA00F09449C0
:10C1F00009680843924908600BE28E480078C0EB5A
:10C20000C00101EB00108C4901EB400090F82800C0
:10C2100080BB88480078C0EBC00101EB0010864964
:10C2200001EB400090F82D00012830DB81480078B8
:10C23000C0EBC00101EB00107F4901EB400090F81A
:10C240002D000B2823DC7B480078C0EBC00101EBFC
:10C250000010794901EB400090F8260058B175486C
:10C260000078083801218140754800688843744986
:10C270000860CEE12EE06F4800780838012101FA0D
:10C2800000F06F49096808436D490860C1E16948D9
:10C290000078C0EBC00101EB0010674901EB4000E2
:10C2A00090F8260058B1634800780838012101FA57
:10C2B00000F063490968084361490860A9E15D48E5
:10C2C00000780838012181405D48006888435C4956
:10C2D00008609EE157480078C0EBC00101EB0010F8
:10C2E000554901EB400090F82D000F280CD0514823
:10C2F0000078C0EBC00101EB00104F4901EB40009A
:10C3000090F82D00192821D14E484A490978405CFF
:10C3100001280FD14748007808380121814048485A
:10C32000006888434649086000204649414A12781F
:10C3300088546EE13F4800780838012101FA00F086
:10C340003F49096808433E49086062E1394800787E
:10C35000C0EBC00101EB0010374901EB400090F841
:10C360002D00012830DB33480078C0EBC00101EB21
:10C370000010314901EB400090F82D000A2823DC21
:10C380002C480078C0EBC00101EB00102A4901EBFA
:10C390004000D0F81E0000280ADB26480078083844
:10C3A000012181402648006888432549086030E122
:10C3B000204800780838012101FA00F02049096876
:10C3C00008431F49086024E11A480078C0EBC00107
:10C3D00001EB0010184901EB400090F82D001328E4
:10C3E00032D114480078C0EBC00101EB00101249B3
:10C3F00001EB4000D0F81E0041F2883188420ADB90
:10C400000C4800780838012181400D4800688843B5
:10C410000B490860FDE0074800780838012101FA5F
:10C4200000F007490968084305490860F1E0000089
:10C430005000002060000020E76C0020E016002083
:10C440005400002020170020F8480078C0EBC001FD
:10C4500001EB0010F64901EB400090F82D000B288D
:10C4600025D1F2480078C0EBC00101EB0010F04983
:10C4700001EB4000D0F81E0040F6C41188420ADBF0
:10C48000EA480078083801218140EA48006888437A
:10C49000E8490860BDE0E54800780838012101FA64
:10C4A00000F0E44909680843E2490860B1E0DF4868
:10C4B0000078C0EBC00101EB0010DD4901EB40004A
:10C4C00090F82D000B2825D1D8480078C0EBC0018A
:10C4D00001EB0010D64901EB4000D0F81E0040F6F9
:10C4E000C41188420ADBD148007808380121814014
:10C4F000D04800688843CF4908608AE0CB4800787C
:10C500000838012101FA00F0CA4909680843C949FD
:10C5100008607EE0C5480078C0EBC00101EB001068
:10C52000C34901EB400090F82D000D2825D1BF48EC
:10C530000078C0EBC00101EB0010BD4901EB4000E9
:10C54000D0F81E0042F2107188420ADBB74800782A
:10C55000083801218140B74800688843B549086020
:10C5600057E0B24800780838012101FA00F0B149DB
:10C5700009680843AF4908604BE0AC480078C0EB5D
:10C58000C00101EB0010AA4901EB400090F82D001A
:10C59000102819D0A5480078C0EBC00101EB0010AD
:10C5A000A34901EB400090F82D0012280CD09F48C1
:10C5B0000078C0EBC00101EB00109D4901EB400089
:10C5C00090F82D00112824D198480078C0EBC001C4
:10C5D00001EB0010964901EB4000D0F81E004CF230
:10C5E000503188420ADB91480078083801218140A7
:10C5F0009048006888438F4908600AE08B480078BB
:10C600000838012101FA00F08A490968084389497C
:10C61000086086480078401C844908708348007888
:10C620001B28FFF6D2AD1B208049087025E27F4809
:10C630000078C0EBC00101EB00107D4901EB400028
:10C6400090F82D0058B9794800780D38012101FA89
:10C6500000F07949096808437749086008E273489F
:10C660000078C0EBC00101EB0010714901EB400004
:10C6700090F8280080BB6D480078C0EBC00101EB4A
:10C6800000106B4901EB400090F82D00012830DBD1
:10C6900066480078C0EBC00101EB0010644901EB73
:10C6A000400090F82D000B2823DC60480078C0EB98
:10C6B000C00101EB00105E4901EB400090F826003C
:10C6C00058B15A4800780D38012181405A48006815
:10C6D000884359490860CBE12EE0544800780D3872
:10C6E000012101FA00F054490968084352490860E1
:10C6F000BEE14E480078C0EBC00101EB00104C4990
:10C7000001EB400090F8260058B1484800780D38F9
:10C71000012101FA00F048490968084346490860C8
:10C72000A6E1424800780D38012181404248006866
:10C730008843414908609BE13C480078C0EBC00158
:10C7400001EB00103A4901EB400090F82D000F2852
:10C750000CD036480078C0EBC00101EB0010344922
:10C7600001EB400090F82D00192821D133482F49C2
:10C770000978405C01280FD12C4800780D38012140
:10C7800081402D48006888432B49086000212B48D0
:10C79000264A127881546BE1244800780D38012133
:10C7A00001FA00F0244909680843234908605FE161
:10C7B0001E480078C0EBC00101EB00101C4901EBE2
:10C7C000400090F82D0001283ADB18480078C0EBB3
:10C7D000C00101EB0010164901EB400090F82D005C
:10C7E0000A282DDC11480078C0EBC00101EB0010D5
:10C7F0000F4901EB4000D0F81E0000280ADB0B486F
:10C8000000780D38012181400B48006888430A49AF
:10C8100008602DE1054800780D38012101FA00F08B
:10C820000549096808430449086021E160000020C7
:10C83000E76C00205400002050000020201700204A
:10C84000FC480078C0EBC00101EB0010FA4901EB95
:10C85000400090F82D00132825D1F6480078C0EB51
:10C86000C00101EB0010F44901EB4000D0F81E00BC
:10C8700041F2883188420ADBEE4800780D38012108
:10C880008140EE4800688843EC490860F0E0E948E0
:10C8900000780D38012101FA00F0E84909680843E1
:10C8A000E6490860E4E0E3480078C0EBC00101EB32
:10C8B0000010E14901EB400090F82D000B2825D134
:10C8C000DC480078C0EBC00101EB0010DA4901EB55
:10C8D0004000D0F81E0040F6C41188420ADBD5485B
:10C8E00000780D3801218140D44800688843D3493D
:10C8F0000860BDE0CF4800780D38012101FA00F052
:10C90000CE4909680843CD490860B1E0C9480078BC
:10C91000C0EBC00101EB0010C74901EB400090F8EB
:10C920002D000B2825D1C3480078C0EBC00101EBD6
:10C930000010C14901EB4000D0F81E0040F6C411C0
:10C9400088420ADBBB4800780D3801218140BB4892
:10C9500000688843B94908608AE0B64800780D3815
:10C96000012101FA00F0B54909680843B34908609C
:10C970007EE0B0480078C0EBC00101EB0010AE498A
:10C9800001EB400090F82D000D2825D1A948007832
:10C99000C0EBC00101EB0010A74901EB4000D0F84B
:10C9A0001E0042F2107188420ADBA24800780D385E
:10C9B00001218140A14800688843A049086057E0F0
:10C9C0009C4800780D38012101FA00F09B49096864
:10C9D00008439A4908604BE096480078C0EBC001D4
:10C9E00001EB0010944901EB400090F82D00102855
:10C9F00019D090480078C0EBC00101EB00108E49BF
:10CA000001EB400090F82D0012280CD089480078E6
:10CA1000C0EBC00101EB0010874901EB400090F82A
:10CA20002D00112824D183480078C0EBC00101EB10
:10CA30000010814901EB4000D0F81E004CF250314B
:10CA400088420ADB7B4800780D38012181407B4811
:10CA500000688843794908600AE0764800780D3814
:10CA6000012101FA00F0754909680843734908601B
:10CA700070480078401C6F4908706E480078202884
:10CA8000FFF6D5AD6E480078002804DD6C480078CC
:10CA9000401E6B4908706B480078002804DD694827
:10CAA0000078401E6749087065480078002806DD58
:10CAB0006248006820F480506049086005E05F48E3
:10CAC000006840F480505D4908605E4800780028A6
:10CAD00006DD5A48006820F400605849086005E007
:10CAE0005648006840F40060544908605648007891
:10CAF000002804DD54480078401E5349087053480C
:10CB00000078002804DD51480078401E4F49087025
:10CB10004D480078002806DD4D48006820F400608C
:10CB20004B49086005E04A48006840F40060484905
:10CB3000086046480078002806DD4548006820F473
:10CB400080504349086005E04148006840F4805047
:10CB50003F490860704710B53E48007808B9012089
:10CB600000E000203B4908700846007800287BD090
:10CB70003948C07B002806DC3048008881B237483D
:10CB8000FDF704F93EE201203549086000203549EF
:10CB9000C1F8B0012948007800F0010020B101205F
:10CBA0002F493C39086003E000202D493C390860DA
:10CBB0002248007800F0020020B1012028493839CD
:10CBC000086003E000202649383908601B480078D7
:10CBD00000F0040020B1012021493439086003E04D
:10CBE00000201F49343908601448007800F008001C
:10CBF00020B101201A493039086003E000201849AB
:10CC0000303908600D48007800F0100020B1012094
:10CC100013492C39086003E0002011492C390860C1
:10CC20000648007800F02000F8B101200C492839AE
:10CC300008601DE060000020E76C0020500000202C
:10CC40005B0000205C000020590000205A000020FA
:10CC500054000020610000205860002000180140AE
:10CC6000BC01234200002142B3E00020E6490860F5
:10CC7000E648007800F0400020B10120E249091D9B
:10CC8000086003E00020E049091D0860DF480078E3
:10CC900000F0800020B10120DB490831086003E08A
:10CCA0000020D94908310860D848008800F4807015
:10CCB00020B10120D4490C31086003E00020D249A2
:10CCC0000C310860D148008800F4007020B10120C8
:10CCD000CD491031086003E00020CB4910310860D5
:10CCE000CA48008800F4806020B10120C649143190
:10CCF000086003E00020C44914310860C34800887C
:10CD000000F4006020B10120BF491831086003E041
:10CD10000020BD4918310860BC48008800F48050EC
:10CD200020B10120B8491C31086003E00020B64959
:10CD30001C310860B548008800F4005018B101208B
:10CD4000B349086002E00020B1490860AF480068BC
:10CD500000F4802018B10120AE49086002E00020F4
:10CD6000AC490860A948006800F4003020B10120F7
:10CD7000A849091D086003E00020A649091D0860B4
:10CD8000A248006800F4803020B10120A149083198
:10CD9000086003E000209F49083108609B48008834
:10CDA00000F4004020B101209A490C31086003E0F2
:10CDB000002098490C3108609448008800F48040B5
:10CDC00018B10120944908601CE1002092490860D4
:10CDD00018E19248C07B002806DC9148008881B2A7
:10CDE0009048FCF7D3FF0DE1002087492831086007
:10CDF00001208D49C1F8B0018948007800F0010098
:10CE000020B1012080491439086003E000207E49E8
:10CE1000143908608248007800F0020020B1012037
:10CE200079491039086003E000207749103908601B
:10CE30007B48007800F0040020B1012072490C39D1
:10CE4000086003E0002070490C39086074480078DD
:10CE500000F0080020B101206B490839086003E0A8
:10CE600000206949083908606D48007800F010001A
:10CE700020B101206449091F086003E000206249D5
:10CE8000091F08606648007800F0200018B10120F2
:10CE90005D49086002E000205B4908606048007856
:10CEA00000F0400020B101205749091D086003E04F
:10CEB00000205549091D08605948007800F080009D
:10CEC00020B1012050490831086003E000204E499C
:10CED000083108605248008800F4807020B10120B9
:10CEE00049490C31086003E0002047490C310860D3
:10CEF0004B48008800F4007020B1012042491031F5
:10CF0000086003E000204049103108604448008870
:10CF100000F4806020B101203B491431086003E037
:10CF200000203949143108603D48008800F4006051
:10CF300020B1012034491831086003E00020324953
:10CF4000183108603648008800F4805020B1012074
:10CF50002D491C31086003E000202B491C3108607A
:10CF60002F48008800F4005018B1012028490860BB
:10CF700002E00020264908602948008800F480402B
:10CF800020B1012023492039086003E00020214915
:10CF9000203908602248008800F4004020B10120B8
:10CFA0001C491C39086003E000201A491C3908603C
:10CFB0001B48006800F4803020B101201549143965
:10CFC000086003E000201349143908601448006821
:10CFD00000F4003020B101200E491039086003E050
:10CFE00000200C49103908600D48006800F48020CA
:10CFF00020B101200749091F086003E0002005490E
:10D00000091F086010BD0000940123425000002059
:10D01000B4012142A0812242B40122425860002082
:10D0200054000020001801400000214208B50121F1
:10D030000820FDF7D1F80320ADF8000010208DF88E
:10D04000030003208DF8020069469748FCF7E8FDCD
:10D0500003219548FCF791FE01211020FDF7BCF853
:10D060002020ADF8000010208DF8030003208DF87B
:10D07000020069468D48FCF7D3FD20218B48FCF760
:10D080007CFE08BD10B58848006820F00F00864976
:10D0900008600846006840F00300086001208449E9
:10D0A00008608449C1F88401042002F0E3FB0020F9
:10D0B0007F490860042002F0DDFB00207D49C1F8B3
:10D0C000840110BD10B57848006820F00F00764943
:10D0D00008600846006840F00300086000207449BA
:10D0E000091D08607349C1F88001042002F0C2FBE9
:10D0F00001206F49091D08606E49C1F880010420B4
:10D1000002F0B8FB10BD10B500246748006820F09D
:10D110000F00654908600846006840F00800086094
:10D1200001206349086002F0A5FB01206149C1F8B4
:10D13000840102F09FFB07E0601CC4B2FA2C03DDFF
:10D14000FFF7C0FF012010BD594880380068002853
:10D15000F2D15749091D086000BFF4E710B500205F
:10D160005349091D08605048006820F00F004E49DF
:10D1700008600846006840F00300086000204D4940
:10D18000C1F88001022002F075FB01204849091D09
:10D190000860022002F06EFB00204649C1F88401BD
:10D1A00010BD10B500204249091D08603E480068C6
:10D1B00020F00F003C4908600846006840F003007A
:10D1C000086001203B49C1F88001022002F052FBB7
:10D1D00001203749091D0860022002F04BFB0020A6
:10D1E0003449C1F8840110BD70B504462E4800686A
:10D1F00020F00F002C4908600846006840F003004A
:10D20000086000202A49091D0860002517E0E00990
:10D21000274908606006040E022002F02BFB012063
:10D220002449C1F88401022002F024FB0020204997
:10D23000091D0860022002F01DFB681CC5B2082D04
:10D24000E5DB70BD70B5054600241748006820F086
:10D250000F00154908600846006840F008000860A3
:10D26000002617E000201249091D0860022002F084
:10D2700001FB01200F49C1F884016006040E0C482F
:10D280008038006808B1601CC4B2012002F0F2FAD4
:10D29000701CC6B2082EE5DB15B9FFF782FF01E06E
:10D2A000FFF75CFF204670BD000C014000100140FC
:10D2B000808121420080214210B5FFF7B7FE10BDEA
:10D2C00070B504460026FFF7DDFE2546E11704EBA6
:10D2D00011610912A02202EB4101C8B2FFF784FFDD
:10D2E000FFF711FFE11704EB11610912A4EB012113
:10D2F000C8B2FFF779FFFFF706FFFFF7C3FEA120D3
:10D30000FFF772FFFFF7FFFE0020FFF79BFF0646C7
:10D31000FFF7D8FE304670BD70B504460E460020BB
:10D3200049490860012002F0D0FAFFF7ABFE25461C
:10D33000E11704EB11610912A02202EB4101C8B20E
:10D34000FFF752FFFFF7DFFEE11704EB116109124F
:10D35000A4EB0121C8B2FFF747FFFFF7D4FE304628
:10D36000FFF742FFFFF7CFFEFFF7ACFE0120374982
:10D37000C1F89401052002F0A8FA70BD2DE9F04132
:10D3800005460E461746002409E0E20026FA02F29E
:10D39000D1B22A1990B2FFF7BFFF601CC4B2BC42E1
:10D3A000F3DBBDE8F0812DE9F04107460C4600268D
:10D3B000002509E036023919491B491E88B2FFF7DA
:10D3C0007FFF0644681CC5B2A542F3DB3046BDE8CA
:10D3D000F08110B5FF20FFF773FF0446552C01D1F3
:10D3E000002010BD5521FF20FFF796FFFF20FFF71B
:10D3F00067FF0446552C01D10020F2E70120F0E739
:10D4000070B506460C46154608E03046721C96B2CA
:10D41000FFF756FF04F8010B681E85B2002DF4D10A
:10D4200070BD70B505460C46164606E021782846C4
:10D43000FFF772FF681C85B2641C301EA6F1010163
:10D440008EB2F3D170BD000094012242000022424E
:10D4500070B50546002406E0601C84B2B4F5803F38
:10D4600001DB002070BD02217F48FDF768F800282D
:10D47000F2D029467C48FDF70FF806E0601C84B224
:10D48000B4F5803F01DB0020ECE701217648FDF791
:10D4900056F80028F2D07448FDF700F8C0B2E1E772
:10D4A00010B50446704800884FF6C77108406E49B1
:10D4B0000880084600882043088001216A48FCF75C
:10D4C000BAFF10BD00B587B0012141F20900FCF799
:10D4D00083FE01210846FCF774FC3820ADF81800E3
:10D4E00018208DF81B0003208DF81A0006A95F484C
:10D4F000FCF796FBBDF818105C48FCF73EFC01A851
:10D50000FCF783FF0020ADF804004FF48270ADF803
:10D5100006000020ADF80800ADF80A00ADF80C00D8
:10D520004FF40070ADF80E003820ADF81000002068
:10D53000ADF812000720ADF8140001A94A48FCF725
:10D54000D5FE01214848FCF776FF322002F0BDF9F4
:10D550000820FFF7A5FFFF20FFF77AFF07B000BD07
:10D5600010B50446424800884FF6C771084040494C
:10D570000880084600882043088001213C48FCF7C9
:10D580005AFF10BD70B50546002406E0601C84B249
:10D59000B4F5803F01DB002070BD02213448FCF768
:10D5A000CEFF0028F2D029463148FCF775FF06E08F
:10D5B000601C84B2B4F5803F01DB0020ECE7012160
:10D5C0002B48FCF7BCFF0028F2D02948FCF766FF87
:10D5D000C0B2E1E700B587B001210820FCF7FCFDEF
:10D5E00001218803FCF705FE4FF46040ADF81800F8
:10D5F00018208DF81B0003208DF81A0006A91B487F
:10D60000FCF70EFB4FF460411848FCF7B6FB002016
:10D61000ADF804004FF48270ADF806000020ADF8BC
:10D6200008000220ADF80A000120ADF80C0040020D
:10D63000ADF80E001820ADF810000020ADF8120073
:10D640000720ADF8140001A90948FCF74FFE01219D
:10D650000748FCF7F0FEFF20FFF794FF3820FFF7A4
:10D660007FFF07B000BD000000300140000C01400A
:10D6700000380040B548B6494860B6484860704731
:10D68000B348006940F08000B14908617047B04874
:10D69000C16801F0010008B10120704701F00400E9
:10D6A00008B10220F9E701F0100008B10320F4E707
:10D6B0000020F2E770B5044600BFFFF7E8FF05461B
:10D6C000012D00D006E0012002F0D4F8601E84B2E3
:10D6D000002CF2D100BF04B9FF25284670BD70B5FB
:10D6E0000546002445F6FF70FFF7E4FF0446C4B981
:10D6F0009748006940F00200954908610846456175
:10D70000006940F04000086145F6FF70FFF7D2FF66
:10D710000446012C05D08E48006920F002008C4997
:10D720000861204670BD70B505460E46FF20FFF724
:10D73000C1FF044694B98648006940F0010084495D
:10D7400008612E80FF20FFF7B5FF0446012C05D0AD
:10D750007F48006920F001007D490861204670BDC6
:10D76000014608887047014601F0010010B9088899
:10D77000C0B2704731F8010C000AFAE72DE9F04118
:10D7800005460E461746002407E036F814102846D2
:10D79000FFF7C9FFAD1C601C84B2BC42F5DBBDE8DD
:10D7A000F08130B503460C461546002207E01846C6
:10D7B000FFF7D6FF24F812009B1C501C82B2AA422D
:10D7C000F5DB30BD2DE9F05F80468A461746B8F19B
:10D7D000006F02D36048804501D3BDE8F09F72B668
:10D7E000FFF748FFA8F1006B4FEADB25CBF34909AF
:10D7F000C9F58064A74200DC3C464EE04FF0006172
:10D8000001EBC5204A145549FFF7CBFF00260BE07A
:10D8100009EB0600514931F810004FF6FF718842BC
:10D8200000D003E0701C86B2A642F1DB00BFA64226
:10D830001BDA4FF0006101EBC520FFF750FF002617
:10D8400008E03AF8160006EB0901444A22F81100F4
:10D85000701C86B2A642F4DB4FF0006101EBC520DC
:10D860004A143E49FFF78AFF04E0224651464046EB
:10D87000FFF784FFA74200D110E06D1C4FF00009B4
:10D880000AEB440A08EB4408381B87B2B7F5806FEF
:10D8900002DD4FF4806400E03C46AFE700BFFFF7D5
:10D8A000EFFE62B600BF98E730B503460C4615465A
:10D8B000002206E01846FFF756FFA0545B1C501CE0
:10D8C00082B2AA42F6DB30BD13B50446012201A99B
:10D8D0002046FFF777FF1CBD2DE9F05F044689461F
:10D8E000924600252746C846B4F1006F02D31A4875
:10D8F000844201D3BDE8F09F00261DE098F80100A6
:10D900004FEA002B98F8000058441FFA80FB08F1FA
:10D9100002082846691C8DB2114921F810B0B5F5EE
:10D92000806F07D100254FF480623846FFF726FF4D
:10D9300007F50067B01C86B25645DFD325B12A46ED
:10D9400007493846FFF71AFF00BFD3E723016745B1
:10D9500000200240AB89EFCD00000808A00E002097
:10D96000A006002010B501215048FDF70CFD012153
:10D970004E48FDF711FD10BD7FB505460C4601214F
:10D980000220FCF736FCADF80850ADF8044000204A
:10D99000ADF80A00ADF8060001A94448FCF7DAFE2C
:10D9A0001D208DF8000000208DF8010002208DF868
:10D9B000020001208DF803006846FBF788FC012275
:10D9C00011463A48FDF73DFA01213848FDF71EFAA5
:10D9D0007FBD10B501213648FDF7D5FC012804D1E3
:10D9E00034480068401C3349086033480188008887
:10D9F000401C314A1080B1F57A7F07DB00201146C8
:10DA000008802E480068401C2C4908602C4800887B
:10DA100041F28831884205DA29480088401C2849AB
:10DA2000088002E000202649088026480078401C33
:10DA300024490870084600780A2804D1FFF78BF8BB
:10DA400000202049087001211948FDF7A5FC10BDF0
:10DA50007FB505460C4601211020FCF7CAFBADF846
:10DA60000850ADF804400020ADF80A00ADF80600FB
:10DA700001A90F48FCF76EFE36208DF8000001204A
:10DA80008DF8010003208DF8020001208DF80300BD
:10DA90006846FBF71CFC012211460548FDF7D1F949
:10DAA00001210348FDF7B2F97FBD000000040040EA
:10DAB00000100040640000206A000020C401002023
:10DAC000F40300206800002008B501210820FCF7BD
:10DAD00083FBC020ADF8000010208DF80300032068
:10DAE0008DF802006946FC48FCF79AF84FF4807004
:10DAF000ADF8000048208DF8030003208DF80200E7
:10DB00006946F548FCF78CF840F2CF216420FFF716
:10DB10009FFF8021F048FCF732F90A2001F0D5FE82
:10DB20008021ED48FCF729F90A2001F0CEFE802182
:10DB3000E948FCF724F90A2001F0C7FE8021E648F5
:10DB4000FCF71BF90A2001F0C0FE8021E248FCF737
:10DB500016F90A2001F0B9FE8021DF48FCF70DF923
:10DB60000A2001F0B2FE8021DB48FCF708F90A2008
:10DB700001F0ABFE8021D848FCF7FFF80A2001F045
:10DB8000A4FE08BD70B505460C4600264021D248CB
:10DB9000FCF7F5F804F01F0040EA05063046FFF7F1
:10DBA00057FCFF20FFF754FC064604F0800018B134
:10DBB000FF20FFF74DFC06464021C748FCF7DDF883
:10DBC000304670BD2DE9F04104460D46164600274B
:10DBD0004021C148FCF7D3F805F01F0040EA0407D4
:10DBE0003846FFF735FC3046FFF732FC4021BA4893
:10DBF000FCF7C3F8BDE8F08170B505460C4640213E
:10DC0000B548FCF7BCF83A20FFF722FC05E06D1E92
:10DC10000020FFF71DFC2070641C002DF7D10020B0
:10DC200020704021AC48FCF7A8F870BD70B50446E0
:10DC30000D464021A848FCF7A2F87A20FFF708FC1F
:10DC400004E0641E2878FFF703FC6D1C002CF8D15B
:10DC50004021A148FCF791F870BD10B5044604F0CE
:10DC600060009E49097888420ED003221F21A0201F
:10DC7000FFF7A8FFC4F341121F218020FFF7A2FF86
:10DC800004F060009549087010BD10B504462046A8
:10DC9000FFF7E3FF21460020FFF774FF10BD70B5CA
:10DCA00004460D462046FFF7D8FF2A46214640206D
:10DCB000FFF788FF70BD70B505460C460026294663
:10DCC000D420FFF7ECFFE1B2D620FFF7E8FFC4F362
:10DCD0000721D720FFF7E3FF01E0701C86B2EA209E
:10DCE000FFF7D3FF00F0010018B140F6FF70864245
:10DCF000F3DB70BD70B504460025FFF7E5FE09E0D3
:10DD0000FF2200211046FFF75DFF681C85B20A2044
:10DD100001F0DBFD1D20FFF7B8FF00F0010010B996
:10DD2000B5F5FA7FECDBB5F5FA7F01DB012070BDBC
:10DD300000206B49086000210820FFF7B0FF002198
:10DD40000920FFF7ACFF00210C20FFF7A8FF0021FE
:10DD50000D20FFF7A4FF10210A20FFF7A0FF1A21D2
:10DD60000B20FFF79CFF11210420FFF798FF1A21D9
:10DD70000520FFF794FFFF210620FFF790FF1F21EA
:10DD80000720FFF78CFFA1213820FFF788FF3F21F4
:10DD90002820FFF784FF30212920FFF780FFF92199
:10DDA0003020FFF77CFFF7213120FFF778FF0D21AE
:10DDB000C020FFF774FF0021C120FFF770FF33225E
:10DDC000C2218020FFF7FEFE1221C620FFF767FF69
:10DDD0000C21C720FFF763FF1521C420FFF75FFF69
:10DDE000EE21CA20FFF75BFF0521CB20FFF757FF8D
:10DDF0002178E420FFF753FF6178E520FFF74FFF1C
:10DE0000A178E220FFF74BFFE178E320FFF747FF1F
:10DE10002179E020FFF743FF6179E120FFF73FFF21
:10DE20004FF480710020FFF746FF4FF480711020FF
:10DE3000FFF741FF1F20FFF710FFC0221B218020AA
:10DE4000FFF7C0FE04221F218020FFF7BBFEE42065
:10DE5000FFF71BFF2178884201D1002067E70120EE
:10DE600065E710B57220FFF710FF10BD70B50446CE
:10DE70000D4611210220FFF712FF1A210320FFF7A0
:10DE80000EFF11202044C1B20620FFF708FF41F623
:10DE900011202044C0F307210720FFF700FF0022D4
:10DEA00011467A20FFF78EFE29462046FFF7BEFE78
:10DEB00008221F218020FFF785FE1C20FFF7E5FECA
:10DEC00000F0020030B108221F21A020FFF77AFEE7
:10DED00003F076FB70BD0000000C01406C000020D8
:10DEE000700000202DE9F04105460F463920FFF76C
:10DEF000CCFE10B90020BDE8F0812D48017800204B
:10DF0000FFF7CDFE2A480088C0F307210120FFF764
:10DF1000C6FE00213A20FFF735FE254908600021A2
:10DF20003A20FFF72FFE2249096841EA00202049E4
:10DF3000086000213A20FFF725FE044600213A2020
:10DF4000FFF720FE44EA0024241F00213A20FFF7B7
:10DF500019FE064600213A20FFF714FE46EA002685
:10DF6000681EA04204D203F02BFB6C1E0020C2E707
:10DF700006F0800020B903F023FB00240020BAE75C
:10DF800039462046FFF738FE094801780C20FFF794
:10DF900086FE07480088C0F307210D20FFF77FFEAB
:10DFA00040221E218020FFF70DFE2046A3E700003F
:10DFB0007000002008B51F20ADF8000010208DF87B
:10DFC000030002208DF802006946FE48FBF728FE98
:10DFD000FD48C07B00280EDC4FF44070ADF8000017
:10DFE00010208DF8030002208DF802006946F748E2
:10DFF000FBF716FE11E001214020FCF7EDF84FF48D
:10E00000C040ADF8000010208DF8030002208DF80C
:10E0100002006946EE48FBF703FE01214FF404704D
:10E02000FCF7DAF81020ADF8000000208DF80300AE
:10E030006946E648FBF7F4FD08BD00B585B04FF42E
:10E040000040FCF72DF801214802FCF7C5F800203C
:10E0500000908DF804008DF805004FF460200290C8
:10E060000020039001208DF810006946D948FBF785
:10E07000BEF90121D748FBF7E6F9D648FBF705FAC8
:10E0800000BFD448FBF706FA0128FAD0D148FBF7C5
:10E090000BFA00BFCF48FBF70CFA0128FAD005B005
:10E0A00000BD08B501210420FCF796F80120ADF869
:10E0B000000028208DF803006946C248FBF7B0FD38
:10E0C000052001F002FCC448006818B10120C349D2
:10E0D000087002E00020C149087008BD10B5FFF7C4
:10E0E000E0FFFFF767FFFFF7A8FF10BD70B504461C
:10E0F000C4EBC40000EB0410B94901EB400090F8F8
:10E10000235005F00F05C4EBC40000EB041001EB35
:10E11000400090F82800012870D1C4EBC40000EB47
:10E12000041001EB400090F82D00142809DBC4EB2B
:10E13000C40000EB041001EB400090F82D001828FB
:10E1400014DDC4EBC40000EB0410A54901EB400052
:10E1500090F82D000F2809D0C4EBC40000EB041088
:10E1600001EB400090F82D00192874D1C4EBC400D5
:10E1700000EB04109A4901EB400090F82300C0F333
:10E180000310022816D19048C07B002807DC01202C
:10E190009449086000209449C1F8A40106E00120D8
:10E1A0009249086000209249C1F8B80102209149C3
:10E1B000085515E2C4EBC40000EB0410884901EBDC
:10E1C000400090F82300C0F30310032817D17E48C5
:10E1D000C07B002807DC00208249086001208249BA
:10E1E000C1F8A40106E000208049086001208049B0
:10E1F000C1F8B80103207F490855F1E12BE0C4EBD9
:10E20000C40000EB0410764901EB400090F82300B5
:10E21000C0F30310012809D1002072490860724937
:10E22000C1F8A401012073490855D9E16648C07BB3
:10E23000002806DC01206B4908606B49C1F8A40185
:10E2400005E00120694908606949C1F8B80100206A
:10E2500068490855C4E1C4EBC40000EB04106049F0
:10E2600001EB400090F82800012836D1C4EBC4002F
:10E2700000EB041001EB400090F82D000B2809D0B2
:10E28000C4EBC40000EB041001EB400090F82D003B
:10E29000112822D14C48C07B002807DC01205149BD
:10E2A000086000205049C1F8A40106E001204F4950
:10E2B000086000204E49C1F8B80145F0200040B286
:10E2C000C4EBC40101EB0411454A02EB410181F8A2
:10E2D000230002204749085582E1C4EBC40000EB4B
:10E2E00004103F4901EB400090F82800012851D16B
:10E2F000C4EBC40000EB041001EB400090F82D00CB
:10E30000132809D0C4EBC40000EB041001EB40005B
:10E3100090F82D0010283DD12B48C07B002807DC49
:10E3200000203049086001202F49C1F8A40106E00F
:10E3300000202E49086001202D49C1F8B801C4EB26
:10E34000C40000EB0410264901EB400090F82300C4
:10E3500000F00F00C4EBC40101EB0411204A02EBF2
:10E36000410181F82300C4EBC40000EB0410114606
:10E3700001EB400090F9230040F03000C4EBC401F1
:10E3800001EB041102EB410181F82300032019493C
:10E39000085525E1C4EBC40000EB0410104901EB63
:10E3A000400090F8280001287DD1C4EBC40000EBA8
:10E3B000041001EB400090F82D000C2856D0C4EB5F
:10E3C000C40019E00008014058600020001001401E
:10E3D0000018014000240140000121427400002087
:10E3E000E76C0020A001224200002242B401234237
:10E3F00000002342A772002000EB041001EB400054
:10E4000090F82D00282831D0C4EBC40000EB041094
:10E4100001EB400090F82D00292827D0C4EBC40060
:10E4200000EB041001EB400090F82D002A281DD0CD
:10E43000C4EBC40000EB041001EB400090F82D0089
:10E440000C2813D0C4EBC40000EB041001EB400017
:10E4500090F82D000D2809D0C4EBC40000EB041087
:10E4600001EB400090F82D00122840D1FE48C07BFF
:10E47000002806DC0020FD490860FD49C1F8A40120
:10E4800005E00020FB490860FB49C1F8B801C4EB76
:10E49000C40000EB0410F94901EB400090F82300A0
:10E4A00000F00F0000E022E0C4EBC40101EB041116
:10E4B000F24A02EB410181F82300C4EBC40000EBF7
:10E4C0000410114601EB400090F9230040F01000C9
:10E4D000C4EBC40101EB041102EB410181F82300FC
:10E4E0000120E74908550A2001F0EFF978E0C4EB74
:10E4F000C40000EB0410E14901EB400090F82D004E
:10E50000092809D0C4EBC40000EB041001EB400063
:10E5100090F82D000A282AD10520D9490855C4EBC6
:10E52000C40000EB0410D54901EB400090F8230033
:10E5300000F00F00C4EBC40101EB0411CF4A02EB61
:10E54000410181F82300C4EBC40000EB0410114624
:10E5500001EB400090F9230040F05000C4EBC401EF
:10E5600001EB041102EB410181F8230038E0BE48C1
:10E57000C07B002806DC0120BC490860BC49C1F80A
:10E58000A40105E00120BB490860BB49C1F8B801FE
:10E59000C4EBC40000EB0410B84901EB400090F854
:10E5A000230000F00F00C4EBC40101EB0411B34AD7
:10E5B00002EB410181F82300C4EBC40000EB04101E
:10E5C000114601EB400090F92300C4EBC40101EBBC
:10E5D000041102EB410181F823000020A8490855ED
:10E5E00070BD70B504460D46002602212046FBF79B
:10E5F000E4F80523012229462046FAF790FF01217D
:10E600002046FAF760FF00BF02212046FBF7CCF856
:10E610000028F9D02046FAF7E9FF0646304670BDDB
:10E620002DE9F0474FF000084FF0010A95480078B7
:10E63000C0EBC00101EB0010904901EB400090F8E5
:10E640002D0019282ED000251EE00E218E48FFF740
:10E65000C8FF0446A044BAF1010F04D12646A146E2
:10E660004FF0000A0BE0A64201DD304600E02046F4
:10E670000646A14501DA484600E0204681460120D1
:10E6800001F023F9681CC5B20C2DDEDBA8EB0600F7
:10E69000A0EB09000A21B0FBF1F07C49794A12781D
:10E6A00021F8120077480078C0EBC00101EB0010A0
:10E6B000724901EB400090F82D000F280CD07148F2
:10E6C0000078C0EBC00101EB00106C4901EB400089
:10E6D00090F82D00192844D16C486A49097830F81F
:10E6E00011006B49674A127821F8120065480078DA
:10E6F0000B2836DB67486349097830F81100644914
:10E70000604A127831F81210884220DD61485D4974
:10E71000097830F811005E495A4A127831F812101F
:10E72000401AB0F5FA6F12DD4F484030554909786C
:10E7300050F83100401C4C494031524A127841F89F
:10E740003200012154484F4A127820F812105048E4
:10E750004C49097830F811004E494A4A127821F89C
:10E76000120048480078401C464908700846007866
:10E77000202801DB00200870424800780B282ADAA4
:10E7800027E040480078C0EBC00101EB00103B4996
:10E7900001EB400090F82D000F280CD0394800788C
:10E7A000C0EBC00101EB0010344901EB400090F8D0
:10E7B0002D0019280CD1642001F087F83148007829
:10E7C000401C30490870084600780B2801D101E050
:10E7D00000E0D6E700BF3148FBF7CBFA07464FF61B
:10E7E000E07007402748007847EA00012B48FBF714
:10E7F000CDFA24480078FFF779FCBDE8F0871FB513
:10E80000044604EB840000EBC400254908448088DA
:10E81000ADF80C0048208DF80F0003208DF80E0095
:10E8200004EB840101EBC4011D4A1144086803A9EB
:10E83000FBF7F6F904EB840202EBC402184B1A440E
:10E84000918804EB840202EBC4021A441068FBF7BF
:10E8500094FA04EB840202EBC402114B1A44D179FE
:10E8600004EB84021EE0000058600020A001224258
:10E8700000002242B401234200002342E76C002042
:10E88000A7720020B600002000240140E0160020FE
:10E890002C17002076000020A01600200008014060
:10E8A000244F020802EBC4021A449079FBF7CEFA17
:10E8B00004EB840000EBC4007D490844D0F8090053
:10E8C000019000208DF808000C208DF8090001202F
:10E8D0008DF80A0001A8FBF7C3F804EB840000EBF5
:10E8E000C40073490844007A8DF8000000208DF8B8
:10E8F000010001208DF802008DF803006846FAF748
:10E90000E6FC1FBD6B48006800F0010010B101205B
:10E91000684908606848D0F88800401C6649C1F81A
:10E9200088000120654948726549488270476148FE
:10E93000006800F0020010B102205E4908605E48E5
:10E94000006F401C5C49086701205D4988815B4974
:10E95000887170475748006800F0040010B1042027
:10E96000544908605448806F401C5349886701200F
:10E970005349C8815149C87170474E48006800F03A
:10E98000080010B108204B4908604B48806E401CBD
:10E990004949886601204A49488148494871704779
:10E9A0004448006800F0800060B180204149086060
:10E9B0004148006C401C40490864012040490880DF
:10E9C0003E4908703B48006800F0400060B14020BC
:10E9D000384908603848806C401C374988640120F9
:10E9E00037494880354948703248006800F02000B7
:10E9F00060B120202F4908602F48006D401C2E492F
:10EA0000086501202E4988802C4988707047294864
:10EA1000006800F4006068B14FF4006025490860A8
:10EA20002548806D401C2449886501202449C88000
:10EA30002249C8701F48006800F4805078B14FF434
:10EA400080501C4908601C48D0F88000401C1A49BE
:10EA5000C1F8800001201A49088218490872154837
:10EA6000006800F4806068B14FF48060114908606C
:10EA70001148006E401C10490866012010490881A9
:10EA80000E4908710B48006800F4804078B14FF4DB
:10EA90008040084908600848D0F89000401C0649AA
:10EAA000C1F89000012006498882044988727047A5
:10EAB000244F020814040140586000202017002051
:10EAC000A016002010B5002407E004EB8401F94AE9
:10EAD00002EB810000F0FCFC641C0A2CF5D3F64824
:10EAE00000F0F6FCF54800F0F3FCF54800F0F0FC0F
:10EAF000F44800F0EDFCF44800F0EAFCEE48F3497D
:10EB00000860EE48F249086010BD2DE9F041044666
:10EB10000E4615469846069F1022314604F13400F1
:10EB200013F0DBFE0021432001550A2D00D30925F7
:10EB3000E562201D00F0D9FC04F1180000F0D5FCBE
:10EB40002461C5F10A00A0616462BDE8F08170B57E
:10EB500005460E46442000F05FFD044694B11EB900
:10EB6000A80000F059FD00E030462063206B20B97A
:10EB7000204600F0B2FD002404E0A900A522206B8D
:10EB800013F05AFE204670BD2DE9FF4F81B080463C
:10EB900015469946DDE90E7A28461099FFF7D7FF0A
:10EBA0000446002C56D0681E216B01EB800B2BF025
:10EBB000070B00953A462046119B0299FFF7A5FFE7
:10EBC0004A464146584600F0CDFC2060BAF1000F9D
:10EBD00001D0CAF8004000F0F5FCBE480068401CB7
:10EBE000BC490860BC48006840B9BB48046008469E
:10EBF000006801280CD1FFF765FF09E0B7480068FD
:10EC000030B9B5480068C06AB84201D8B24804605B
:10EC1000B349E06A0968884202D9B149E06A0860EC
:10EC2000B0480068401CAF490860AF49E06A096815
:10EC3000884202D9AC49E06A0860E16A01EB8101CF
:10EC40009C4A02EB8100211D00F052FC012600F0DD
:10EC5000C2FC01E04FF0FF36012E09D19F48006849
:10EC600030B19D480068C06AB84201D200F0A4FCEF
:10EC7000304605B0BDE8F08F70B5044600F0A2FC48
:10EC800095480068844200D1002414B99248006875
:10EC900000E020460546281D00F052FCA86A18B185
:10ECA00005F1180000F04CFC291D864800F020FCFE
:10ECB0008E480068401C8D4908608A480068401CE6
:10ECC0008849086000F087FC8448006810B10CB9DE
:10ECD00000F072FC70BD70B585480068002866D1F0
:10ECE00084480068401C834908600846006808BBE7
:10ECF0007649086876490968744A11607449086061
:10ED00007D490968491C7C4A116070490968096895
:10ED100009B9012100E0002121B14FF0FF31774A0C
:10ED2000116006E069490968C968CC68734A61687E
:10ED3000116000BF6F48006870490968884235D388
:10ED400000BF62480068006808B9012000E00020A8
:10ED500020B14FF0FF306949086026E05B48006849
:10ED6000C068C468656863480068A84202D2634806
:10ED700005601AE0201D00F0E3FBA06A18B104F161
:10ED8000180000F0DDFB5849E06A0968884202D9A2
:10ED90005549E06A0860E16A01EB8101454A02EBEE
:10EDA0008100211D00F0A4FBCBE700BF04E0544824
:10EDB0000068401C5249086070BD70B5002500F025
:10EDC00001FC4B480068401E49490860084600683D
:10EDD00000284CD13F480068002848D0002621E098
:10EDE0003748C068C46804F1180000F0A9FB201D72
:10EDF00000F0A6FB3C49E06A0968884202D93A491A
:10EE0000E06A0860E16A01EB81012A4A02EB8100B5
:10EE1000211D00F06DFB3049E06A0968C96A88422B
:10EE200000D301262648006808B9012000E0002030
:10EE30000028D5D03248006860B106E0FFF74BFFEC
:10EE40002F480068401E2E4908602D4800680028A1
:10EE5000F4D10126012E03D02A480068012805D1EB
:10EE6000012500202749086000F0A6FB00BF00F044
:10EE7000B2FB284670BD10B50446174800684460D0
:10EE80001C480068844207D213480168091D1048D5
:10EE9000006800F03BFB0CE00F480168091D0B48BF
:10EEA000006800F033FB15480068844201D2134823
:10EEB000046010BD6C170020341800204818002092
:10EEC0005C1800207018002084180020BC0000206E
:10EED000C0000020C8000020B8000020D80000209A
:10EEE000D0000020EC000020D4000020C40000204E
:10EEF000DC000020CC000020E8000020F000002012
:10EF0000E0000020E4000020F9480068401CF849B7
:10EF1000086070472DE9F04104460F464FF00008A5
:10EF2000FFF7F2FF2068C519F24920680968884296
:10EF300009D92068A8420FD9EE48006885420BD94C
:10EF40004FF0010808E02068A84203D8E9480068AB
:10EF5000854201D94FF001082560B8F1000F07D0B4
:10EF6000E5480068001D00F0EBFA2846FFF783FF34
:10EF7000FFF723FF06460EB900F01EFBBDE8F08147
:10EF800070B5044600267CB1FFF7BEFFD948006883
:10EF90000519D9480068001D00F0D2FA2846FFF78D
:10EFA0006AFFFFF70AFF06460EB900F005FB70BDC9
:10EFB00070B5044600F006FB14B9CF48006800E0C5
:10EFC00020460646F56A00F006FB284670BD2DE98E
:10EFD000F04106460D464FF000080A2D00D30925E2
:10EFE00000F0F0FAC4480068864200D1002616B945
:10EFF000C148006800E030460446E76AAF422DD0C1
:10F00000BD4203D92EB14FF0010802E00EB94FF016
:10F010000108E562C5F10A00A06107EB8701B74A64
:10F0200002EB81016069884213D1201D00F088FA4B
:10F03000B349E06A0968884202D9B149E06A0860C8
:10F04000E16A01EB8101AD4A02EB8100211D00F074
:10F050004FFAB8F1010F01D100F0AEFA00F0BBFA9F
:10F06000BDE8F081A248006818B10120A5490860F8
:10F0700025E004E0A2480068401EA1490860A048BD
:10F08000006800EB80009D4951F820000028F1D075
:10F090009B49096801EB8101984A02EB81004168B4
:10F0A0004968416000F1080142688A4202D1416822
:10F0B000496841604168C9688F4A116000BF704764
:10F0C00070B5044600F07EFA8B480068844200D197
:10F0D000002414B98848006800E020460546281D31
:10F0E00000F02EFAA86A18B105F1180000F028FA0D
:10F0F000291D854800F0FCF900F06DFA8CB98348B1
:10F10000006810B100F058FA0BE07F4800688049B1
:10F110000968884203D100207749086001E0FFF7C1
:10F12000A1FF70BD10B5014600200A46764C536918
:10F13000A34201D1012300E0002383B1754C936AFF
:10F14000A34201D1012300E00023012B07D0936AE1
:10F150000BB9012300E00023012B00D1012010BDD9
:10F1600070B505462C4644B363480068844224D0F9
:10F1700000F028FA2046FFF7D5FF01281BD1201DFB
:10F1800000F0DEF95E49E06A0968884202D95C490C
:10F19000E06A0860E16A01EB8101584A02EB8100F4
:10F1A000211D00F0A5F95449E06A0968C96A88423E
:10F1B00001D300F001FA00F00EFA70BD70B50546FB
:10F1C00000262C462046FFF7ADFF012826D14848EF
:10F1D0000068F0B94849E06A0968C96A884201D301
:10F1E000012000E000200646201D00F0A9F9444956
:10F1F000E06A0968884202D94149E06A0860E16A28
:10F2000001EB81013D4A02EB8100211D00F070F904
:10F2100004E004F118013F4800F06AF9304670BD7F
:10F2200010B50446206B00F058FA204600F055FA5D
:10F2300010BD70B53848006818B3FFF765FE374851
:10F24000006808B9012000E000200546FFF7B5FD81
:10F25000BDB900F0B7F93148C068C468201D00F09E
:10F260006FF92B480068401E294908602A48006849
:10F27000401E2949086000F0AEF92046FFF7D0FF94
:10F2800000BF70BD00BFFFF7D4FF1C480068012815
:10F29000F9D900F091F9F6E71FB500200090019030
:10F2A0000290034680221EA103901F48FFF76CFCCA
:10F2B0000446012C09D1F9F709F801201349086027
:10F2C00000200C49086000F061F91FBD10B5F8F787
:10F2D000FDFF00200D49086000F06DF910BD10B56C
:10F2E00000F070F90348046800F075F9204610BD7D
:10F2F000DC000020CC000020B80000206C170020AB
:10F30000D4000020E400002084180020D800002051
:10F31000C80000205C180020C400002070180020E5
:10F3200049444C450000000085F2000870B50025F6
:10F33000F8F7CCFF5B480468F8F7CFFF204670BDB4
:10F3400059480068704770B506460C465748016832
:10F350001831304600F0DAF854480068001D00F01B
:10F36000EFF8601C30B951480168091D504800F0A1
:10F37000BFF805E04B48006805192846FFF77BFDFC
:10F3800070BD70B50646F068C46804F1180000F05E
:10F39000D7F848480068A0B9201D00F0D1F84649C8
:10F3A000E06A0968884202D94349E06A0860E16A74
:10F3B00001EB8101414A02EB8100211D00F098F828
:10F3C00004E004F118013E4800F092F83749E06A81
:10F3D0000968C96A884201D3012500E00025284652
:10F3E00070BD3849096801602E490968416070475D
:10F3F00070B504460D4600F0E5F82868401C08B9D1
:10F4000000261FE02F4920680968884206D0254958
:10F4100060680968884201D8012613E021496068C4
:10F420000968081A296888420BD228681D4A616851
:10F430001268511A401A28602046FFF7D2FF0026B2
:10F4400000E0012600F0C7F8304670BD01201E49DB
:10F45000086070470146002002E0491C421C90B23F
:10F460000A78A52AF9D0800870472DE9F0410446B2
:10F4700014B90E48006800E0204607463D6B284658
:10F48000FFF7E8FF06463046BDE8F0810F490968FE
:10F4900009B9002005E00749096809B9012000E021
:10F4A00002207047CC000020C8000020B8000020D7
:10F4B00084180020DC000020D40000206C170020FD
:10F4C0005C180020E8000020E4000020D8000020A4
:10F4D00000F1080141604FF0FF31816000F1080147
:10F4E000C160016100210160704700210161704726
:10F4F000426853684B6043688B6053689960516001
:10F500004160086103685B1C0360704710B50246E8
:10F510000B685C1C0CB9106907E002F1080000E000
:10F520004068446824689C42FAD944684C604C683E
:10F53000A160886041600A611468641C146010BD99
:10F54000D0E901329A60D0E901235A6001694A6822
:10F55000824201D182684A60002202610A68521E1A
:10F560000A607047001F4FF080730360001F016046
:10F57000001F0023036014380260203870472348BE
:10F580004FF0E021486107200861704710B520481E
:10F59000006840F47F001E4908600846006840F09B
:10F5A0007F400860FFF7EBFF00201A490860F8F77A
:10F5B00065FE002010BD70474FF0805014491C3983
:10F5C0000860704710B5F8F781FE12480068401CCB
:10F5D0001049086010BD10B50E480068401E0D4966
:10F5E00008600846006808B9F8F777FE10BD10B546
:10F5F0004FF0805006491C3908600024F8F766FE79
:10F60000FFF769FBF8F769FE10BD00003F19010024
:10F6100020ED00E0F40000202DE9F04104464FF019
:10F620000008FFF771FC3D48006898B93C493D4A25
:10F630001160002151604FF440513B4A516000215C
:10F64000116037484FF4405141601146016001207C
:10F650003249086044B1103404F0070020B104F0CE
:10F660000700C0F108000444002C31D0B4F5405F1D
:10F670002ED22C4F3846056801E02F462D68686869
:10F68000A04202D228680028F7D1274885421FD01F
:10F69000386800F11008286838606868001B202866
:10F6A00010D92E196868001B70606C6071681D4865
:10F6B00000E00068026852688A42FAD30268326049
:10F6C000066000BF194968680968081A1749086088
:10F6D000FFF773FB4046BDE8F08170B5064635463E
:10F6E000B6B1103D2C46FFF70FFC61680D4800E0F5
:10F6F0000068026852688A42FAD302682260046095
:10F700000A4960680968084408490860FFF755FB22
:10F7100070BD064800687047704700000C0100206B
:10F7200098180020F80000200001002008010020A7
:10F73000014600BF704770B504460D4601203849A8
:10F74000086000BF40213748FBF7E8FF0028F9D0E8
:10F75000A1B23448FBF774FF00203149086020460D
:10F7600070BD10B586B00446012144F20400FAF7DA
:10F7700033FD2C48FBF728FE4FF40070ADF8140061
:10F7800003208DF8160018208DF8170005A92648CB
:10F79000FAF746FA4FF48060ADF8140004208DF8B3
:10F7A000170005A92048FAF73BFA4FF48070ADF82E
:10F7B000140010208DF8170005A91B48FAF730FA3D
:10F7C0004FF480711848FAF7D8FA25208DF8000018
:10F7D00000208DF801008DF8020001208DF8030053
:10F7E0006846F9F774FD01940020ADF80800ADF803
:10F7F0000A00ADF80C00ADF810000C20ADF80E00BA
:10F8000001A90848FBF723FE012240F225510548D3
:10F81000FBF7B5FE01210348FBF7A5FE06B010BDBE
:10F82000A0012142003801400008014010B54FF00E
:10F83000E022126922F004024FF0E0231A61C3179C
:10F8400000EB5373C3F3C7032F4C2370C31700EBB4
:10F850005373D9104FF47A72514301222B4B1A8003
:10F860004FF0E0225161126942F001024FF0E023B3
:10F870001A6110BD2DE9F047074600264FF0E02041
:10F88000D0F814902048007807FB00F800BFFFF77D
:10F8900099FE4FF0E020856911E04FF0E020846987
:10F8A000AC420CD0AC4202D2281B064403E0A9EBC8
:10F8B0000400284406442546464500D300E0ECE712
:10F8C00000BFFFF788FEBDE8F08770B50446FFF77C
:10F8D000DDFD88B10D480088844206DB0B480088B6
:10F8E00094FBF0F52846FFF74BFB0848008894FB93
:10F8F000F0F100FB114084B24FF47A7104FB01F087
:10F90000FFF7B8FF70BD00001601002018010020AD
:10F9100070B504460D46656001F04CFE206070BD78
:10F92000D0E9001211440160704710B5044601F09F
:10F9300041FE206010BD10B5044601F03BFE216879
:10F94000401A6168884201DB012010BD0020FCE7FD
:10F95000F74908807047C2780A44F64BDA7082781B
:10F9600002EB21229A7042785A7002781A701A4675
:10F970009278B2EB212F0ADA1A465278521C5A704A
:10F980001A4652781AB91A461278521C1A70E94A65
:10F99000D278CBB29A4212DAE64A9278521CE54B00
:10F9A0009A701A46927852B91A465278521C5A7076
:10F9B0001A4652781AB91A461278521C1A707047B1
:10F9C000F0B50B46144619461E19751E0BE04E780D
:10F9D0000F7806EB0726B2B28618B0B2904201DA71
:10F9E000461CB0B2891CA942F1D3A9420AD10E78B3
:10F9F000002707EB0626B2B28618B0B2904201DAB1
:10FA0000461CB0B2F0BD0146080240EA212080B297
:10FA1000704770B504460D462A4621460020FFF780
:10FA2000CFFF0646FFF7EFFF70BD10B51422C249A5
:10FA30000020FFF7C5FF044614B94FF6FF7010BD54
:10FA40002046FFF7E0FFFAE770B50446BA480E38E3
:10FA5000417C007C01EB0020143885B2281986B265
:10FA60000822B5490C313046FFF7AAFF06462A4660
:10FA7000B14914313046FFF7A3FF064616B94FF6D9
:10FA8000FF7070BD3046FFF7BEFFFAE710B50620E5
:10FA9000FFF7DAFF10BD10B51120FFF7D5FF10BD3D
:10FAA0000020A64908700AE00020A549A34A127860
:10FAB00021F81200A1480078401CA04908709F4816
:10FAC00000781E28F0DB00209C49087012E000201E
:10FAD0009A49097801EB81019A4A02EBC101487603
:10FAE00014219948954A1278815494480078401C12
:10FAF00092490870914800781E28E8DB4FF4806036
:10FB00009249088000208D4908700BE00020904940
:10FB10008A4A127801EB8211888088480078401C5C
:10FB200086490870854800780A28EFDB7047002076
:10FB300017E000EB8001834A02EBC101497E71B1FD
:10FB40008149095C491E804A11541146095C31B94A
:10FB5000002100EB80027B4B03EBC2025176411C7B
:10FB6000C8B20528E5DB704730B504460D4600BF36
:10FB700076480088401C7549088008460088B0F522
:10FB8000FA4F02DB4FF48050088000206B49087068
:10FB900015E06A48007800EB80006A4901EBC0027A
:10FBA000507E38B169480088FFF72DFF9188884260
:10FBB00000D1DDE761480078401C604908705F486B
:10FBC00000781E28E5DB002200205C49087018E060
:10FBD0005A48007800EB80005A4901EBC003587E78
:10FBE00008B91A4611E0587E072805D11AB1987E47
:10FBF000917E884200DD1A4650480078401C4F49EB
:10FC000008704E4800781E28E2DB00BF0AB90020C9
:10FC100030BD022050764F48007810734D4841782F
:10FC2000517381789173C178D17340F2CA70508258
:10FC30009082012010820020D0760120907603204F
:10FC40001076002090751020D07540480088FFF78E
:10FC5000DAFE9080D58000BF2088108060885080B8
:10FC600000BF1046D4E730B503460C4600BF374806
:10FC70000088401C3549088008460088B0F5FA4FD6
:10FC800002DB4FF48050088000202C49087011E0FE
:10FC90002E480088FFF7B7FE2D49284D2D7801EB3F
:10FCA00085118988884200D1E1E724480078401C0A
:10FCB00022490870214800780A28E9DB0022002048
:10FCC0001E49087011E022481C49097800EB811098
:10FCD000808828B91E481949097800EB811208E08C
:10FCE00016480078401C15490870144800780A2806
:10FCF000E9DB00BF0AB9002030BD144800780002DB
:10FD00001249098840EA21209080D48013B900204C
:10FD1000106005E000BF188810805888508000BF30
:10FD2000402010721046E7E70021044A117026E0D7
:10FD30004C01002054010020A6480020580100205A
:10FD40004C5500209C5000203C58002052010020BF
:10FD5000885500204E010020FD49FE4A127831F8F6
:10FD60001210814206D10021F94AFA4B1B7822F881
:10FD700013107047F7490978491CF64A1170F54984
:10FD800009781E29E8DB00BFF3E70021F14A117072
:10FD900010E0EF49EF4A127831F8121029B9EC4916
:10FDA000EC4A127821F812007047EA490978491C98
:10FDB000E84A1170E74909781E29EADB00BFF3E73A
:10FDC00010B504462146E44800680830FFF7C3FD3B
:10FDD000E2480078E04909680872E0484178DE4866
:10FDE00000684172DD488178DB4800688172DB4839
:10FDF000C178D9480068C17210BD7CB50546D648A7
:10FE00000468042D00D15DE3D548D6490860D64981
:10FE10000860032D0FD1607E00F00F00032808D189
:10FE2000208A30B90820D149087001F060FD01F046
:10FE300010B801F08FB9022D74D1CD48C078401CA4
:10FE4000C0B2CB49C87078B908468078401CC0B2AF
:10FE5000887048B908464078401CC0B2487018B94C
:10FE600008460078401C08700020C2490880C2493A
:10FE70000880607E072802D0607E052808D1A07E19
:10FE8000401CA076A07E782862D1002060765FE0DA
:10FE9000607E00285CD0208A00284ED0A17E481EBB
:10FEA000A076002954D1E07E082808D0607E022880
:10FEB00002D0607E012810D1E07E05280DD10020FF
:10FEC00060768020A949087001F011FD1421A44832
:10FED000363880F82F1001F0ABB8E07E042801DD41
:10FEE000042000E0E07E03218140A176E07E401CFA
:10FEF000E076A248C08C401C81B2A048C184607EDC
:10FF000000F00F00092823D2DFE800F02205060DDB
:10FF1000142215221600FDE300219148363880F89E
:10FF20002F10F8E315E004209049087001F0DFFC81
:10FF300000F0D1BF00BF00BFEEE3607E00F00F0015
:10FF4000032805D108208949087001F0D0FC6EE72C
:10FF50006FE7052D18D18A480068808898B1002085
:10FF60007D4908607E480C387E4908607E490860FB
:10FF70000020814908807F49088008207B4908705B
:10FF800002F030FC9EE254E77C484088401C7B49EC
:10FF9000488073483638807B45280BD00846008857
:10FFA000401C08800846C088401CC88075A001F02D
:10FFB000C5FC3EE76A483638417C007C01EB0020F6
:10FFC0006C490988884208DC65483638417C007CE9
:10FFD00001EB00206749088003E074A001F0AEFC4B
:10FFE00027E75F483638007D00F03F0018B95C48CD
:10FFF0003638407D60B161480088401C5F49088008
:020000040801F1
:1000000008468089401C888174A001F097FC10E7A5
:100010007848008878490988884205D17548408821
:1000200075494988884235D04D483638C07D1128F9
:100030001CD14B483638C08B70490988884206D19C
:1000400047483638008C6D49498888420DD044486D
:100050003638C08B6A490988884207D1404836380B
:10006000008C67494988884200D111E13C48363804
:10007000C08B60490988884206D139483638008CDF
:100080005C494988884205D03C480088401C3B496F
:100090000880CEE6FFF7C9FC4FF6FF7188420CD00E
:1000A00036480088401C354908800846C089401CF5
:1000B000C88154A001F042FCBBE629483638C07D17
:1000C000062800D151E226483638C07D112800D1DB
:1000D000DEE023483638C07D01280CD02748008850
:1000E000401C264908800846008A401C08824AA015
:1000F00001F024FC9DE62148808A401C81B21F4803
:1001000081821748363890F8220008280ED01B4804
:10011000408A401C194948820846008B401C81B225
:100120001648018343A001F009FC82E600210C4837
:10013000363880F82210808C4FF6F771884205DB44
:1001400007483638808C093081B27FE081E00000BA
:100150004C5500205801002044010020540100208B
:10016000CE4800203401002038010020400100204A
:100170004E0100203C0100203E01002008580020D4
:100180004801002069703A20696E76616C696420CC
:1001900076657273696F6E206F7220686561646541
:1001A00072206C656E6774682E00000069703A20DA
:1001B0007061636B65742073686F7274657220740C
:1001C00068616E207265706F7274656420696E205C
:1001D0004950206865616465722E000069703A209C
:1001E000667261676D656E742064726F70706564AD
:1001F0002E0000001C010020B84F0208B44F020876
:100200002801002069703A20626164206368656398
:100210006B73756D2E0D0A0069703A206E656974F6
:1002200068657220746370206E6F722069636D70F0
:100230002E0D0A0069636D703A206E6F7420696339
:100240006D70206563686F2E0D0A0000FC48818484
:1002500005E0FB48808C083081B2F948818400BFFA
:10026000F748418BC183818B018400BF00BFF548F3
:100270000188F3484183F3484188F148818300BFF6
:10028000F148C08A401C81B2EF48C18200F059BFDA
:10029000EE4800881C38ED490880E9482A30EC49CE
:1002A00008602A38008D88B1FFF7F5FB4FF6FF7123
:1002B00088420BD0E448808D401CE349888508467D
:1002C000408E401C81B2E0484186B2E5E148E249F7
:1002D0000860DBE0E0480068808800287ED0D848CD
:1002E000808CDD4909688988884277D1DA480068BE
:1002F0000088DA490988884206D1D74800684088D2
:10030000D649498888423FD0D34800680088D449FC
:100310000988884206D1D04800684088D049498879
:10032000884231D0C648408BCB4909680988884249
:1003300006D1C348808BC84909684988884223D0C0
:10034000BF48C08BC6490988884205D1BC48008C8B
:10035000C3494988884217D0B948C08BB949098830
:10036000884205D1B648008CB649498888420BD0EE
:10037000B348C08BBB49098888422FD1B048008C54
:10038000B849498888427CD1B3480068C08860B1C8
:10039000AB48808CB04909688988884270D1AE48E2
:1003A00000688088B0F5884F6AD0A548408CAA497B
:1003B0000968C88000BFA248408BADF80400A0487F
:1003C000808BADF8060000BFA748006800909DF83C
:1003D00004009DF80010C1F1FF0100E051E0084366
:1003E0008DF804009DF805009DF80110C1F1FF0192
:1003F00008438DF805009DF806009DF80210C1F134
:10040000FF0108438DF806009DF807009DF80310D2
:10041000C1F1FF0108438DF80700BDF804009149C0
:100420000988884205D1BDF806008E49498888426E
:1004300019D08948006800790002874909688988CD
:1004400040EA212080B240F2D24188420BD100BF65
:1004500083480088804909680880814840887E492F
:10046000096848800BE000BF7548408B7A490968ED
:1004700008807348808B78490968488000BF00BFB6
:100480000EE07548006840307349086072480168A2
:1004900076488142FFF41EAF75A001F04FFAC8E420
:1004A00000207C49086002207B49087064482A309B
:1004B000674908607949086000207949088002F09E
:1004C00091F900BF7648008800B9B2E4744800880A
:1004D0001C305E49088008460088011258480174A3
:1004E0005A480178564841741121C1756C480088FA
:1004F0000830C0F307216A480078083041EA00203C
:1005000081B24F48C1840021018553480068818829
:100510004B48418450480068C1884948818400BFE5
:100520004848018846484183464841884448818379
:1005300000BF00BF4848006801884148C183464861
:10054000006841883E48018400BF36304049086059
:10055000FFF7A1FAC04381B239480185008D18B96F
:100560004FF6FF7136480185F8E33748808B401C11
:1005700081B235488183FFF789FA4FF6FF718842CF
:100580000ED03148408B401C2F4948830846008CD0
:10059000401C81B22C48018442A001F0CFF948E40C
:1005A000454C17E0607EA0B12548808CA188884228
:1005B0000FD12348408CE18888420AD12048408BE3
:1005C0002188884205D11E48808B6188884200D1ED
:1005D00005E2283439488442E4D9194890F82F00BC
:1005E00000F03F00022800D021E01548808C3449FB
:1005F00008800020334908700EE0334831490978FB
:1006000030F811002E490988884200D1E6E02D48D3
:100610000078401C2B4908702A4800781E28ECDB23
:100620000948408D401C81B20748418500BF0448FD
:1006300090F82F0000F0040000B189E446E00000CB
:10064000984800201C010020085800203C01002090
:10065000340100208855002048010020B84F0208CE
:10066000B44F02082801002024010020085800206F
:100670007564703A206E6F206D61746368696E678F
:1006800020636F6E6E656374696F6E20666F756E42
:1006900064000000440100204001002038010020D7
:1006A0003E0100207463703A2062616420636865D3
:1006B000636B73756D2E00009C5000202455002044
:1006C0005A010020580100204C550020FE48808C23
:1006D000401C81B2FC4881841421FC4880F82F1012
:1006E0002820FB4908805021F84880F82E1090F807
:1006F0002900F8490870F54890F82D1080F8291065
:10070000F4480178F14880F82D1090F82800F1495C
:10071000087002E042E146E13FE3EC4890F82C101B
:1007200080F82810EB480178E84880F82C1090F801
:100730002700E8490870E54890F82B1080F827104A
:10074000E4480178E14880F82B1090F82600E14950
:100750000870DE4890F82A1080F82610DD480178ED
:10076000DA4880F82A1090F82D00401CC1B2D74812
:1007700080F82D10B1B990F82C00401CC1B2D348BC
:1007800080F82C1071B990F82B00401CC1B2CF48F2
:1007900080F82B1031B990F82A00401CC1B2CB4828
:1007A00080F82A10C948408CCB490880C748818C02
:1007B0004184C9480188C548818400BF418BC183F9
:1007C000818B018400BF00BFC4480188BF484183BA
:1007D000C2484188BD48818300BFEFE30024002068
:1007E000BC49087030E0BB48007800EB8000BC4991
:1007F00001EBC000407E30B9B648007800EB8000C5
:1008000001EBC00424E0B348007800EB8000B44959
:1008100001EBC000407E072811D14CB1AD480078F3
:1008200000EB800001EBC000807EA17E884206DDE7
:10083000A848007800EB8000A94901EBC004A54856
:100840000078401CA3490870A24800781E28CADB23
:1008500000BF4CB99C48008D401C81B29A4801856C
:10086000A0A001F06BF814E4A74804600320A07670
:1008700020760020A0750420E0750020E0769348E3
:10088000808CA0809148408CE08000BF8F48408BD6
:1008900020808E48808B608000BF012060769B485E
:1008A000007820739948417861738178A173C17889
:1008B000E17301202082854890F82910E17290F8B8
:1008C0002810A17290F82710617290F8260020720B
:1008D0000120FFF775FA7D4890F82E0000F0F00037
:1008E00050285ADD00207B4908704AE0794800789A
:1008F00036307649085C864908700846007800B9A9
:100900004AE083480078012805D172480078401CED
:100910007049087035E07E480078022820D16D4883
:10092000007837306949085C042819D16948007893
:100930003930095C674800783830644A105C41EA15
:100940000020654908800846008840F2CA71884244
:1009500001DD084601E0604800886082A0821BE05B
:100960005C48007837305949085C00B914E05948B0
:10097000007837305549085C56490978084455498C
:100980000870524890F82E000521C1EB2010514903
:100990000978B1EB800FA9DB00BF00BF10214B48E5
:1009A00080F82F1000BF494890F82F0040F0020156
:1009B000464880F82F10022180F83610042180F874
:1009C0003710072180F83810CA2180F839102C2000
:1009D0003F49088060213D4880F82E1031E34A48A5
:1009E000046000204B490870384890F82F0000F050
:1009F000040050B10020607647A000F09FFF202047
:100A00004449087000F073FFA4E3304890F82E00CA
:100A1000001180002F4908702D4800880978401A7D
:100A200014382B490880607E00F00F00022806D1A0
:100A3000264890F82F0000F03F00122822D02448CA
:100A40000088002805DC214890F82F0000F0030002
:100A5000C0B11E4890F82600217A884211D11B4867
:100A600090F82710607A81420BD1184890F828102E
:100A7000A07A814205D1154890F82910E07A814288
:100A800000D0D0E2114890F82F0000F01000C8B15B
:100A9000208AB8B1218A04F10C00FEF75CFF0B48F4
:100AA00090F82A002649097888420BD1074890F827
:100AB0002B002349497888427DD1044890F82C00C6
:100AC0001F493FE077E000000858002098480020C8
:100AD0003C010020580100205A0100201C01002088
:100AE0009C5000207463703A20666F756E64206EAF
:100AF0006F20756E7573656420636F6E6E656374C9
:100B0000696F6E732E000000440100204E0100202A
:100B100059010020400100207463703A20676F740F
:100B20002072657365742C2061626F7274696E67E0
:100B300020636F6E6E656374696F6E2E0000000037
:100B4000540100208978884235D1FA4890F82D0068
:100B5000F949C97888422ED1F74800782073F648C1
:100B6000417861738178A173C178E173E07ED8B96F
:100B7000217EA27E891A48B2A17DA0EBE10148B294
:100B8000A17D0144A175002801DA414248B2E17D0E
:100B9000A0EBA10148B2E17D0144E175E17DA27DB8
:100BA00001EBE201217600BF0120E4490870207EBC
:100BB000A07600202082607E00F00F0009286AD213
:100BC000DFE800F0690525BFF4F3F2F1F000DB483F
:100BD000007800F00100C8B1032060764020D749BA
:100BE000087000202082D6480088002808DD0846CA
:100BF000007840F002000870D1480088FFF7E0F864
:100C00000020D049088000F072FE22E1A2E2CB4829
:100C1000007800F00100E8B3C64890F82F0000F01B
:100C20003F00122836D1C34890F82E0000F0F000A3
:100C300050285DDD0020C44908704DE0C2480078AE
:100C40003630BC49085CC14908700846007800B9D4
:100C50004DE0BE480078012805D1BB480078401C13
:100C6000B949087038E0B9480078022823D1B6485D
:100C700000783730AF49085C04281CD1B2480078AE
:100C80003930095CB04800783830AA4A105C41EA33
:100C9000002001E04BE0C4E1AD490880084600882F
:100CA00040F2CA71884201DD084601E0A848008888
:100CB0006082A0821BE0A448007837309D49085C20
:100CC00000B914E0A048007837309A49085C9E4982
:100CD000097808449C490870964890F82E00052130
:100CE000C1EB201098490978B1EB800FA6DB00BF5B
:100CF000032060768F4890F8260020728D4890F887
:100D00002710617290F82810A17290F82910E172F2
:100D10000120FFF755F84220884908700020208202
:100D2000874908808749088000F0E1FD91E0202094
:100D30008249087000F0DBFD00208649096848768A
:100D400075E47C4890F82F0000F0010078B3607ED5
:100D500000F0100058BB208A08B1FBE1CCE17849D3
:100D60000988491C88B2FFF72BF87448007840F0D6
:100D700010007249087072480088002804DD084697
:100D8000007840F00200087000F0B1FD01202082E0
:100D9000082060760020E07600BF1121654880F8C9
:100DA0002F1045E1B9E031E131E10EE1D8E0FFE794
:100DB000604890F82F0000F02000B8B15D4890F82E
:100DC000351090F8340041EA00206349096808446E
:100DD00061490860574890F8351090F8340041EAAE
:100DE000002057490988081A554908805448008846
:100DF00000280DDD607E00F0100048B94F480078F3
:100E000040F002004D4908704D480088FEF7D8FFB9
:100E1000484890F8311090F8300001EB00204C4920
:100E20000880A08A0988884202DB4948008810B9F6
:100E3000A08A474908804648008860823F48007879
:100E400000F00300F0B300203E49088000F04FFDA1
:100E500000BF3A48007800F0200040B10020394936
:100E6000088060761421334880F82F10E0E0334882
:100E7000007800F0100068B100203249088001209D
:100E80002082042060760020E0761121294880F835
:100E90002F10CDE02B480088002819DD2748007866
:100EA00000F0010008B100202082208A68B9608A21
:100EB00024490988884202DA608A22490880214848
:100EC000008800E028E0208202E0208A1D49088096
:100ED0000020E07600BF214800681F4908601948DB
:100EE000008800280BDD208A002808DD208A2830B1
:100EF0001349088018210F4880F82F109CE00F48F4
:100F0000007800F0020038B128200D490880102137
:100F1000084880F82F108FE01CE10848007800F0A6
:100F2000010030B10020607610200449087000F004
:100F3000DEFC76E0984800205401002040010020AB
:100F40003C0100203E0100205801002059010020F2
:100F50005A01002044010020340100203801002003
:100F600089480088002803DD87480088FEF728FFAD
:100F7000864890F82F0000F00100A8B1844800785E
:100F800000F0010028B1072060760020A0762082C2
:100F900001E0062060760120FEF712FF10207C4958
:100FA000087000F0A4FC3EE07948007800F00100F1
:100FB00028B10520607600202082CBE083E07248D3
:100FC0000088002800DD2EE0C4E06F48008800287B
:100FD00003DD6D480088FEF7F3FE6C4890F82F00A3
:100FE00000F0010060B1072060760020A0760120AB
:100FF000FEF7E6FE10206649087000F078FC12E06B
:1010000061480088002800DD0DE0A3E00BE06048A7
:10101000007800F0010018B1072060760020A0766B
:1010200000BF00BF96E01021584880F82F1000BF85
:1010300028205549088000BF5021544880F82E10C0
:1010400000BF217A514880F82A10617A80F82B106D
:10105000A17A80F82C10E17A80F82D10217B80F89D
:101060002610617B80F82710A17B80F82810E17B97
:1010700080F829100621C175A1884184E188818406
:1010800000BF4448018841484183424841883F4865
:10109000818300BF00BF2188C1836188018400BFB4
:1010A000607E00F0100030B10021384880F8311027
:1010B00080F8301006E00721344880F83010CA214B
:1010C00080F8311000BF4021304881752E480088DB
:1010D00001122E4801742C4801782C4841740021DB
:1010E00080F8351080F834104186FEF7CFFCC043FD
:1010F00081B22648418600BF4520244988730021DB
:101100002248C1734175017523480088401C22495B
:1011100008800846008801121C4881741E48017826
:101120001A48C17400210183FEF77FFCC04381B2DD
:10113000164801831948C08B401C81B21748C183EF
:1011400000BF16488088401C144988800020104940
:1011500008707CBD00200C4908800D49087000BF54
:10116000F7E770B504460D46002D0CDD0C490D80E7
:101170000C480068844206D0084602882146094887
:10118000006811F0E2FA70BD3C0100209848002090
:10119000400100201C0100204C01002008580020C4
:1011A0003E010020380100200020F34908700DE0C6
:1011B000F148007800EB4000F04901EB800000218D
:1011C0000160ED480078401CEB490870EA4800785F
:1011D0000828EDDB7047EA490978491CE84A117094
:1011E0000021E54A117017E0E349097801EB41015C
:1011F000E24A02EB810001884288114339B1817AC9
:10120000DF4A1278511A782901DB00210160DA499E
:101210000978491CD84A1170D74909780829E3DBB5
:10122000704710B502460023D34C23701FE0D24B09
:101230001B7803EB4303D14C04EB830003888BB191
:1012400043887BB113880488A3420BD15388448818
:10125000A34207D10B6843608B880381C84B1B787E
:10126000837210BDC44B1B785B1CC34C2370C24BF4
:101270001B78082BDBDB0023BF4C237010E0BE4B38
:101280001B7803EB4303BD4C04EB8300038813B9C5
:10129000438803B908E0B84B1B785B1CB64C23703D
:1012A000B54B1B78082BEADB00BFB34B1B78082B30
:1012B00034D10023B34C2370B34C2370AE4C237055
:1012C0001DE0AD4B1B7803EB4303AC4C04EB8300F8
:1012D000837AAB4C2478E31AAA4C2478A34209DD24
:1012E000837AA74C2478E31AA64C2370A24B1B7870
:1012F000A54C2370A04B1B785B1C9F4C23709E4B0E
:101300001B78082BDDDBA04B1B789B4C23702346FE
:101310001B7803EB4303994C04EB830013680360D1
:101320000B6843608B880381954B1B78837200BFE9
:1013300097E710B5954800882A2803D200209349E2
:10134000088010BD0020914908809148808AB0F53E
:10135000807F03D0B0F5007F54D141E08C48C08C31
:101360008C49098888423AD18948008D8949498841
:10137000884234D186491631881DFFF752FF4FF459
:101380000070834988820846D1F816200262498B92
:10139000818481490A68C0F81620898841837E4982
:1013A0000A68C0F806208988418101460A6A0260FD
:1013B000898C8180808B7649C8840846C18B0185E1
:1013C0007448008872498883724841887048C18394
:1013D0004FF4C1606E4988812A206C49088011E071
:1013E0006B48C08C6B49098888420AD16848008DD7
:1013F00068494988884204D165491631881DFFF73C
:1014000010FF00BF00BF00BF9BE710B56048C08B56
:101410006249098888420CD15D48008C5F4949883F
:10142000884206D15A485E490A68026089888180EC
:1014300091E05748C08B5B490988084055490988A5
:10144000584A1288114088420BD15148008C5549A6
:10145000498808404F494988524A52881140884279
:1014600008D000BF50480088504908804E48408846
:10147000488008E000BF4648C08B4C49088044487B
:10148000008C488000BF00203B49087016E03A48B5
:10149000007800EB4000394901EB800443480088A4
:1014A0002188884205D1414840886188884200D11E
:1014B00008E031480078401C2F4908702E48007819
:1014C0000828E4DB00BF2C48007808283ED1FF2222
:1014D00006212F4811F0B0F92D48002101628184C6
:1014E0002D490A68C0F80620898841812A490A687E
:1014F000C0F816208988418300BF2C480088244901
:10150000C8842A4841882248018500BF00BF21487D
:1015100000881F4988831F4841881D48C18300BF38
:101520004FF480701A498882C881082008820620FA
:1015300088740420C8744FF4C160888101F13600BA
:101540001B4908602A201149088010BD10486168B5
:101550000160218981800E480F490A68C0F8062081
:101560008988418108200A498881084800880E300E
:101570000649088000BFE8E7600100205A580020B3
:101580006201002063010020610100203C01002075
:10159000984800201C0100202C010020C24F0208A6
:1015A000BC4F020824010020200100205C01002023
:1015B00034010020014800687047000064000020EA
:1015C0007CB50025A948FCF795FB0546002405E0FD
:1015D000A648005DA6490855601CC4B2062CF7DB7E
:1015E00040F276411420FCF766FBFEF759FA9F485B
:1015F000143890F82F0000287ED100BF9B48143883
:10160000C07E9A491439897E40EA01200102974838
:101610001438C07E954A143A927E40EA022041EA8C
:10162000202080B2ADF8000090481438417F007F40
:1016300041EA002001028D481438427F007F42EACF
:10164000002041EA202080B2ADF8020000BF00BFB8
:10165000BDF8000087490880BDF80200488000BF3F
:1016600000BF8248143890F824008049143991F85A
:10167000231040EA012001027C48143890F824002D
:101680007A4A143A92F8232040EA022041EA2020C4
:1016900080B2ADF800007548143890F8261090F824
:1016A000250041EA002001027048143890F82620F5
:1016B00090F8250042EA002041EA202080B2ADF8EF
:1016C000020000BF00BFBDF800006B490880BDF8F4
:1016D0000200488000BF00BF6448143890F8200022
:1016E00062491439C97F40EA012001025F48143879
:1016F00090F820005D4A00E0A0E0143AD27F40EA72
:10170000022041EA202080B2ADF80000574814388A
:1017100090F8221090F8210041EA0020010253487D
:10172000143890F8222090F8210042EA002041EA83
:10173000202080B2ADF8020000BF00BFBDF800005D
:101740004E490880BDF80200488000BF4748143861
:10175000807E8DF8040045481438C07E8DF8050061
:1017600042481438007F8DF8060040481438407F06
:101770008DF807009DF804003C491439C97FC1F178
:10178000FF0108438DF804009DF80500374914391E
:1017900091F82010C1F1FF0108438DF805009DF874
:1017A00006003249143991F82110C1F1FF010843B4
:1017B0008DF806009DF807002C49143991F8221085
:1017C000C1F1FF0108438DF8070000BF9DF8050037
:1017D0009DF8041040EA012000029DF805109DF8D4
:1017E000042041EA022140EA2120254908809DF891
:1017F00007009DF8061040EA012000029DF807103E
:101800009DF8062041EA022140EA21201C49488037
:1018100000BF0120FEF759F81449143991F8281037
:101820000902124A143A128D41EA222188B2FEF7C7
:10183000ACFA00F015FE04F0BCFF05E006210B48F1
:1018400000F0D7FA00F0FCFA28467CBD10B50D492F
:1018500040F2EE50FCF746FB80B210BD10B50949CE
:1018600009480088FCF702FB10BD00006C600020F6
:101870002C0100201C010020200100202401002058
:1018800028010020984800203C0100202DE9F0416B
:1018900007460E46002525E005EB8500284901EBAB
:1018A000C00404223946204610F0E0FE68B9E08802
:1018B000B0420AD1607E10B1607E072803D14FF09C
:1018C000FF30BDE8F08168B2FBE7042239462046CC
:1018D00010F0CCFE20B9A088B04201D168B2F0E788
:1018E000681CC5B21E2DD7DB4FF0FF30E9E710B5FD
:1018F0004FF0FF3400BF134890F828000002114950
:10190000098D40EA212080B20F4909688988884200
:1019100013D100F0C6FC0C48006881880A480068B2
:10192000FFF7B4FF0446002C07DB0848007800F0FE
:10193000020010B114200649085510BD7047000080
:101940009C500020586000204401002040010020ED
:101950003C580020352200F8012B012200F8012B11
:1019600000F8011B70470146362001F8010B0420E6
:1019700001F8010BFE48C0690860081D7047014668
:10198000322001F8010B042001F8010BF848406AED
:101990000860081D7047372100F8011B032100F87B
:1019A000011B012100F8011B032100F8011B062186
:1019B00000F8011B7047FF2100F8011B704710B5AC
:1019C0000446012020706070E948007EA07000206D
:1019D000E070E8480068606000202081802060811D
:1019E000E5480068E060002020616061A061E04897
:1019F0008269416904F11C0010F0A7FEDC4A92697B
:101A0000C2F11001DA4A936904F11C02981810F02F
:101A10001BFF402104F12C0010F016FF802104F17F
:101A20006C0010F011FFD5490968C4F8EC1010BD26
:101A300070B5D34805682846FFF7C1FF012105F1BD
:101A4000F000FFF787FF04462046FFF7A4FF044697
:101A50002046FFF7B0FF0446C9480068211AC8486D
:101A60000068FFF77EFB70BD70B5C5480568284665
:101A7000FFF7A5FF032105F1F000FFF76BFF044618
:101A80002046FFF770FF04462046FFF778FF044624
:101A90002046FFF790FF0446B9480068211AB8486D
:101AA0000068FFF75EFB70BD30B50246531800209A
:101AB00031E01478332C24D006DC012C0BD0032C1D
:101AC0000ED0062C23D110E0352C13D0362C13D099
:101AD000FF2C1CD11AE0A64CD2F80250A56216E0E9
:101AE000A34CD2F80250256311E0A14CD2F8025069
:101AF000E5620CE090780AE09D4CD2F80250E56176
:101B000005E09B4CD2F80250256200E030BD00BFDA
:101B10005478A41C22449A42CBD300BFF6E710B5F8
:101B2000974804682078022817D104229149201D83
:101B300010F09CFD88B98E488269416904F11C004F
:101B400010F094FD48B98A48216941628D480188A6
:101B500004F1F000FFF7A8FF10BD0020FCE7002013
:101B60008349496888808848817EC07E01EB0020D7
:101B70007F4988848448017F407F01EB002081B247
:101B80007B48C1848048C17F90F8200001EB002091
:101B9000774908857C4890F8211090F8220001EBE5
:101BA000002081B272484185774890F8231090F860
:101BB000240001EB00206E498885734890F82510B9
:101BC00090F8260001EB002081B26948C1856E487B
:101BD00090F8231090F8240001EB00206449088657
:101BE000694890F8251090F8260001EB002081B29A
:101BF0005F484186704710B5012400BF5C480088EB
:101C0000B0F5BE7F69D005DC58B1A0F253100028B2
:101C10006FD11AE0B0F5D77F6CD0B0F5DA7FF7D18D
:101C2000DCE00120524988704FF47A70088200BFCE
:101C3000FFF7FEFE4E48018A0830FDF769FE00BF3F
:101C400040F253104A49088000BF5048007800F025
:101C5000020030B946480830FDF76DFE08B9002093
:101C600010BD00BF4948007800F0020030B1FFF716
:101C700056FF022802D13E49887017E03C48008A8E
:101C80004EF66021884207DA3948008A4FF6FF7124
:101C900001EA4000364908823548008AB0F57A5F8B
:101CA00000DB54E0324880780228C1D100BF4FF4F5
:101CB0007A702F49088200203449087000BF00BFA5
:101CC000FFF7D2FE2A48018A0830FDF721FE00BF47
:101CD0004FF4BE702649088000BF2C48007800F001
:101CE000020040B922480830FDF725FE18B900204F
:101CF000B6E778E062E000BF2448007800F0020018
:101D000038B1FFF70CFF052803D10320184988706C
:101D10001BE01748008A42F21071884206DC144822
:101D2000008A00F57A701249088204E000BF0020A2
:101D30000F49088094E70E48008AB0F5FA5F00DB8F
:101D400005E00B4880780328BAD100BF02E0FFF716
:101D500006FF00BF064800F071FD054890F822001C
:101D600002020348408C42EA1022014810E00000C1
:101D7000BC580020C64F02081C010020CA4F0208B0
:101D8000340100203C010020586000204001002068
:101D900090F820000002354B1B8C40EA132002EB28
:101DA0000040322200FB02F130480830FDF7B0FD60
:101DB00000BF4FF4D7702D49088000BF2B48083072
:101DC000FDF7B9FD08B900204AE700BF77E700BF7B
:101DD00000244FF4DA702549088000BF0CB90320B5
:101DE0003EE700BFF3E700BF002020490880022043
:101DF00036E738B504460D461C484461856100202D
:101E00001A49887000BF4FF6FF70ADF80000ADF8BA
:101E1000020000BF4FF486416846FDF724FF1349D6
:101E200048600846406818B14FF488404968888087
:101E300000200E49088038BD10B5FFF7DCFE10BD4C
:101E400008B50A48807878B900BF0020ADF80000D6
:101E5000ADF8020000BF00BFBDF8000004490880D3
:101E6000BDF80200488000BF08BD0000BC5800203B
:101E70001C010020014600BF11F8012B02E0491CA3
:101E8000501EC2B2002AFADC08780028F4D1481C9F
:101E900070472DE9F0410020CB49087071E0CA4835
:101EA0000078C0EBC00000EB4000C84901EB4004E3
:101EB0002078012802D0207802285CD120780228DE
:101EC00011D16078401EC0B2607058B9A078401C33
:101ED000C0B2A070082802D1042020704CE0A07885
:101EE000607006E048E00220207001206070002051
:101EF000A070B7480768002038607860B860B248C2
:101F00000078FDF780FD38800120B8700002B880AD
:101F1000AF48006800F10C05661D761E00BF761CF8
:101F2000A8466D1C0020AB49087008E03078287086
:101F30006D1CA8480078401CA6490870761C3078B3
:101F40002E2802D030780028F0D1A248007888F8F6
:101F5000000030780028E2D19F48016829600079AC
:101F60002871681D9A4A1278801AC1B29848006890
:101F7000FFF7F7F809E000BF93480078401C92494A
:101F8000087091480078042889DB00BFBDE8F08123
:101F90002DE9F0418E4807683888FDF734FD8F49F8
:101FA000087008460078C0EBC00000EB400087498D
:101FB00001EB40068948007804284DDA3078022881
:101FC0004AD103203070F87800F00F00307130797A
:101FD00018B104203070BDE8F081B888FDF713FD1A
:101FE0007F490870084600780870F888FDF70BFDF7
:101FF0007C490870764800680C30FFF73BFF041DF1
:1020000026E0207800F0C00008B1A41C03E02046C0
:10201000FFF730FF044625462888B0F5807F0CD1B5
:102020006888B0F5807F08D12889B0F5806F04D129
:102030006889F084A9893185CDE72889FDF7E3FC1B
:1020400004F10A01441867480078401E6549087089
:10205000644800780028D4DC00BFBCE710B56248B3
:102060000068C088B0F5545F0DD16048007800F07A
:10207000080008B1FFF70DFF5C48007800F002008F
:1020800008B1FFF785FF10BD70B50546002058491F
:102090000870584908705849087022E0564800787E
:1020A000C0EBC00000EB4000484901EB4004207841
:1020B00000B91AE0E07851490978081A4D490978C1
:1020C000884209DDE0784D490978081A49490870C5
:1020D000494800784649087047480078401C4649FE
:1020E0000870454800780428D8DB00BF42480078D3
:1020F00004280CD13E4800783F4908700846007813
:10210000C0EBC00000EB4000304901EB4004294621
:10211000601D10F0D7FA0120207038480078E07078
:1021200036480078401C3549087070BD70B50546CA
:1021300000203349087018E031480078C0EBC00037
:1021400000EB4000214901EB40042078032807D12F
:10215000611D284610F0ECFB10B904F1260070BD9B
:1021600027480078401C2649087025480078042834
:10217000E2DB0020F3E72348006808B9002070473D
:1021800020480068FBE71F49096819B100211D4A72
:1021900012689180704700201B4908700EE00320F0
:1021A00019490978C1EBC10101EB4101074A02F865
:1021B000110015480078401C134908701248007837
:1021C0000428ECDB704770476C010020F0580020B9
:1021D000340100206D0100206E01002075010020F7
:1021E00073010020740100204801002040010020FC
:1021F0007801002077010020760100206401002092
:1022000079010020680100207A01002010B56C4897
:10221000006800F11C04A068002803DDD4E9010176
:10222000FEF79FFF10BD10B56548006800F11C0463
:102230000020A06063A0FFF781FB10BD10B56048CF
:10224000006800F11C046448007840F08000624996
:10225000087062A0FFF772FB00202070A06010BD24
:1022600010B55D48007820F080005B49087061A0DF
:10227000FFF764FB10BD10B55748007820F08000D0
:102280005549087061A0FFF759FB10BD10B55248C1
:10229000007820F080005049087062A0FFF74EFBE4
:1022A00010BD70B500254648006800F11C04634865
:1022B000007800F0200008B1FFF7E8FF5F480078E1
:1022C00000F0800008B1FFF7D6FF5C48007800F00E
:1022D000100008B1FFF7C4FF5848007800F0400034
:1022E00008B1FFF7ABFF5548007800F0010008B1D6
:1022F000FFF799FF5148007800F0020000283BD01A
:102300004F4802884F4801684F4810F01EFA4E4867
:102310000078EE281AD14C484078102816D14A4847
:10232000807898B94848C07880B94748007968B93A
:102330004548407950B94448807938B94248C07915
:1023400020B9012501204149087015E03E488079F7
:102350003F490979884203D03B488079FF280BD157
:1023600002203C49087001253749012001F097FD02
:102370003549012000F0BAFE3048007800F0040032
:1023800098B92E48007800F0020070B92B48007808
:1023900000F0010048B92948007800F0400020B959
:1023A0002648007800F0080040B1012D04D12A48E9
:1023B00060602A480088A060FFF728FF70BD000019
:1023C000440100207463705F7365727665722061EA
:1023D000636B6564210D0A007C0100207463705FEB
:1023E00073657276657220636F6E6E656374656483
:1023F000210D0A007463705F7365727665722063E5
:102400006C6F736564210D0A000000007463705FD7
:102410007365727665722074696D656F7574210DD0
:102420000A0000007463705F7365727665722061E4
:10243000626F72746564210D0A0000004001002083
:102440003C010020340100209859002000000020A9
:10245000586000205C000020C45A00207E0100204B
:1024600010B54DF20420FDF790FC4DF20420FE491A
:10247000888010BD10B504463C21FC4810F0E4F9FA
:102480001CB96520F949087004E0012C02D16720CD
:10249000F64908700020F5494870F5480078087141
:1024A000F34840788871F24880780872F048C07824
:1024B0008872EF48807B0873ED4800798873EC4898
:1024C000807E0874EA48C07E8874E948007F0875F9
:1024D000E748407F8875E64890F828000876E44889
:1024E000008D00124876002088764720C8760020AC
:1024F0000877DF48C07B487700208877C87781F865
:10250000200081F82100DB480088000A81F82200C1
:10251000D848007881F82300D748007881F8240053
:102520001422D649D148253010F00FF9D14800685F
:10253000000ECE4981F83900CE480068000C81F8C1
:102540003A00002081F83B003C21C848FEF709FE14
:102550000120CB49087010BD70B50024C94800782F
:1025600000F00200002842D0C74806783246C7482B
:102570000168C74810F0E9F8C5480078642837D1E9
:102580000120BF49087000BF24E0A000401CC049E2
:10259000085CB749897E88421AD1A000801CBC49DA
:1025A000095CB348C07E814212D1A000C01CB8496A
:1025B000095CAF48007F81420AD1A000001DB449E8
:1025C000095CAB48407F814202D10020AC490870D1
:1025D000601CC4B2F11706EB9171B4EBA10FD4DB10
:1025E000A74800780028BED00020FFF743FFF8E09E
:1025F000A74800786628FAD1A54840789C49897E8A
:102600008842F4D1A24881789948C07E8142EED1B7
:102610009F48C1789648007F8142E8D19C48017963
:102620009348407F8142E2D19948407C90490978A3
:10263000884211D19648807C8D49497888420BD1D7
:102640009348C07C8A498978884205D19048007DAA
:102650008749C97888420FD08D48407C0028C6D170
:102660008B48807C0028C2D18948C07C0028BED11C
:102670008748007D0028BAD105240120FFF7FAFE23
:1026800000207B4988772146641C8148405C78495A
:1026900088762146641C7E48415C7548C176214697
:1026A000641C7B48415C724801772146641C784871
:1026B000415C6F484177807E6D4981F82B00084668
:1026C000C17E80F82C10017F80F82D10417F80F8AA
:1026D0002E102146641C6E48405C6549C877204630
:1026E000611CCCB26A49095C614880F82010204620
:1026F000611CCCB26649095C5D4880F82110204617
:10270000611CCCB26249095C594880F82210C07F34
:10271000574981F83000084690F8201080F83110B1
:1027200090F8211080F8321090F8221080F83310C1
:102730002046611CCCB25649085C4D4981F8230003
:102740002046611CCCB25249095C494880F82410EB
:102750002046611CCCB24E49095C454880F82510E2
:102760002046611CCCB24A49095C414880F82610D9
:1027700090F823003E4981F83400084690F8241070
:1027800080F8351090F8251080F8361090F8261053
:1027900080F8371001203F4908703548807E00B32B
:1027A0003348C07EE8B13248407FD0B1002516E002
:1027B0002F4A1A32515D05F12F00FAF7ADFD2C4A70
:1027C0001F32515D05F13300FAF7A6FD284A233286
:1027D000515D05F13700FAF79FFD681CC5B2042D65
:1027E000E6DB70BD10B5224890F83C00000220499D
:1027F000898F40EA212084B22748006880884DF202
:102800000421884202D1FFF7A7FE06E022480068B3
:102810008088A04201D103F0EFFF1F480068C08804
:10282000B0F5545F05D0B0F5864F05D1FFF704FB36
:1028300002E0FFF713FC00BF00BF10BD38B504462F
:1028400000BFA08C15490880E08C488000BF00BF05
:10285000208D13490880608D488000BF00BF208E06
:1028600010490880608E1FE088550020F05B002032
:1028700058600020040000208E010020C462002067
:1028800080010020400100203C0100203401002094
:102890002C5C002082010020480100201C01002047
:1028A0002401002020010020488000BF04F12C00FA
:1028B000FFF769FCFFF7D4FDB14991F82810090230
:1028C000AF4A128D41EA222188B2FDF75EFA042256
:1028D000AC49AB481A300FF0C9FE002846D0A949D0
:1028E0000888FDF790F8001288B9A6490888FDF716
:1028F0008AF8C0B258B9A3494888FDF784F8001295
:1029000028B9A0494888FDF77EF8C0B270B39D4948
:102910000888FDF778F8001299498876994908885F
:10292000FDF771F8C1B29648C17696494888FDF71F
:102930006AF801129248017792494888FDF763F8D6
:10294000C1B28F484177817E2F20FAF7E5FC8C4891
:10295000C17E3020FAF7E0FC8948017F3120FAF788
:10296000DBFC8748417F3220FAF7D6FC04228649F7
:1029700083481F300FF07AFE00284CD08249088827
:10298000FDF741F8001288B97F490888FDF73BF848
:10299000C0B258B97C494888FDF735F8001228B90B
:1029A00079494888FDF72FF8C0B2A0B37649088866
:1029B000FDF729F800127249C87773490888FDF7B6
:1029C00022F8C1B26E4880F820106F494888FDF7A0
:1029D0001AF801126A4880F821106B494888FDF7FF
:1029E00012F8C1B2664880F82210C17F3320FAF78E
:1029F00093FC634890F820103420FAF78DFC60486F
:102A000090F821103520FAF787FC5D4890F82210E5
:102A10003620FAF781FC04225C49594823300FF034
:102A200025FE00284ED059490888FCF7ECFF00121B
:102A300088B956490888FCF7E6FFC0B258B953492F
:102A40004888FCF7E0FF001228B950494888FCF795
:102A5000DAFFC0B2B0B34D490888FCF7D4FF0012CA
:102A6000474981F8230049490888FCF7CCFFC1B2E7
:102A7000434880F8241045494888FCF7C4FF0112F8
:102A80003F4880F8251041494888FCF7BCFFC1B297
:102A90003B4880F8261090F823103720FAF73CFCCA
:102AA000374890F824103820FAF736FC344890F86C
:102AB00025103920FAF730FC314890F826103A20DA
:102AC000FAF72AFC2E48807E8DF800002C48C07E44
:102AD0008DF801002A48007F8DF802002848407FC9
:102AE0008DF803009DF800002549C97FC1F1FF0161
:102AF00008438DF800009DF80100214991F820104D
:102B0000C1F1FF0108438DF801009DF802001C4946
:102B100091F82110C1F1FF0108438DF802009DF8E2
:102B20000300174991F82210C1F1FF0108438DF805
:102B3000030000BF9DF801009DF8001040EA01204D
:102B400000029DF801109DF8002041EA022140EAB0
:102B500021200F4908809DF803009DF8021040EAEB
:102B6000012000029DF803109DF8022041EA022195
:102B700040EA21200649488000BF03F01AFE38BD14
:102B8000586000201C0100202401002020010020AA
:102B9000280100200020FA490860FA490870FA4923
:102BA0000870704770B540F22551F848F8F7CCFD31
:102BB000012878D10220F6490870F648807C032865
:102BC00073D1F0480078FA280BDAF048F8F73CFDAA
:102BD000C1B2EC480578681CEA4A1070EE484155CD
:102BE00001E0FFF7D7FFE7480078012807D1FA2076
:102BF000EA490870EA480078EA490870A4E0E14828
:102C00000078032807D1E44840781928F6D1062037
:102C1000E249087098E0DB480078042813D1DE48C8
:102C2000C078DD49897800EB01200A28E6D1DA482E
:102C300040780628E2D10C20D8490870D84800789E
:102C4000D849087080E0CF48007807281ED1D248C4
:102C50004078032803D0D0484078062803D10820C4
:102C6000CE49087070E0CC48407810280AD1CA4894
:102C700080790930C9490870C74880790830C94946
:102C8000087061E0FA20C54908705DE0BD48007831
:102C9000C2490978884257D10020C24908700520EE
:102CA000B949087050E013E0FFE7BA48807CE8BB00
:102CB00040F22551B548F8F747FD012844D1B34803
:102CC000F8F7C2FCC4B22146B74809F074FB3BE0F8
:102CD00040F22771AD48F8F737FD012834D10220C2
:102CE000B2490870AB48807C032802D0A948807C98
:102CF000E0B9AF4802880088401CAD4B1880AD4851
:102D0000815CA248F8F79CFC09F005FCA848008803
:102D1000A9490988884217DB00BF40219B48F8F782
:102D2000FDFC0028F9D04021984800E00CE0F8F7BD
:102D300002FD002240F227719448F8F720FC0020A1
:102D40009B490880FFF726FF70BD01208C49086071
:102D5000704770B504460D4640218C48F8F7EBFCEF
:102D600021468A48F8F76CFC15B1204602F0D2FAE9
:102D700070BD70B5044690480480012240F227716E
:102D80008248F8F7FCFB8D48808D642832D1814859
:102D90008068B0F5165F05D104F10A0188B2FCF72E
:102DA00094FD25E07B488068B0F5964F08D1254614
:102DB00004EBD57149100A3188B2FCF786FD17E0A3
:102DC00074488068B0F5164F09D12546E11704EB29
:102DD000917189100A3188B2FCF777FD08E0254629
:102DE000E11704EB5171C9100A3188B2FCF76DFD8F
:102DF0007248048670BD00B5FFF7CCFE0320684919
:102E00000870084600786749087000BD012080F30B
:102E1000138800BF00BF6A48006800F4E060694999
:102E20000843001D66490860BFF34F8F00BF00BF15
:102E3000FEE72DE9F04106460C4615461F46B6F55D
:102E4000FA6F0CD1601D285C5F49087001205F4952
:102E5000487104F0C1FA04F016FEFFF7D7FF40F204
:102E6000D370864210D1601D285C012814D104F073
:102E70000AFE7C2154480FF0E7FC012053494871B9
:102E800004F0AAFAFFF7C2FF40F2D170864204D1E3
:102E9000601D285C4C49487026E140F2D57086429E
:102EA00008D1601D295C201D285C01EB00204649EB
:102EB000888019E140F2D470864208D1601D295CF7
:102EC000201D285C01EB00203F4948800CE140F2C6
:102ED000D770864209D1601D285C012802D104F018
:102EE000E8FD01E104F0FAFDFEE0B6F5FB6F08D164
:102EF000601D285C0028CFD100212120FAF70CFAB0
:102F0000F2E040F2DA7086421ADB40F2F970864253
:102F100016DCA6F2DA70C11700EBD1614911A0EB03
:102F200041110029B8D1402127480A300FF08CFC0C
:102F3000E01D2918402224480A300FF006FCD3E097
:102F400040F2FA70864243DB40F6090086423FDCDD
:102F5000A6F2FA70C11700EB11710911A0EB011173
:102F600000290BD1202118484A300FF06DFCE01DDC
:102F70002918202214484A300FF0E7FBB4E0000083
:102F8000A0012142860100208A0100200038014072
:102F90005A00002058600020585D00208701002062
:102FA000890100208801002034BA00205900002047
:102FB00092010020585E00208C01002068650020EE
:102FC0000CED00E00000FA058B8A0020E2010020F1
:102FD00040F60A00864251D1A6F60A000C2190FB69
:102FE000F1F201FB120000287ED104F10800285CF8
:102FF000FE4981F86A0004F10A00295CFB4880F868
:103000006B1004F10C00295CF84880F86C1004F196
:103010000E00295CF54880F86D1004F11000285C62
:10302000F24981F86E0004F11200295CEF4880F843
:103030006F1004F11400295CEC4880F8701004F162
:103040001600295CE94880F8711004F11800285C2A
:10305000E64981F8720004F11A00295CE34880F81F
:10306000731004F11C00295CE04880F8741004F12E
:103070001E00295CDD4880F8751035E040F616002A
:10308000864231D1A6F61600062190FBF1F201FB33
:10309000120048BB04F10800285CD44981F876008E
:1030A00004F10A00295CD14880F8771004F10C0083
:1030B000295CCE4880F8781004F10E00295CCB48DA
:1030C00080F8791004F11000295CC84880F87A1063
:1030D00004F11200295CC54880F87B10763005F0B9
:1030E00019FE0120C2490870BDE8F0812DE9F047C2
:1030F00082460D46BAF1000F02D0BAF1040F01D199
:10310000002400E00624E01C295CA01C285C01EBE4
:10311000002086B2601C285C10287CD1282E3CD16F
:10312000B44890F82A00012836D1A01D285C0C284C
:10313000FAD104F10800285CAE49087504F10A00D0
:10314000295CAC48417504F10C00295CA9488175E3
:1031500004F10E00295CA748C17504F11000295C38
:10316000A448017604F11200295CA24841760027A8
:1031700009E0A04A1432D15D07F1280290B2FAF7B3
:10318000CBF8781C87B2062FF3DB01209A49087030
:103190000020984981F82A0013E240F2CB208642B1
:1031A0001DDB40F2D520864219DCA01D285C1428C6
:1031B000F2DC00270EE0E21D3A44A95C07F2BA22D5
:1031C00090B2FAF7A9F8E01D3844285C8B49C8553D
:1031D000781C87B2A01D285CB842ECDCDCE742F624
:1031E000D04086424FDB42F6AF7086424BDCA6F5FC
:1031F0003050D0381721B0FBF1F201FB120098B922
:10320000A6F53050D038B0FBF1F087B2E21DA91816
:10321000C7EBC70200E092E002EB0712784B03EB2A
:1032200042002E220FF091FA03F0F5F901207549C2
:103230004870C7EBC70000EB0710714901EB400075
:1032400090F82D000F2809D0C7EBC70000EB07103E
:1032500001EB400090F82D0019289DD1C7EBC70065
:1032600000EB0710664901EB4000D0F81E0020B9C2
:1032700000216048403040F837100B2F8CDAF8B24C
:10328000FBF7BDFA88E743F29020864222DB43F247
:10329000974086421EDC01205A498870A6F54850A6
:1032A00090380A21B0FBF1F201FB1200002895D101
:1032B000A6F548509038B0FBF1F087B2E21DA9188E
:1032C00007EB470202EB07124F4BD01813220FF007
:1032D0003CFA61E748F2A800864222DB48F2B010CF
:1032E00086421EDC01204749C870A6F50040A83878
:1032F0003521B0FBF1F201FB12000028C2D1A6F586
:103300000040A838B0FBF1F087B2E21DA918C7EB66
:103310000712C2EBC2023D4BD01869220FF015FA1A
:103320003AE7B6F5FA6FADDB40F634008642A9DC29
:1033300000232A4621463046FFF77BFD2CE7601C20
:10334000285C06289ED1632E4FDC012E26DC601DF2
:10335000295C0020F9F7E0FF201D295C0120F9F726
:10336000DBFF601D285C23490870201D285C487025
:103370000846007C40F0010008740846017C1120DA
:10338000F9F7CAFF1B48007C0028A2D00020194989
:10339000487300211020F9F7BFFFFDE6032E3ADC49
:1033A000601D295C0220F9F7B7FF201D295C03206E
:1033B000F9F7B2FF601D285C0E498870201D285C5B
:1033C000C8700846007C40F0020008740846017C82
:1033D0001120F9F7A1FF0748007C0028A0D00020A9
:1033E000044948730021102012E093E28B8A0020E8
:1033F000E90100205860002082010020C462002002
:10340000E76C0020E2010020C77A0020DA6A002081
:10341000F9F782FFC0E6062E1AD1601D285C00284D
:103420008CD0601D285CFF2888D0601D295C062098
:10343000F9F772FF601D285CFE49087108460079A3
:10344000FD490870F4F774FF002008F089F9A3E63D
:10345000072E13D1601D295C0720F9F75DFF601D61
:10346000285CF44988730846007C40F00800087422
:103470000846017C1120F9F74FFF8DE6082E13D185
:10348000601D295C0820F9F747FF601D285CE949A9
:10349000C8730846007C40F0040008740846017CAC
:1034A0001120F9F739FF77E60F2E70D1601D285CE7
:1034B000E04908730846007B06287ED2DFE800F06A
:1034C00003172B3F53694FF41650DA498860FCF715
:1034D00048F9601D295C1520F9F71EFF601D295C65
:1034E0001320F9F719FF0620D449087066E04FF45D
:1034F0009640D0498860FCF734F9601D295C15209E
:10350000F9F70AFF601D295C1320F9F705FF032076
:10351000CA49087052E04FF41640C6498860FCF76B
:1035200020F9601D295C1520F9F7F6FE601D295C65
:103530001320F9F7F1FE0220C04908703EE04FF475
:103540006140BC498860FCF70CF9601D295C1520BE
:10355000F9F7E2FE601D295C1320F9F7DDFE01207A
:10356000B64908702AE04FF4E130B2498860FCF7B0
:10357000F8F8601D295C1520F9F7CEFE601D295C66
:103580001320F9F7C9FE0120AC49087016E019E0D4
:1035900013E04FF49630A7498860FCF7E2F8601D0D
:1035A000295C1520F9F7B8FE601D295C1320F9F796
:1035B000B3FE0120A149087000BF00BF00BFFFF7A4
:1035C0001AFC81E3102E04D1601D285C99494873D0
:1035D0007AE3152E19D1601D285C032803D0601DE5
:1035E000285C0028EDD1601D285C92498874601D1C
:1035F000295C1420F9F790FE8E48807C0028E0D1E9
:1036000008F062FFFFF7C6FA5EE3252E0DD1601DBC
:10361000285C0128D5DD601D285C89490870601D83
:10362000295C1220F9F778FE4EE3272E15D1601D94
:10363000295C0620F9F770FE601D285C7E49087041
:10364000084600787B490871F4F772FE002008F004
:1036500087F8002008F038FF36E3162E2AD1601DC7
:10366000295C201D285C01EB002076490968B0EB3D
:10367000114F16D0601D285C0104201D285C01EB51
:1036800000607049098889B208446E490860601D6D
:10369000295C1820F9F740FE201D295C1920F9F754
:1036A0003BFEF4F745FE002008F05AF8002008F031
:1036B0000BFF09E3172E2DD16248D0F80090601D52
:1036C000295C201D285C01EB00205E490968B0EBF5
:1036D000114F16D06FF30F09601D295C201D285C67
:1036E00001EB002040EA09095648C0F80090601D2F
:1036F000295C1620F9F710FE201D295C1720F9F728
:103700000BFEF4F715FE002008F02AF8002008F060
:10371000DBFED9E2262E1AD1601D295C201D285C13
:1037200041EA002043498887201D295C1B20F9F7C6
:10373000F3FD601D295C1C20F9F7EEFDF4F7F8FDA0
:10374000002008F00DF8002008F0BEFEBCE2282E94
:1037500012DB2D2E10DCA6F1280000F0FF08601D02
:10376000295C3448143000F80810621DA95C08F187
:103770002800F9F7D1FDA7E23D2E05D1601D285C98
:103780002C4981F82F009FE23E2E0CDB412E0ADCF3
:10379000A6F13E0000F0FF08601D295C25482B3093
:1037A00000F8081090E2422E0CDB452E0ADCA6F150
:1037B000420000F0FF08601D295C1E48303000F810
:1037C000081081E2462E0CDB492E0ADCA6F14600E9
:1037D00000F0FF08601D295C1648343000F808101E
:1037E00072E24A2E05D1601D285C124981F838002A
:1037F0006AE24B2E08D1601D295C201D285C01EB7C
:1038000000200C4948875FE24C2E6AD1601D285C7D
:10381000084981F83E00084690F83E00012895D1FD
:10382000084690F82F008877084690F8380081F80D
:10383000270009E0586000208E0100208901002047
:103840008F010020040000200846408F08850846AC
:10385000817F2E20F9F760FDFA4890F827103B2071
:10386000F9F75AFDF748008D01123C20F9F754FD95
:10387000F44890F828103D20F9F74EFD002726E087
:10388000F0482B30C15D1138C1551630C15D11387B
:10389000C1551530C15D1138C155A0F10902D15D86
:1038A00007F12F0290B2F9F737FDE64A1F32D15DDA
:1038B00007F1330290B2F9F72FFDE24A2332D15DCE
:1038C00007F1370290B2F9F727FD781C87B2042F71
:1038D000D6DB0120DC4908700020DA4981F83E007F
:1038E000F2E15D2E05D1601D285CD64981F82A00E1
:1038F000EAE15A2E87D1601D295C201D285C4FF417
:10390000807202FB0010D14908800846008802F04E
:103910000EFED9E1642E4EDBA32E4CDCA6F1640032
:1039200000F0FF0808EBD8714FEA6109C9EBC90044
:1039300000EB0910C64901EB400090F82D000F285C
:1039400009D0C9EBC90000EB091001EB400090F869
:103950002D0019282ED10021BA48403040F83910E6
:10396000024612F839104FEA890202F1BE00F9F757
:10397000D3FCB44A403202EBC90251784FEA8902C3
:1039800002F1BF00F9F7C8FCAE4A403202EBC902AF
:1039900091784FEA890202F1C000F9F7BDFCA94A0B
:1039A000403202EBC902D1784FEA890202F1C1002C
:1039B000F9F7B2FC88E1B6F5827F15DBB6F5927FA8
:1039C00012DA301F00F0FF08601D285C40B2C8EB1F
:1039D000C80101EB08119E4A02EB410181F8280061
:1039E00001209C4948706FE1B6F5927F34DBB6F553
:1039F000A27F31DAA6F5927000F0FF08C8EBC8008C
:103A000000EB0810924901EB400090F8230000F011
:103A10000F00C8EBC80101EB08118D4A02EB410110
:103A200081F82300C8EBC80000EB0810114601EB39
:103A3000400090F82310601D285C41EA001040B25D
:103A4000C8EBC80101EB081102EB410181F823002A
:103A500001208049487037E1A42E14DBC32E12DC0C
:103A6000A6F1A40000F0FF08601D285CC8EBC801A7
:103A700001EB0811764A02EB410181F82200012096
:103A80007449487020E1C42E76DBE32E74DCA6F185
:103A9000C40000F0FF08601D285C1F2814DA601DB8
:103AA000285CC8EBC80101EB0811694A02EB41012F
:103AB00081F82D000020C8EBC80101EB081102EBD2
:103AC000410181F8280014E0601D285C1E38C8EB15
:103AD000C80101EB08115E4A02EB410181F82D009B
:103AE0000120C8EBC80101EB081102EB410181F88C
:103AF00028000020C8EBC80101EB0811544A02EB72
:103B0000410181F82B00C8EBC80101EB081102EB61
:103B1000410181F82C0001204E494870C8EBC800D3
:103B200000EB0810114601EB400090F82D000F2823
:103B300009D0C8EBC80000EB081001EB400090F87A
:103B40002D00192814D1C8EBC80000EB081040491B
:103B500001EB4000D0F81E0020B900213948403068
:103B600040F83810B8F10B0F02DA4046FAF747FE7A
:103B700002F051FDA8E0FFE7E42E16DBB6F5827FE8
:103B800013DAA6F1E40000F0FF08601D285C40B2E3
:103B9000C8EBC80101EB08112D4A02EB410181F885
:103BA000270001202B4948708EE0B6F5A27F16DB76
:103BB000B6F5B27F13DAA6F5A27000F0FF08601D1B
:103BC000285C40B2C8EBC80101EB0811204A02EBA7
:103BD000410181F8290001201E49487074E0B6F5C2
:103BE000B27F39DBB6F5D27F36DAA6F5B27000F0D7
:103BF000FF08404608EBD0714910A8EB410171B9AC
:103C0000611D695C08EBD8725210C2EBC20303EB72
:103C100002120F4B03EB420282F82B100DE0611DE4
:103C2000695C08EBD8725210C2EBC20303EB0212BC
:103C3000074B03EB420282F82C1001200549487023
:103C400042E000005860002082010020C0010020F6
:103C5000E76C0020E2010020B6F5487F21D1201D4D
:103C6000285CC8B9601D285CF749C8740846C07C48
:103C7000012809D1002705E0FF213846F9F74CFB60
:103C8000781C87B2FF2FF7DDF4F724FD0021102008
:103C9000F9F742FBFFF7BAF8611D685C03F078FCA6
:103CA00012E0B6F5487F0FDD40F2513086420BDC62
:103CB000601D295C201D285C01EB002081B2A6F567
:103CC0004870E24A22F81010DF48407B7F2801D17B
:103CD000FFF79CF8DC48407B8E282DD100271AE0A6
:103CE000102F16D0AFB1012F13D0062F11D0152FE2
:103CF0000FD0022F0DD0032F0BD03D2F01DC282F2A
:103D000007DA082F05D0072F03D0FF213846F9F72F
:103D100003FB781C87B2FF2FE2DBF4F7DBFC00210A
:103D20001020F9F7F9FA0020C74908740021112082
:103D3000F9F7F2FAFFF76AF8BDE8F0872DE9F041EC
:103D40000446B4F5FA6F03D1C1480078BDE8F081AC
:103D500040F2D170844202D1BD484078F6E740F28B
:103D6000D270844202D1BA488079EFE740F2D47031
:103D7000844202D1B6484088E8E740F2D5708442D8
:103D800002D1B3488088E1E740F2D670844202D184
:103D9000AF48C079DAE7B4F5FB6F03D12120F9F71A
:103DA0008FFAD3E740F2DA70844211DB40F2F97007
:103DB00084420DDCA64F0A37A4F2DA70C11700EB7B
:103DC000D1614911A0EB4111CDB237F81500BDE723
:103DD00040F2FA70844211DB40F6090084420DDCA7
:103DE0009B4F4A37A4F2FA70C11700EB1171091109
:103DF000A0EB0111CDB237F81500A7E740F60A0095
:103E000084420FDBC01C84420CDC914E6A36A4F65F
:103E10000A00C11700EB91718910A0EB8101CDB2AE
:103E2000705D93E740F60E0084420FDBC01C8442B5
:103E30000CDC874E6E36A4F60E00C11700EB9171B4
:103E40008910A0EB8101CDB2705D7FE740F61200D2
:103E500084420FDBC01C84420CDC7D4E7236A4F61B
:103E60001200C11700EB91718910A0EB8101CDB256
:103E7000705D6BE740F6160084420EDB401D844205
:103E80000BDC734E7636A4F61600062190FBF1F299
:103E900001FB1200C5B2705D58E7002056E72DE91E
:103EA000F34FD1B08B46002700260024A14651983D
:103EB00010B15198042802D14FF000090FE04FF0E3
:103EC00006094FF0000A07E0002006A901F80A00E1
:103ED0000AF1010000F0FF0ABAF1060FF4DB09F164
:103EE00001001BF80000049009F103001BF800100A
:103EF000401E1BF8000001EB002080B2039009F186
:103F000005001BF8000005900498062853D14C4684
:103F1000519810B1519804281BD14FF0000A0AE0C3
:103F20001BF80A202046611C8CB206A90A540AF12B
:103F3000010000F0FF0A474800788245F0DB224686
:103F400006A945480EF046FC2046FEF712FF01F098
:103F50008AB89BF800008DF818009BF801008DF8D6
:103F6000190000208DF81A008DF81B008DF81C0038
:103F700006208DF81D0051980128E8D14FF0000A65
:103F80000BE009EB0A001BF8000009EB0A0106AA86
:103F900050540AF1010000F0FF0ABAF1060FF0DBFD
:103FA00009F1060206A92D480EF0CFFB09F1060023
:103FB0002B490880CBE70498102872D1519850BB48
:103FC0004FF0000A10E009EB0A001BF8000009EBB3
:103FD0000A0106AA505409EB0A01505C01F09AF953
:103FE0000AF1010000F0FF0ABAF1060FEBDB1D48F1
:103FF000007809EB0A0106AA50541B48017809EB26
:104000000A00401C11541448DDE9061206C00820BD
:10401000FEF7AFFE9BE75198042898D09BF800006C
:104020008DF818009BF801008DF8190000208DF81C
:104030001A008DF81B008DF81C0006208DF81D005D
:104040004FF0000A1EE00000586000206865002064
:104050008B8A002087010020585E0020C45A00206F
:104060007E010020960100209501002009EB0A0046
:104070001BF8000009EB0A0106AA50540AF10100DE
:1040800000F0FF0ABAF1060FF0DB09F1060206A9FB
:10409000FA480EF05AFB09F10600F949088056E784
:1040A000FFE70498032840F081871BF8090006A960
:1040B00001F8090009F101001BF8001006AA1154CB
:1040C00005984006010E09F10200115406A911F8E5
:1040D000090001F01FF906AA09F10101505C01F085
:1040E00019F906AA09F10201505C01F013F909F16E
:1040F00003044FF0000A00F007BF0398504485B254
:10410000032D14DC0027DF48465D2046611C8CB27D
:1041100006A90F542046611C8CB206A90E543846DD
:1041200001F0F8F8304601F0F5F800F0E9BE042D92
:1041300012D1002747262046611C8CB206A90F54D5
:104140002046611C8CB206A90E54384601F0E2F8F4
:10415000304601F0DFF8E8E7052D12D100270026F0
:104160002046611C8CB206A90F542046611C8CB2FB
:1041700006A90E54384601F0CDF8304601F0CAF8D1
:10418000D3E7062D13D10027BE4806792046611CCF
:104190008CB206A90F542046611C8CB206A90E549D
:1041A000384601F0B7F8304601F0B4F8BDE7072D06
:1041B00013D10027B348867B2046611C8CB206A928
:1041C0000F542046611C8CB206A90E54384601F0EB
:1041D000A1F8304601F09EF8A7E7082D13D100277B
:1041E000A848C67B2046611C8CB206A90F54204605
:1041F000611C8CB206A90E54384601F08BF830468B
:1042000001F088F891E70F2D13D100279D48067B18
:104210002046611C8CB206A90F542046611C8CB24A
:1042200006A90E54384601F075F8304601F072F8D0
:104230007BE70B2D15D100270F20F9F741F8064633
:104240002046611C8CB206A90F542046611C8CB21A
:1042500006A90E54384601F05DF8304601F05AF8D0
:1042600063E7102D13D100278648467B2046611C4A
:104270008CB206A90F542046611C8CB206A90E54BC
:10428000384601F047F8304601F044F84DE7632D19
:1042900013D100277B48067C2046611C8CB206A9FE
:1042A0000F542046611C8CB206A90E54384601F00A
:1042B00031F8304601F02EF837E7152D13D10027DD
:1042C0007048867C2046611C8CB206A90F5420469B
:1042D000611C8CB206A90E54384601F01BF830461A
:1042E00001F018F821E7252D13D10027664806783C
:1042F0002046611C8CB206A90F542046611C8CB26A
:1043000006A90E54384601F005F8304601F002F8CF
:104310000BE7272D13D100275C4806782046611C47
:104320008CB206A90F542046611C8CB206A90E540B
:10433000384600F0EFFF304600F0ECFFF5E6162DB2
:1043400017D153480068070E51480068C0F307466C
:104350002046611C8CB206A90F542046611C8CB209
:1043600006A90E54384600F0D5FF304600F0D2FFC3
:10437000DBE6172D16D146480088C0F307274448CE
:1043800006782046611C8CB206A90F542046611C99
:104390008CB206A90E54384600F0BCFF304600F03F
:1043A000B9FFC2E6262D16D13648808F070A354858
:1043B00090F83C602046611C8CB206A90F54204640
:1043C000611C8CB206A90E54384600F0A3FF30469B
:1043D00000F0A0FFA9E6282D1BDB2D2D19DCA5F18F
:1043E00028001FFA80F800272648143010F80860CB
:1043F0002046611C8CB206A90F542046611C8CB269
:1044000006A90E54384600F085FF304600F082FFC2
:104410008BE62E2D13D100271A48867F2046611C7B
:104420008CB206A90F542046611C8CB206A90E540A
:10443000384600F06FFF304600F06CFF75E62F2D18
:1044400028DB322D26DCA5F12F001FFA80F800278B
:104450000C481A3010F808602046611C8CB206A97E
:104460000F542046611C8CB206A90E54384600F049
:1044700051FF304600F04EFF57E60000C45A0020BE
:104480007E010020586000208F0100208E01002056
:1044900004000020332D1ADB362D18DCA5F1330083
:1044A0001FFA80F80027FE4810F808602046611CBB
:1044B0008CB206A90F542046611C8CB206A90E547A
:1044C000384600F027FF304600F024FF2DE6372D58
:1044D0001BDB3A2D19DCA5F137001FFA80F8002705
:1044E000EF48001D10F808602046611C8CB206A938
:1044F0000F542046611C8CB206A90E54384600F0B9
:1045000009FF304600F006FF0FE63B2D15D10027CE
:10451000E3481F3890F827602046611C8CB206A93A
:104520000F542046611C8CB206A90E54384600F088
:10453000F1FE304600F0EEFEF7E53C2D18D1D848EC
:104540001F38008D070AD6481F3890F8286020468B
:10455000611C8CB206A90F542046611C8CB206A9BE
:104560000E54384600F0D6FE304600F0D3FEDCE5AF
:104570003D2D15D10027CA481F3890F82F602046DE
:10458000611C8CB206A90F542046611C8CB206A98E
:104590000E54384600F0BEFE304600F0BBFEC4E5C7
:1045A0003E2D1BDB412D19DCA5F13E001FFA80F8E2
:1045B0000027BB480C3010F808602046611C8CB204
:1045C00006A90F542046611C8CB206A90E54384629
:1045D00000F0A0FE304600F09DFEA6E5422D1BDB5C
:1045E000452D19DCA5F142001FFA80F80027AC48E0
:1045F000113010F808602046611C8CB206A90F54D7
:104600002046611C8CB206A90E54384600F082FE8A
:10461000304600F07FFE88E5462D1BDB492D19DC76
:10462000A5F146001FFA80F800279D48153010F8C4
:1046300008602046611C8CB206A90F542046611CFC
:104640008CB206A90E54384600F064FE304600F0E5
:1046500061FE6AE54A2D15D1002791481F3890F870
:1046600038602046611C8CB206A90F542046611C9C
:104670008CB206A90E54384600F04CFE304600F0CD
:1046800049FE52E54B2D18D185481F38408F070A47
:1046900083481F3890F83A602046611C8CB206A906
:1046A0000F542046611C8CB206A90E54384600F007
:1046B00031FE304600F02EFE37E54C2D15D1002797
:1046C00077481F3890F83E602046611C8CB206A9DE
:1046D0000F542046611C8CB206A90E54384600F0D7
:1046E00019FE304600F016FE1FE55D2D15D100279E
:1046F0006B481F3890F82A602046611C8CB206A9CE
:104700000F542046611C8CB206A90E54384600F0A6
:1047100001FE304600F0FEFDF2E35A2D15D161484E
:10472000008807125F4806782046611C8CB206A9F3
:104730000F542046611C8CB206A90E54384600F076
:10474000E9FD304600F0E6FDDAE3642D7DDBA32DC4
:104750007BDCA5F164001FFA80F808EBD8714910E2
:10476000C1EBC10202EB01114F4A02EB410191F88A
:10477000281001296AD108EBD8725210C2EBC2038B
:1047800003EB0212484B03EB420292F82D200F2A52
:104790000DD008EBD8725210C2EBC20303EB021229
:1047A000414B03EB420292F82D20192A3AD14046A0
:1047B00008EBD0714910A8EB410189B908EBD07121
:1047C0004A103749213151F832100F0E08EBD071E1
:1047D0004A103349213151F83210C1F3074610E035
:1047E000404608EBD0714A102D49213131F8321082
:1047F000C1F3072708EBD0714A102949213111F87C
:1048000032602046611C8CB206A90F542046611C00
:104810008CB206A90E54384600F07CFD304600F0FC
:1048200079FD6DE3404608EBD0714910A8EB4101DA
:1048300001293BD108EBD8714910C1EBC10202EB51
:104840000111194A02EB410101E0A5E041E0D1F874
:104850001E100A2291FBF2F1C1F3072708EBD87171
:104860004910C1EBC10202EB01110F4A02EB4101F9
:10487000D1F81E100A2291FBF2F1CEB22046611C43
:104880008CB206A90F542046611C8CB206A90E54A6
:10489000384600F03FFD304600F03CFD30E30000BC
:1048A00077600020C0010020E76C00200027002670
:1048B0002046611C8CB206A90F542046611C8CB2A4
:1048C00006A90E54384600F025FD304600F022FDC2
:1048D00016E3404608EBD0714910A8EB41010129CD
:1048E00047D108EBD8714910C1EBC10202EB0111AD
:1048F000FE4A02EB410191F82D100B2914DC08EB64
:10490000D8714910C1EBC10202EB0111F74A02EB69
:104910004101D1F81E10B1F57A7F02DB0027012694
:1049200016E00027002613E008EBD8714910C1EB10
:10493000C10202EB0111ED4A02EB4101D1F81E1058
:10494000B1F57A7F02DB0027002601E0002701266F
:104950002046611C8CB206A90F542046611C8CB203
:1049600006A90E54384600F0D5FC304600F0D2FCC3
:10497000C6E2002700262046611C8CB206A90F540F
:104980002046611C8CB206A90E54384600F0C2FCC9
:10499000304600F0BFFCB3E2B5F5827F21DBB5F510
:1049A000927F1EDAA5F582701FFA80F80027C8EB07
:1049B000C80000EB0810CD4901EB400090F82860DA
:1049C0002046611C8CB206A90F542046611C8CB293
:1049D00006A90E54384600F09DFC304600F09AFCC3
:1049E0008EE2B5F5927F23DBB5F5A27F20DAA5F53F
:1049F00092701FFA80F80027C8EBC80000EB08107F
:104A0000BA4901EB400090F82300C0F3031620469A
:104A1000611C8CB206A90F542046611C8CB206A9F9
:104A20000E54384600F076FC304600F073FC67E226
:104A3000A42D20DBC32D1EDCA5F1A4001FFA80F8F5
:104A40000027C8EBC80000EB0810A84901EB4000A4
:104A500090F822602046611C8CB206A90F542046B3
:104A6000611C8CB206A90E54384600F053FC304647
:104A700000F050FC44E2C42D20DBE32D1EDCA5F148
:104A8000C4001FFA80F80027C8EBC80000EB08102C
:104A9000964901EB400090F82D602046611C8CB2D5
:104AA00006A90F542046611C8CB206A90E54384644
:104AB00000F030FC304600F02DFC21E2E42D21DB3B
:104AC000B5F5827F1EDAA5F1E4001FFA80F8002711
:104AD000C8EBC80000EB0810844901EB400090F8D7
:104AE00027602046611C8CB206A90F542046611C29
:104AF0008CB206A90E54384600F00CFC304600F08B
:104B000009FCFDE1B5F5A27F21DBB5F5B27F1EDA28
:104B1000A5F5A2701FFA80F80027C8EBC80000EBCB
:104B20000810724901EB400090F829602046611C92
:104B30008CB206A90F542046611C8CB206A90E54F3
:104B4000384600F0E7FB304600F0E4FBD8E1B5F56D
:104B5000B27F32DBB5F5D27F2FDAA5F5B2701FFA3E
:104B600080F80027404608EBD0714910A8EB4101BE
:104B700049B9C8EBC80000EB08105C4901EB4000E4
:104B800090F82B6008E0C8EBC80000EB081057490C
:104B900001EB400090F82C602046611C8CB206A905
:104BA0000F542046611C8CB206A90E54384600F002
:104BB000B1FB304600F0AEFBA2E1B5F5D27F23DBBE
:104BC000B5F5E27F20DAA5F5D2701FFA80F800274C
:104BD000C8EBC80000EB0810444901EB400090F816
:104BE000230000F00F062046611C8CB206A90F546A
:104BF0002046611C8CB206A90E54384600F08AFB90
:104C0000304600F087FB7BE140F2CA20854212D19A
:104C1000002756262046611C8CB206A90F54204658
:104C2000611C8CB206A90E54384600F073FB304666
:104C300000F070FB64E140F2CB20854222DB40F2C1
:104C4000D52085421EDCA5F2CB2080B202902849F7
:104C5000029811F810700121029801EB40012448DC
:104C6000465C2046611C8CB206A90F542046611C8C
:104C70008CB206A90E54384600F04CFB304600F0CA
:104C800049FB3DE1B5F5487F13D100271948C67CA3
:104C90002046611C8CB206A90F542046611C8CB2C0
:104CA00006A90E54384600F035FB304600F032FBC2
:104CB00026E1B5F5487F27DD40F25130854223DCFF
:104CC000A5F548700C4931F810000712A5F5487099
:104CD00011F810602046611C8CB206A90F542046C2
:104CE000611C8CB206A90E54384607E0E76C002020
:104CF000C4620020586000206865002000F00AFBB4
:104D0000304600F007FBFBE0B5F5FA6F1CDB40F620
:104D10003400854218DC2846FFF710F8029002980C
:104D2000070A0298C6B22046611C8CB206A90F542D
:104D30002046611C8CB206A90E54384600F0EAFAEF
:104D4000304600F0E7FADBE04FF6F250854213D12F
:104D50000027F84806782046611C8CB206A90F543B
:104D60002046611C8CB206A90E54384600F0D2FAD7
:104D7000304600F0CFFAC3E042F6D040854237DB40
:104D800042F6AF70854233DCA5F53050D03817219C
:104D9000B0FBF1F0C0B202900298C0EBC00101EB91
:104DA0000010E54901EB40000090A5F53050D038E7
:104DB0001721B0FBF1F201FB12000190DDE90001C7
:104DC00030F81100070ADDE9000110F811602046F3
:104DD000611C8CB206A90F542046611C8CB206A936
:104DE0000E54384600F096FA304600F093FA87E009
:104DF00043F29020854236DB43F29740854232DC15
:104E0000A5F5485090380A21B0FBF1F0C0B20290ED
:104E1000029800EB400101EB0010C84908440090E3
:104E2000A5F5485090380A21B0FBF1F201FB1200C1
:104E30000190DDE9000130F81100070ADDE9000109
:104E400010F811602046611C8CB206A90F54204650
:104E5000611C8CB206A90E54384600F05BFA30464D
:104E600000F058FA4CE048F2A800854236DB48F2E0
:104E7000B010854232DCA5F50040A8383521B0FBE2
:104E8000F1F0C0B202900298C0EB0010C0EBC0007D
:104E9000AB4908440090A5F50040A8383521B0FB87
:104EA000F1F201FB12000190DDE9000130F8110080
:104EB000070ADDE9000110F811602046611C8CB280
:104EC00006A90F542046611C8CB206A90E54384620
:104ED00000F020FA304600F01DFA11E0002700260D
:104EE0002046611C8CB206A90F542046611C8CB26E
:104EF00006A90E54384600F00DFA304600F00AFAC2
:104F00000AF1010000F0FF0A05988245FFF6F5A8B6
:104F10008C4807788C4806782046611C8CB206A91C
:104F20000F542046611C8CB206A90E5451980428D7
:104F300006D105984200C91C84480DF006FC34E0F7
:104F4000519840B9224606A981480DF043FC2046FD
:104F5000FDF70FFF29E09BF800008DF818009BF883
:104F600001008DF8190000208DF81A008DF81B0043
:104F70000321059801EB4000000A8DF81C000598FC
:104F800001EB4000C0B28DF81D00059801EB400018
:104F900000EB090206A96F480DF0D7FB0321059825
:104FA00001EB400048446C4908805CE06B48407865
:104FB000192858D11BF809602046611C8CB264493D
:104FC0000E54304600F0A6F909F101001BF800600C
:104FD0002046611C8CB25E490E54304600F09AF9AE
:104FE0005F4806792046611C8CB259490E54304600
:104FF00000F090F95A4806782046611C8CB254495A
:105000000E54304600F086F9554846782046611C1B
:105010008CB24F490E54304600F07CF950488678E7
:105020002046611C8CB24A490E54304600F072F999
:105030004B48C6782046611C8CB245490E54304618
:1050400000F068F93F4806782046611C8CB2404960
:105050000E543D4806782046611C8CB23C490E54E3
:105060002046FDF786FE53B0BDE8F08F2DE9F047EE
:1050700007463C480078401C3A4908703A48007896
:105080003A490978884202D00020BDE8F0873348C9
:105090000078FF280AD031480078314909798842E0
:1050A00004D02E48007808B10020EEE72B48407865
:1050B000192866D10421294800F03CF90546274803
:1050C00040792649097900EB0120A84201D000204F
:1050D000DBE7224880782149C978884202DB1F48F3
:1050E000C07801E01D48807880461C4880781B49C4
:1050F000C978884202DB1948807801E01748C078F7
:10510000814617480079404503DB1548007948453A
:1051100001DD0020B9E7134800780DF077FAF3F7C6
:10512000E3F8142190FBF1F201FB1200C6B2002457
:1051300023E0000009000020E76C0020C77A00206F
:10514000DA6A002096010020950100209861002075
:10515000585E0020C45A00207E010020585D0020C7
:105160005860002094010020860100208701002063
:105170006420FAF77FFB601CC4B2B442F8DB012064
:1051800083E75D484078032809D05B4840780628CB
:1051900005D059484078102801D0002075E75648BE
:1051A000C178807801EB0020092847D15248407827
:1051B00006281FD15048807950490978884201D08B
:1051C000002062E74C48C0794C494978884201D0B8
:1051D00000205AE74848007A48498978884201D037
:1051E000002052E74448407A4449C978884201D0B7
:1051F00000204AE740484078032808D1F3F774F8C4
:10520000052190FBF1F201FB12003D4908703C487A
:105210000078012801D0002037E7F3F765F8142162
:1052200090FBF1F201FB1200C6B2002404E06420FE
:10523000FAF720FB601CC4B2B442F8DB2E48407879
:10524000062822D1082F20DC2B48C078022806DA55
:105250002A48007C00F00100B8B1002015E726487C
:10526000C078042806DA2548007C00F0020060B10E
:1052700000200AE72048C078082806D11F48007C93
:1052800000F0040008B10020FFE61E480078801EF0
:10529000C1B2194800F04EF805461A480078401E81
:1052A0001549095C17480078801E134A105C01EB11
:1052B0000020A84201D10120E7E60020E5E610B574
:1052C0000D48C0780C49897800EB012084B2204653
:1052D000FFF7CCFE60B1FDF738FD00F015F8064988
:1052E0000020FEF7DCFD04490020FDF7FFFE01E091
:1052F000FDF750FC10BD7047585D0020586000203D
:105300008401002087010020FF20184908701849F7
:1053100008707047164A127882EA0001154A525CFA
:10532000124B1B785A40124B1A70134A525C0F4BA7
:105330001A707047F0B502460B46FF24FF25002681
:105340000BE03046771CFEB2105C80EA040109488D
:10535000405C80EA05040848455C181EA3F101077B
:10536000FBB2EED145EA0420F0BD0000950100201B
:1053700096010020CE4F0208CE50020870477047B9
:1053800010B5FDF743FD10BD10B5044614222146AB
:10539000FE480DF0DAF91422FC4940F2BA20F8F781
:1053A00040F810BD10B50446F9480078F84949782E
:1053B00000EB0120F649897800EB0140F449C978F7
:1053C00000EB0160D4F8B410884212D1142204F129
:1053D0003401EE480DF04AF958B10021472001553B
:1053E000142204F13401E9480DF0F4F9E748FFF71D
:1053F000CBFFE748007994F8C81088421CD094F895
:10540000C800002818DD94F8C800FF2814DA94F8C2
:10541000C800DF490871084601790620F7F77CFFCC
:10542000DB480079DB49087008460078DA4981F8E2
:10543000F800002006F094F994F8F800D5490978AE
:1054400088421BD094F8F800C0B194F8F800FF2807
:1054500014D094F8F800CF49087008460078CE4977
:1054600081F8F800CB480078C949087108460179ED
:105470000620F7F751FF002006F072F9C4480079C2
:1054800094F84910884215D094F84900002811DD9D
:1054900094F84900FF280DDA94F84900BC490871D6
:1054A000084601790620F7F737FFB9480079BA496D
:1054B00081F84900D4F8CC0001F018FCB74909681C
:1054C00088420CD0D4F8CC0048B1D4F8CC0001F01C
:1054D0000DFCB24908600846006805F0AEFC10BD3E
:1054E00010B5AB480078AA49497800EB0120A849DB
:1054F000897800EB0140A649C97800EB0160A64914
:10550000C1F8B400A248007981F8C800A048007929
:1055100081F84900A1480068C1F8CC00012081F859
:105520004800142299499C4834300DF053F910BDBD
:105530007047704770477047704710B5944880684F
:10554000B0F5964F04D14FF49640FAF70AF930E0DF
:105550008F488068B0F5165F04D14FF41650FAF703
:1055600000F926E08A488068B0F5164F04D14FF460
:105570001640FAF7F6F81CE085488068B0F5614FF0
:1055800004D14FF46140FAF7ECF812E080488068EB
:10559000B0F5E13F04D14FF4E130FAF7E2F808E06A
:1055A0007B488068B0F5963F03D14FF49630FAF708
:1055B000D8F810BD76488068B0F5165F01D1052097
:1055C000704773488068B0F5964F01D10620F7E721
:1055D0006F488068B0F5164F01D10720F0E76C489E
:1055E0008068B0F5614F01D10820E9E7684880681C
:1055F000B0F5E13F01D10920E2E765488068B0F5E8
:10560000963F01D10A20DBE70620D9E77047024622
:1056100000207047704730B504460B46002214B195
:10562000032C2FD117E0002112E0C1EBC10000EBE9
:1056300001105B4D05EB400090F82800012805D1D2
:105640009A4201D1084630BD501CC2B2481CC1B2BA
:105650002029EADB16E0002111E0C1EBC10000EBDC
:1056600001104F4D05EB400090F8280028B99A42F0
:1056700001D10846E7E7501CC2B2481CC1B220293C
:10568000EBDB00BF00BF4FF0FF30DCE770B5044636
:105690000D4621460020FFF7BEFFC6B2701C10B1B8
:1056A0002E70012070BD0020FCE770B504460D4649
:1056B00021460320FFF7AFFFC6B2701C10B12E7059
:1056C000012070BD0020FCE7F8B505460E461446E3
:1056D00035B1012D59D0022D75D0032D74D17DE047
:1056E00024B92C4800780FF013FAF8BD012C04D12E
:1056F000274988680FF00CFAF7E7022C04D12449F7
:10570000887C0FF005FAF0E7032C04D123480068E9
:105710000FF0FEF9E9E7042C08DB072C06DC211F5B
:105720001B4A1A32505C0FF0F3F9DEE7082C09DB54
:105730000B2C07DCA4F10801154A1F32505C0FF056
:10574000E7F9D2E70C2C09DB0F2C07DCA4F10C01E4
:105750000F4A2332505C0FF0DBF9C6E7102C04D15E
:105760000B49088D0FF0D4F9BFE7112C1DDB302C4D
:105770001BDCA4F11101C1EBC10202EB0111084ACB
:1057800002EB410191F82D000CE09FE0C462002083
:10579000586000208E010020D86200200400002004
:1057A000E76C00200FF0B4F99FE7312C04D1F849E1
:1057B000888F0FF0ADF998E7322C06D1F449887F35
:1057C0000FF0A6F991E7A6E0A4E0332C05D1F0494B
:1057D00091F83E000FF09CF987E79DE0694620466E
:1057E000FFF763FF9DF80000C0EBC00101EB001064
:1057F000E84901EB400090F82D00002865DD9DF898
:105800000000C0EBC00101EB0010E24901EB4000D9
:1058100090F82800E8BB9DF80000C0EBC00101EB48
:105820000010DC4901EB400090F82D000C280CDB47
:105830009DF80000C0EBC00101EB0010D54901EB61
:10584000400090F82D00162819DD9DF80000C0EBEF
:10585000C00101EB0010CF4901EB400090F82D0092
:10586000172820DB9DF80000C0EBC00101EB001001
:10587000C84901EB400090F82D001E2813DC9DF86C
:105880000000C0EBC00101EB0010C24901EB400079
:1058900000E01AE090F82600012801D1002024E75A
:1058A0004FF07E5021E79DF80000C0EBC00101EBF6
:1058B0000010B84901EB400090F82600012802D101
:1058C0004FF07E5011E700200FE700BF69462046E9
:1058D000FFF7DCFE9DF80000C0EBC00101EB0010FB
:1058E000AC4901EB400090F82D00002811DD9DF837
:1058F0000010C1EBC10202EB0111A64A02EB41010B
:10590000D1F81E000FF0ECF80746A3490EF0B6FFE1
:10591000EBE600BF00BF00BF00BF00BFE5E62DE91A
:10592000F8430546884614461E4625B1012D7DD014
:10593000032D7CD11EE2D4B930460FF0B1F8944962
:10594000087130460FF0ACF89449087030460FF0FB
:10595000A7F8C7B239460620F7F7DEFCF2F7E8FCF5
:10596000002005F0FDFE002006F0AEFDC0E1012C98
:105970007ED130460FF094F88549886008468068EB
:10598000B0F5165F13D1002008730846017B15207F
:10599000F7F7C2FC7E48017B1320F7F7BDFC4FF4FC
:1059A0001650F9F7DEFE06207D490870A0E1784820
:1059B0008068B0F5964F14D10120754908730846E8
:1059C000017B1520F7F7A8FC7148017B1320F7F73E
:1059D000A3FC4FF49640F9F7C4FE03207049087009
:1059E00086E16B488068B0F5164F0FD102206849F8
:1059F00008730846017B1520F7F78EFC4FF416401C
:105A0000F9F7AFFE02206649087071E160488068CE
:105A1000B0F5614F17D103205D4908730846017B3B
:105A20001520F7F779FC5A48017B01E061E16CE24F
:105A30001320F7F771FC0120594908704FF46140B9
:105A4000F9F78FFE54E152488068B0F5E13F16D176
:105A500004204F4908730846017B1520F7F75CFCCA
:105A60004B48017B1320F7F757FC01204C4900E01D
:105A70001FE008704FF4E130F9F773FE38E1444855
:105A80008068B0F5963F91D10520414908730846DA
:105A9000017B1520F7F740FC3D48017B1320F7F709
:105AA0003BFC01203E4908704FF49630F9F759FE4F
:105AB0001EE1022C0AD130460EF0F2FF3449887400
:105AC0000846817C1420F7F727FC11E1032C20D134
:105AD00030460EF0E5FF3349086008460068010EC5
:105AE0001620F7F719FC2F480068C0F3074117206C
:105AF000F7F712FC2B480088C0F307211820F7F7AE
:105B00000BFC284801781920F7F706FCF2F710FC87
:105B1000EEE0042C11DB072C0FDC30460EF0C0FF4A
:105B2000C2B2201F1A491A310A54221F0B46995C2F
:105B30002F3290B2F7F7F0FBDAE0082C12DB0B2CD7
:105B400010DC30460EF0ACFFC2B2A4F108001049E0
:105B50001F310A5402460B46995C333290B2F7F774
:105B6000DBFBC5E00C2C1FDB0F2C1DDC30460EF0E0
:105B700097FFC2B2A4F10C00054923310A54024632
:105B80000B46995C373290B2F7F7C6FBB0E00000E5
:105B900058600020E76C002000007A448E0100204D
:105BA0008901002004000020102C11D130460EF095
:105BB00077FFF84908850846008D010A3C20F7F771
:105BC000ABFBF44890F828103D20F7F7A5FB8FE0D9
:105BD000112C45DB302C43DCEF4930460EF0ACFF96
:105BE0001BD230460EF05CFFC1B2A4F11100C0EB35
:105BF000C00202EB0010E94A02EB400080F82D10D1
:105C00000021A4F11100C0EBC00202EB0010E34A36
:105C100002EB400080F828101EE0E14930460FF00A
:105C20008BF807460EF03CFFC1B2A4F11100C0EBA7
:105C3000C00202EB0010D94A02EB400080F82D10A0
:105C40000121A4F11100C0EBC00202EB0010D34A05
:105C500002EB400080F828100120D249487047E04C
:105C6000312C13D130460EF01BFFCA4988870846F5
:105C7000808F010A1B20F7F74FFBC64890F83C10B5
:105C80001C20F7F749FBFBF79BFC31E0322C05D1D8
:105C900030460EF005FFBF49887729E0332C27D125
:105CA00030460EF0FDFEBB4981F83E00084690F8F4
:105CB0003E0001281CD10846817F2E20F7F72CFBDF
:105CC000B44A1A32115D04F12F00F7F725FBB14AEF
:105CD0001F32115D04F13300F7F71EFBAD4A23328A
:105CE000115D04F13700F7F717FB0120AE4908708A
:105CF0000CE169462046FFF7C9FC9DF8000020280A
:105D000000DB03E19DF80000C0EBC00101EB0010D7
:105D1000A24901EB400090F82800012829D19DF804
:105D20000000C0EBC00101EB00109C4901EB4000FA
:105D300090F82D0058B903209DF80010C1EBC10266
:105D400002EB0111954A02EB410181F82D009749C0
:105D500030460EF025FF07460EF086FE9DF8001037
:105D6000C1EBC10202EB01118C4A02EB4101C1F807
:105D70001E00CBE069462046FFF797FC9DF8000027
:105D8000202800DBC2E00120864948709DF8000011
:105D9000C0EBC00101EB0010804901EB400090F81E
:105DA0002800E8BB9DF80000C0EBC00101EB00102B
:105DB0007A4901EB400090F82D0058B901209DF878
:105DC0000010C1EBC10202EB0111744A02EB410168
:105DD00081F82D00754930460EF0E2FE07460EF0C0
:105DE00043FE9DF80010C1EBC10202EB01116B4AAA
:105DF00002EB4101C1F81E009DF80000C0EBC0019C
:105E000001EB0010114601EB400090F82D000C282A
:105E10000EDB9DF80000C0EBC00101EB001000E0BC
:105E200048E0114601EB400090F82D00162819DDDE
:105E30009DF80000C0EBC00101EB0010574901EBD9
:105E4000400090F82D00172820DB9DF80000C0EBE3
:105E5000C00101EB0010514901EB400090F82D000A
:105E60001E2813DC002130460EF0CAFD01D10120AE
:105E700000E000209DF80010C1EBC10202EB01110F
:105E8000464A02EB410181F826003DE00021304600
:105E90000EF0B6FD01D0012000E000209DF80010BA
:105EA000C1EBC10202EB01113C4A02EB410181F856
:105EB000260029E09DF80000C0EBC00101EB0010B6
:105EC000364901EB400090F82D0058B903209DF8A9
:105ED0000010C1EBC10202EB0111304A02EB41019B
:105EE00081F82D00314930460EF05AFE07460EF07B
:105EF000BBFD9DF80010C1EBC10202EB0111274A66
:105F000002EB4101C1F81E0000E000BF00BFBDE888
:105F1000F883F8B504460F4615461E46052C5AD29E
:105F2000DFE804F04803471D460069462846FFF7AE
:105F3000ADFB9DF80000202800DB4DE00120194951
:105F400048709DF80010C1EBC10202EB0111134A29
:105F500002EB4100152231460CF0F7FB3CE06946AC
:105F60002846FFF7A2FB9DF80000202800DB33E065
:105F700001200C4948709DF80010C1EBC10202EBF2
:105F80000111064A02EB4100152231460CF0DDFBFF
:105F900022E00000586000200000F841E76C00207B
:105FA0000000F041E20100208201002000007A445C
:105FB00012E011E005EB450000EB0510FC49084438
:105FC000316840F8061F71684160317A0172012022
:105FD000F849887000BF00BF00BFF8BDF0B50446A7
:105FE000012C7CD1202A00DB82E05F2B09D1002527
:105FF000C2EBC20606EB0216EF4F07EB460686F829
:106000002D503E2B09D10325C2EBC20606EB02162A
:10601000E94F07EB460686F82D50402B09D10425A1
:10602000C2EBC20606EB0216E34F07EB460686F804
:106030002D50032B1ED10D25C2EBC20606EB021616
:10604000DD4F07EB460686F82D50C2EBC20505EB87
:1060500002153E4606EB450595F8230000F00F00BB
:1060600040F01000C2EBC20505EB021506EB45053A
:1060700085F82300052B1ED11325C2EBC20606EBC3
:106080000216CD4F07EB460686F82D50C2EBC2052F
:1060900005EB02153E4606EB450595F8230000F09A
:1060A0000F0040F03000C2EBC20505EB021506EB15
:1060B000450585F82300052B18D0032B16D0C2EB1D
:1060C000C20505EB0215BC4E06EB450595F823000D
:1060D00000F00F0040F04000C2EBC20500E006E017
:1060E00005EB021506EB450585F8230000E000BF2F
:1060F00000BFF0BD0246012A04D0022A0FD0042AB4
:106100000FD10DE0202909DAC1EBC10000EB01102D
:10611000A94B03EB400090F82700704702E001E034
:1061200000E000BF00BF00BFF7E730B5012804D092
:10613000022811D0042810D10DE053B2C1EBC104E4
:1061400004EB01149C4D05EB440484F82730012333
:10615000984C637002E001E000E000BF00BF30BD7A
:10616000704738B505460C4625B1012D0DD0032DDD
:1061700033D11EE0342C07DA04EB440000EB0410AA
:106180008B490844801D38BD28E069462046FFF74A
:106190007DFA9DF80000202801DB0020F3E79DF840
:1061A0000000C0EBC00101EB0010834901EB40008F
:1061B000E9E769462046FFF778FA9DF800002028B5
:1061C00001DB0020DFE79DF80000C0EBC00101EB20
:1061D0000010794901EB4000D5E700BF00BF77A070
:1061E000D1E738B505460C4625B1012D0CD0032D5D
:1061F00034D11EE0342C06DA04EB440000EB04102A
:106200006B49084438BD2AE069462046FFF73EFA4C
:106210009DF80000202801DB0020F3E79DF8000036
:10622000C0EBC00101EB0010634901EB40001530E9
:10623000E8E769462046FFF738FA9DF80000202875
:1062400001DB0020DEE79DF80000C0EBC00101EBA0
:106250000010594901EB40001530D3E700BF00BFE3
:1062600056A0CFE738B504460D460CB95F2038BDBF
:10627000012C7DD169462846FFF708FA9DF80000F9
:10628000202801DB0020F2E79DF80000C0EBC001F0
:1062900001EB0010484901EB400090F8280008B9D4
:1062A0005F20E4E79DF80000C0EBC00101EB0010A7
:1062B000414901EB400090F82D0003280CD09DF8D7
:1062C0000000C0EBC00101EB00103B4901EB4000B6
:1062D00090F82D00072801D13E20C8E79DF8000066
:1062E000C0EBC00101EB0010334901EB400090F816
:1062F0002D0004280CD09DF80000C0EBC00101EB7C
:1063000000102D4901EB400090F82D00082801D124
:106310004020ACE79DF80000C0EBC00101EB00108D
:10632000254901EB400090F82D000D2801D10220F5
:106330009DE79DF80000C0EBC00101EB00101E4975
:1063400001EB400090F82D0013280CD09DF80000C0
:10635000C0EBC00101EB0010174901EB400090F8C1
:106360002D000B2802D1052081E701E05F207EE7A8
:10637000032C05D1052D01DB002078E75F2076E7AF
:106380005F2074E7F8B506460F4615461C46052EF5
:1063900055D2DFE806F04603452944006946284601
:1063A000FFF774F99DF8000020280BDB48E000009F
:1063B000C77A0020E2010020E76C00206E756C6C4B
:1063C000000000000120C84948709DF80000C0EBA3
:1063D000C00101EB0010C54901EB4000216840F805
:1063E000151F616841602BE069462846FFF75DF99B
:1063F0009DF80000202800DB22E00120BA49487007
:106400009DF80000C0EBC00101EB0010B74901EBA3
:106410004000216840F8151F6168416010E00FE0FE
:106420000EE005EB450000EB0510B149084421687A
:106430000160A18881800120AB49887000E000BF25
:1064400000BFF8BDAB48704710B5AB480088FF28C7
:1064500035D008DC002834D0012813D002281FD002
:10646000942847D12AE0A0F2E530D0B10A280AD01A
:10647000A0F2E510002830D0A0F57A403538002889
:1064800038D11DE000BF14229CA1A0480CF0A2F955
:1064900014229FA1A0480CF09DF940F2EF3010BDEE
:1064A00000BF14229DA199480CF094F914229EA1DA
:1064B00099480CF08FF940F2E530F0E700BF00BFDB
:1064C00000BF14229BA191480CF084F914229DA1D5
:1064D00091480CF07FF99420E1E714229DA18B48AC
:1064E0000CF078F914229EA18B480CF073F940F25D
:1064F000CA50D4E780480088D1E78448704786486E
:10650000704710B5044601207749087114222146CE
:106510007E480CF01AF910BD10B5044601207249EE
:106520000871142221467C480CF00FF910BD10B5FB
:106530000446E1B21D20F6F7EFFE21122020F6F707
:10654000EBFE4CB1FF2C07D04FF6FF70844203D016
:10655000012C01D0022C00D110BD6748048000BF7F
:10656000FAE770B505460C4616462246294681488C
:106570000CF0EBF82046FCF7FCFB70BD01207047E7
:1065800018B101217C4A116002E000217A4A1160B1
:1065900070477A480079704710B50446210E1620DE
:1065A000F6F7BAFEC4F307411720F6F7B5FEC4F3B9
:1065B00007211820F6F7B0FEE1B21920F6F7ACFE7D
:1065C00010BD10B5044621461220F6F7A5FE10BDF9
:1065D000002070476A48007860B16A480088002847
:1065E00005DD68480088401E6649088002E00020FA
:1065F00063490870704702460020704770470146A3
:106600000020704702460020704701460020704776
:1066100001460020704710B500220021002019E03B
:10662000C0EBC00303EB0013304C04EB430393F8BF
:106630002830012B06D1544B9854544B1A54531CF8
:10664000DAB205E0524B5854524B19544B1CD9B294
:10665000431CD8B22028E3DB4F4B1A704F4B197004
:1066600010BD30B504460A46002314B1032C2FD1C7
:1066700017E0002112E0C1EBC10000EB01101B4D3F
:1066800005EB400090F82800012805D1914201D186
:10669000184630BD581CC3B2481CC1B22029EADBE1
:1066A00017E0002111E0C1EBC10000EB01100F4D1C
:1066B00005EB400090F8280028B9914201D1184616
:1066C000E7E7581CC3B2481CC1B22029EBDB00E04D
:1066D00000BF00BF4FF0FF30DBE7014600207047EE
:1066E0000246002070470000E2010020E76C002015
:1066F000C77A0020C4620020C00100204E455449E2
:106700005820436F6E74726F6C7300009801002004
:106710004E43434200000000AC0100204A65744330
:106720006F6E74726F6C73004A65742050726F6480
:106730007563740054656D636F436F6E74726F6C34
:106740007300000054656D636F2050726F64756351
:10675000740000004D6963726F67726F0000000083
:106760004D6963726F67726F2050726F64756374E6
:1067700000000000585E0020A00121425860002067
:106780000A0000200C000020E8640020286500209A
:106790000865002048650020F3010020F501002075
:1067A000F44908807047F44908607047F34908606D
:1067B000704710B50020FFF7F9FF0020FFF7F3FF47
:1067C000EF49888FFFF7ECFFED4991F83C10090283
:1067D000EB4A928F41EA222188B2F9F7D6FAE848CB
:1067E00090F83C000002E649898F40EA212081B2FE
:1067F000E448A0F8441010BD30B587B00025E24849
:10680000007800F00200A0B3E048E1490860E148E8
:106810000288E1480168DE4800680BF096FFDD4819
:106820000088DE49088000BFDD4800680088ADF8B8
:106830001800DB4800684088ADF81A0000BFD8484F
:106840000068C18806A8F9F70EFA04460120002363
:106850004FF41672CD49009001A804F0BAFA05462B
:106860002DB101232A46C94901A805F0F0FD0020F9
:10687000A08007B030BDC14800687047BF480068BD
:10688000401C08B1012070470020FCE7BA480068AE
:106890007047C44908607047C24800687047B548EF
:1068A0000088704710B50346002033B1D3F801408B
:1068B0000C60B3F805401480062010BD2DE9F047A8
:1068C00086B005468A4617461E46DDF83880002405
:1068D000A14600200090B448007850B9B8F1010FEB
:1068E00007D1A6480068002803DA002006B0BDE8FA
:1068F000F0878120AD4908700220ADF80800288992
:106900004FF6FF71884206D02889002801DDA87A59
:1069100008B1287848B9A3480068019095480088D4
:1069200000900B20A14948700EE02878062808D175
:106930006A4601A92846FFF7B5FF0A209B4948701F
:1069400002E04FF0FF30D1E701980390BDF800005E
:10695000ADF80A000020049005900224321D91B287
:10696000924A101904F066F9044490490819324615
:1069700039460BF0EAFE3444B8F1010F0ED18A48D3
:10698000007820B921468948FAF7EBFB06E0224659
:10699000864987480BF0D9FE86490C80A14640F213
:1069A000762182480BF050FF002448469EE72DE9EF
:1069B000F0478EB081460C4616461F464FF0000841
:1069C00000200D9009900A900B900C900590069075
:1069D0000790089001900290039004900025824651
:1069E0007148007848B9012F07D164480068002831
:1069F00003DA00200EB0BDE8F0876848B0F80080E8
:106A000063480460012F0CD16748007848B9B8F199
:106A1000000F01DA0020EDE7B8F1000F01D10020EE
:106A2000E8E74FF000082078812804D05E4800781D
:106A300008B90020DEE794F801A00DA9A01C04F01D
:106A4000FEF800200A90ADF826000690ADF816007A
:106A50000290ADF806005448007840B950480068EC
:106A6000C088ADF826004E48006800680A90BDF85E
:106A70003400001F80B20D90BAF10A0F03D0BAF1B2
:106A80000B0F3CD124E0FFF701FF0A99884208D19F
:106A9000FFF705FFBDF82610884202D100200D90B7
:106AA00015E009A9484604F06FF9BDF83400B0427A
:106AB0000BDA002504E0281D205C6055681C85B2B7
:106AC000BDF834008542F6DB01E000200D9017E0B0
:106AD00009A9484604F058F9BDF83400B0420BDA71
:106AE000002504E0281D205C6055681C85B2BDF8B7
:106AF00034008542F6DB01E000200D9000E000BF8D
:106B000000BFBDF8340075E70021B0B10622027065
:106B1000194A1268C0F80120421C164B1B88A0F8C5
:106B2000053000220281827200BF04E0002300F1E0
:106B30000B025354491C0729F8DB70470021C0B1F0
:106B400006220270174A1268C0F80120421C094B45
:106B50001B88A0F805304FF6FF7202810022827276
:106B600000BF04E0002300F10B025354491C072925
:106B7000F8DB7047D0010020D4010020CC010020B8
:106B8000586000208855002040010020CC6500207E
:106B9000DC0100203C01002034010020E001002045
:106BA00048010020D8010020E801002024680020CE
:106BB000A37E0020EA0100200146474830F811007A
:106BC00070477047014641F288304843800A704759
:106BD000014642F210704843800A704702463F481F
:106BE000805C022804D141F288304843800A704713
:106BF0003A48805C012804D144F620604843800A6A
:106C0000F5E73648805C032804D142F2107048430F
:106C1000800AECE73148805C042802D02F48805C71
:106C200020B940F6B8304843800AE0E700BFDEE70D
:106C30002020704701462A4850F831007047002252
:106C4000274941F830207047F0B502460C46002332
:106C500000200021002511462546224E36F81160FD
:106C6000AE1B33B2642B02DA13F1640F08DC1D4E45
:106C700036F8116006EB63061A4F27F8116026E01C
:106C8000184E36F81160C1EBC10707EB0117DFF8AA
:106C900058C00CEB470797F822707E43114F27F836
:106CA00011603E4636F811602E4427F811603E46CA
:106CB00036F81160C1EBC10707EB01170CEB470772
:106CC00097F8227096FBF7F6064F27F81160054EED
:106CD00036F81100F0BD0000E0160020A772002079
:106CE000986000209A6A0020E76C00207047704787
:106CF0002DE9F04F81460B4608254FF0000AA9F117
:106D0000010000F0FF094C464FEA690900BFF9484D
:106D10000078012874D1B9F1030F5EDC642700BF4D
:106D200009EB0910F44E06EB4001088C984205DB94
:106D3000F24800EBC4004068BDE8F08F0888984234
:106D400003DCEE4850F83400F6E7082241E031F861
:106D50001200984222DC501E31F8100098421DDBD0
:106D6000521E31F81260501C31F81000351A9DB1D6
:106D700031F81200C01A00FB07F898FBF5F802FB87
:106D80000788DF4850F824C00CFB08FC9CFBF7FC8C
:106D9000DA4850F8340084446046CDE70DB94FF02E
:106DA000010A284605EBD076751031F8120098429A
:106DB00001DD2A4400E0521B002A03DCCF4850F8D2
:106DC0003400B9E7102A04DBCC4800EBC40040686B
:106DD000B2E7BAF1000FBAD0D5E064271925C94946
:106DE0000888984203DBC54850F83400A4E7B1F89E
:106DF0006400984205DCC14800EBC40040689BE792
:106E000064E019225EE0488E98422DDA192628E0C7
:106E100031F81600984222DC701C31F810009842BC
:106E20001DDB701C31F8100031F816B0A0EB0B051B
:106E30009DB131F81600181A00FB07F898FBF5F819
:106E400006FB0788AE4850F824C00CFB08FC9CFBEE
:106E5000F7FCAA4850F83400844460466CE7701C84
:106E6000C6B2322ED4DB2CE0002628E031F8160022
:106E7000984222DC701C31F8100098421DDB701C17
:106E800031F8100031F816B0A0EB0B059DB131F8C8
:106E90001600181A00FB07F898FBF5F806FB0788A0
:106EA000974850F824C00CFB08FC9CFBF7FC934867
:106EB00050F83400844460463EE7701CC6B2192E78
:106EC000D4DB00BFBAF1000F9DD05CE0642709EB72
:106ED0000910894E06EB40010825088C984204DB16
:106EE000864800EBC400406826E70888984203DC27
:106EF000824850F834001FE7082241E031F81200C0
:106F0000984222DC501E31F8100098421DDB521EC0
:106F100031F81260501C31F81000351A9DB131F86B
:106F20001200C01A00FB07F898FBF5F802FB07886F
:106F3000734850F824C00CFB08FC9CFBF7FC6F481E
:106F400050F8340084446046F6E60DB94FF0010A6B
:106F5000284605EBD076751031F81200984201DD15
:106F60002A4400E0521B002A03DC644850F8340035
:106F7000E2E6102A04DB614800EBC4004068DBE66F
:106F8000BAF1000FBAD00020D6E62DE9F05F07462F
:106F90000E460125A7F1140007B200BFC7EB07108A
:106FA000C0EBC00058490844093005EB450100EB2F
:106FB0004104B4F90000FFF79AFEB04205D1D4F8BD
:106FC0000200FFF793FEBDE8F09FB4F90000FFF761
:106FD0008EFEB04208DD34F9060CFFF788FEB042A1
:106FE00002DA681E05B203E0681C05B20E2DD5DD7D
:106FF00000BF0F2D21DBC7EB0710C0EBC0004249DB
:10700000084400F10F04B4F9000034F9061C88426A
:1070100009DD34F9060CB04202DB54F8040CD2E767
:10702000D4F80200CFE734F9060CB04202DC54F881
:10703000040CC8E7D4F80200C5E7C7EB0710C0EBA3
:10704000C00031490844093005EB450100EB41041B
:10705000B4F90600FFF74BFE0146B4F90000FFF754
:1070600046FE081A05B2BDB1B4F90000FFF73FFEB5
:10707000A6EB000A50460DF033FD814623494846F1
:107080000DF08EFD814628460DF02AFD82465146C0
:1070900048460DF0F3FB8146A068FFF727FE014646
:1070A000D4F80200FFF722FEA1EB000A50460DF0D3
:1070B00017FD8046002140460DF0A2FC15D0414648
:1070C00048460DF06DFD8146104948460DF0D6FB4F
:1070D0008146D4F80200FFF709FE83460DF000FD5B
:1070E000824649460DF05CFB814648460DF0BCFCEB
:1070F00069E700007400002082540208CC530208A3
:10710000A45302081C540208DA6A002000007A44E2
:107110002DE9F0410027AD4C52E1FFF789FDB8425F
:107120007EDD94F92300C0F30710A949C85594F8EF
:107130002700002875D194F82D00002872D0384619
:10714000FFF73AFD064694F82800A8BB14F8235F21
:1071500005F0F00500BF68B22070A07A233C0C282F
:107160000CDB94F82D00162808DCB6F5006F01D969
:10717000012000E0002084F8260007E0B6F5006F4B
:1071800001D3012000E0002084F8260094F82D00AF
:1071900017280BDB94F82D001E2807DCB6F5006FCE
:1071A00001D3012000E0002084F8260094F8260096
:1071B00018B14FF47A7001E002E000200646D9E0F1
:1071C00094F828000128FAD114F8235F05F0F0059F
:1071D00000BF68B22070A07A233C1A286FD2DFE883
:1071E00000F0B00D0E11120F1013143D3E646F73BA
:1071F00078A77D7E82699293949596A800BF00BF80
:1072000000BF00BF00BF00BF00BF3846FFF7D4FC7F
:10721000B0F57A6F0DDD94F8235005F0F00502E02B
:10722000C3E0CAE0ACE045F0010568B284F8230091
:107230000DE03846FFF7C0FC502808DA94F82350D8
:1072400005F0F00545F0020568B284F82300B1B2FC
:1072500094F82D00FFF74CFD064673E000BF38465A
:10726000FFF7AAFC40F6B831884209DD94F82350B4
:1072700005F0F00545F0010568B284F823000DE043
:107280003846FFF799FC502808DA94F8235005F0A7
:10729000F00545F0020568B284F82300B1B294F815
:1072A0002D00FFF725FD06464CE0B008FFF78AFCED
:1072B000064647E0B008FFF78BFC064642E040E098
:1072C00044487043060B3DE044F620607043060BD3
:1072D00038E044F620607043060B33E000BF3D48C1
:1072E0007043060B2EE0CC20B0EB960F01D90026A0
:1072F00008E0CC20C0EB9600364948434FF44C716F
:10730000B0FBF1F61EE000BF00BF00BF00BFB10838
:107310003846FFF763FC6421B0FBF1F694F82D00CA
:1073200031B2FFF732FE06464FF47A70464309E069
:1073300000BF3846FFF77EFC4FF47A7100FB01F680
:1073400000E000BF00BF94F8290048B994F82C1061
:1073500094F82B0001EB0020642101FB006609E09A
:1073600094F82C1094F82B0001EB00206FF06301CF
:1073700001FB00663046FFF7B9FCC4F81E001CE0B4
:107380001E34657905F0F00500BF68B260713846BB
:10739000FFF712FC800840F6B831484340F2FF3155
:1073A000B0FBF1F044F81E0907E094F8235005F013
:1073B000F00500BF68B284F82300781CC7B22E34F1
:1073C000202FFFF6AAAEBDE8F0810000E76C002098
:1073D000A7720020A086010070B50025FE48407805
:1073E00001282CD172B60020FB494870F6F742F90B
:1073F000FA48F6F774F900240FE0C4EBC40202EB7C
:107400000412F74B03EB4201F64A2E2303FB042040
:107410001A460BF09AF9601C84B2202CEDDB4FF475
:10742000B8652A46EF49ED48F6F756FA4FF47A71F7
:10743000EA48801EF6F777F9F6F722F962B6E648D1
:107440008078012832D172B60020E3498870F6F7BF
:1074500011F9E548F6F743F900240EE004EB440285
:1074600002EB0412E14BD118DE4A132303FB042084
:107470001A460BF06AF9601C84B2DD480088844229
:10748000ECDBDB48008800EB400101EB001085B22B
:107490002A46D449D448F6F71FFA4FF47A71D248F5
:1074A000801EF6F740F9F6F7EBF862B6CA48C078E6
:1074B00001282BD10020C849C87072B6F6F7DAF857
:1074C000CC48F6F70CF900240EE0C4EB0412C2EB32
:1074D000C202C94BD118C34A692303FB04201A46D0
:1074E0000BF033F9601C84B2052CEEDB40F20D2565
:1074F0002A46BC49BF48F6F7EFF94FF47A71BD4808
:10750000801EF6F710F9F6F7BBF862B6B2480079BC
:1075100001281CD172B6F6F7ADF8B848F6F7DFF8D7
:107520001422B749B548801CF6F7D6F91422B5499C
:10753000B2483430F6F7D0F942F21071AF48F6F79E
:10754000F2F8F6F79DF862B60020A3490871A24848
:10755000407901281BD1AC48C08B401CAA49C88384
:1075600072B6F6F787F8A948F6F7B9F87C22A84969
:10757000A648801CF6F7B0F942F21071A348F6F75E
:10758000D2F8F6F77DF862B600209349487170BDD5
:1075900010B5044672B6F6F76DF804F0010010B1AC
:1075A0009C48F6F79CF804F0020018B18B48801E46
:1075B000F6F795F804F0040018B18B48801EF6F732
:1075C0008EF804F0080018B18A48801EF6F787F894
:1075D00004F0100010B18948F6F781F804F020009B
:1075E00010B18A48F6F77BF8F6F74AF862B6FBF76F
:1075F0000DFC10BD70B586B0002500267748801EB2
:10760000F6F7AEF805464FF6FF7085427ED172B6AA
:10761000F6F730F87148801EF6F761F800248EE026
:1076200022467DA168460AF08DFDC4EBC40101EB42
:1076300004116B4A02EB4100152269460BF085F8F4
:10764000C4EBC40000EB0410654901EB4000009955
:1076500040F8151F019941609DF808100172002043
:10766000C4EBC40101EB04115D4A02EB4101C1F816
:107670001E000120C4EBC40101EB041102EB410127
:1076800081F822000020C4EBC40101EB041102EBDD
:10769000410181F82300C4EBC40101EB041102EBAA
:1076A000410181F82400C4EBC40101EB041102EB99
:1076B000410181F82500C4EBC40101EB041102EB88
:1076C000410181F82600C4EBC40101EB041102EB77
:1076D000410181F82700C4EBC40101EB041102EB66
:1076E000410181F82800C4EBC40101EB041102EB55
:1076F000410181F82900C4EBC40101EB041102EB44
:10770000410181F82A00C4EBC40100E030E001EB44
:10771000041102EB410181F82B00C4EBC40101EB21
:10772000041102EB410181F82C00C4EBC40101EB10
:10773000041102EB410181F82D00601C84B2202C61
:10774000FFF66EAF4FF4B8663246254925480AF079
:10775000FCFF324623492148F6F7BEF84FF47A7110
:107760001E48801EF5F7DFFFF5F78AFF62B624E0BA
:107770004FF4B86632461A491848F6F795F80024CF
:1077800019E0C4EBC40000EB0410154901EB400004
:1077900090F82D000F2809D0C4EBC40000EB0410B2
:1077A00001EB400090F82D00192802D1E0B2F7F764
:1077B00026F8601C84B20B2CE3DB0B48801EF5F727
:1077C000CFFF05464FF6FF70854272D172B6F5F7CE
:1077D00051FF0548801E23E0E201002002F003086B
:1077E000E76C0020C772002002F80308C77A002067
:1077F000F401002002E00308DA6A00200000040817
:1078000098010020AC0100206865002000080408F1
:107810008B8A002000E8030854332D414925750068
:10782000F5F75DFF00242BE004EB440000EB0410AF
:107830006C49084404EBC4016B4A11440A680260B5
:107840004A684260097A017204EB440000EB0410BC
:107850006449014404EBC400634A1044026841F8DF
:10786000062F42684A60007A0872002004EB440147
:1078700001EB04115B4A1144C1F80F00601C84B293
:10788000342CD1DB4FF477763246564957480AF00C
:107890005CFF324655495648F6F71EF84FF47A71A8
:1078A0005348801EF5F73FFFF5F7EAFE62B607E0A2
:1078B000FFE74FF4777632464A494D48F5F7F4FF33
:1078C0004C48F5F74DFF05464FF6FF70854220D135
:1078D00072B6F5F7CFFE4748F5F701FF40F20D21EC
:1078E00045480AF0B1FF40F20D26324642493F4872
:1078F0000AF02BFF32463D493E48801CF5F7ECFF6D
:107900004FF47A713B48F5F70EFFF5F7B9FE62B612
:1079100007E040F20D26324637493648801CF5F71D
:10792000C3FF3648F5F71CFF054642F2107085424A
:1079300008D0142132480AF087FF142131480AF098
:1079400083FF0BE014222E492C48801CF5F7ACFF76
:1079500014222C4929483430F5F7A6FF2A48F5F7B8
:10796000FFFE054642F21070854218D07C21274860
:107970000AF06AFF72B6F5F77DFE2348F5F7AFFE11
:107980007C2222492048801CF5F7A6FF4FF47A712B
:107990001D48F5F7C8FEF5F773FE62B605E07C22D8
:1079A0001A491948801CF5F77FFF002415E0C4EB45
:1079B000C40000EB0410164901EB400090F82D00C4
:1079C00048B90120C4EBC40101EB0411104A02EBD9
:1079D000410181F82800601C84B2202CE7DB06B04E
:1079E00070BD0000C77A0020CE510208C772002087
:1079F00002F8030800E00308DA6A00200000040827
:107A000098010020AC010020000804088B8A0020A7
:107A1000E76C002010B545F25550F2F74FFA0420FC
:107A2000F2F74FFA4FF47A60F2F74EFAF2F754FA9F
:107A3000F2F74DFA10BD000010B5002414E001F07B
:107A4000A2F8FE49887108468079042804DA0846BD
:107A50008079002800DD09E04FF4FA70F7F735FF70
:107A6000F2F735FA601CC4B20A2CE8DB00BFF34819
:107A70008079032806D14FF4FA730022F0A1F1A017
:107A800000F05DFE10BD10B5002404E0F2F71FFA0F
:107A90006420F7F71AFF4FF47A730022E8A1EDA0F3
:107AA00000F04DFE20B92046611CCCB21428EDDB5D
:107AB00010BD10B5002404E0F2F709FA6420F7F7CE
:107AC00004FF64230022DEA1E5A000F038FE20B907
:107AD0002046611CCCB21428EEDB10BD10B500248A
:107AE00004E0F2F7F4F96420F7F7EFFE64230022D4
:107AF000D3A1DFA000F023FE20B92046611CCCB248
:107B00001428EEDB10BD70B50020DD490870CB48AD
:107B10008079012800D170BDC848007860B100208C
:107B2000D84908704FF4FA730022C5A1D0A000F024
:107B300006FEC820F7F7C9FEC0484078012814D1D6
:107B4000002400F0D0FE41F28830F7F7BEFE00BFFF
:107B50004FF47A73CCA2BAA1CDA000F0F0FDC820FA
:107B6000F7F7B3FE0020C6490870B4480078012832
:107B700027D1002000F06FFEC820F7F7A6FEAF491E
:107B80004A31A1F1400000F088FE002413E00020FB
:107B900001F0A6FD05464FF480622946BE480AF072
:107BA000D4FDA7A1BD480AF04FFD00B108E04FF495
:107BB0007A70F7F78AFE2046611CCCB20A28E6DB11
:107BC00000BFFFF739FF00BFA5E710B5B448007844
:107BD000012806D1FFF797FFFBF718F90020B049FD
:107BE000087010BD8AB0142009900020A5490870C3
:107BF000AB49087004209149C8710020A949087058
:107C00008E48408828B18D4840884FF6FF718842E1
:107C100003D14FF4FB70894948808848807AFF2857
:107C200008D18648C07AFF2804D1402183480A3011
:107C30000AF00AFE814890F84A00FF2809D17F48DF
:107C400090F84B00FF2804D120217C484A300AF0EC
:107C5000FBFD0020924908707848808828B1774859
:107C600080884FF6FF71884203D14BF6C0207349DC
:107C70008880724948880A2207A900F0A5FB00F015
:107C8000C9FC4FF4FA60F7F720FE00F0D0FC4FF487
:107C9000FA60F7F71AFE00F0BDFD0746022F03D089
:107CA0000120664988717CE02120F5F709FB8DF8F9
:107CB00014009DF81400442866D018208DF8150093
:107CC000FE208DF816007848007848B9764840784C
:107CD00030B97548807818B97348C078002857D0F3
:107CE00071480078FF280BD16F484078FF2807D1F2
:107CF0006D488078FF2803D16B48C078FF2847D0B3
:107D000069480078102806DA674800781030C0B259
:107D10008DF8170003E0644800788DF8170062487A
:107D20004078102806DA604840781030C0B28DF8EC
:107D3000180003E05C4840788DF818005A488078B5
:107D4000102806DA584880781030C0B28DF8190033
:107D500003E0554880788DF819005348C078102802
:107D600006DA5148C0781030C0B28DF81A0003E02E
:107D70004D48C0788DF81A000DF1150000F0CAFFCB
:107D800001204849087003E02C48763000F063FF7A
:107D900005202A498871002000F05DFDFFF7B3FE41
:107DA00000BF00BF0520F7F790FDF2F790F8022F13
:107DB0000ED13C48007801280AD12048763000F0E6
:107DC0004AFF00203749087044212120F5F7A4FA22
:107DD000022F00D0E6E735480078142804DD0020A3
:107DE0003249087000F023FC1448807902287DD0C5
:107DF00012488079012879D01048407858B900207D
:107E00000E4981F86A0000210C4880F86B1080F858
:107E10006C1080F86D101B48007850B94FF4FA735D
:107E2000002207A10EA000F08AFC10B10120154924
:107E3000087014480078D8B300253AE08B8A0020F7
:107E40004F4B000041542B434950434C4F53453D49
:107E50003500000041542B524553544F5245000009
:107E600041542B43575354415254534D41525400A3
:107E700041542B435753544F50534D4152540000DB
:107E8000EE010020EF0100207265616479000000BE
:107E900041542B52535400008B8600209F8D0020AC
:107EA000F0010020E901002058600020F1010020CD
:107EB0003DE000BF00F067FEFC4988716420F7F7E1
:107EC00004FDF2F704F8F9488079032804DD284618
:107ED000691C8DB2C828EDDBC82D08DBFFF713FE47
:107EE000F3480078401CF24908705BE723E000206B
:107EF000EE4908704021ED480A300AF0A5FC202127
:107F0000EA484A300AF0A0FC0120EA494871FFF72C
:107F100063FA4FF4FA730022AFF2DC01AFF2B00063
:107F200000F00DFC6420F7F7D0FCFFF7ECFDC82053
:107F3000F7F7CBFCB8E10020DD490870DE48007897
:107F400000286FD12822D9496A3101F10C0001F0D3
:107F500079F8B0B1D54890F86A0078B9D34890F86C
:107F60006B0058B9D14890F86C0038B9CF4890F8F8
:107F70006D0018B90020D049087002E00120CE49F8
:107F80000870002001F03DF94FF4FA730022AFF2BF
:107F90005011CAA000F0D3FB012000F054FDF1F70E
:107FA00096FF4FF4FA730022AFF26C11AFF26C102F
:107FB00000F0C5FB002501E0F1F789FF00200090EB
:107FC000BA48828881880223C0A000F08AFD20B9C7
:107FD0002846691C8DB20528EEDB002501E0F1F78B
:107FE00076FF0120022340F2D24211460090B7A052
:107FF00000F077FD20B92846691C8DB20528EEDB1C
:10800000002501E0F1F763FF09AA07A9012000F0AC
:1080100095FD00288ED12846691C8DB20528F1DB1C
:1080200042E1FFE74FF48061AC480AF00DFC4FF4E9
:108030008061AB480AF008FC4FF00009002001F015
:108040004FFB04464FF480622146A5480AF07DFBB1
:10805000A348C0793038C6B2A049A14801F0B4FBAA
:108060008146B9F1000F23DD022E4CDB042E4ADCE1
:108070009A480078EE281CD198484078102818D1EA
:1080800096488078A8B99548C07890B99348007907
:1080900078B99248407960B99048807948B98F485A
:1080A000C07930B97F211020F5F736F9FAF7AEFE26
:1080B000C8E08A4880798B490979884207D0874887
:1080C0008079FF28F4D18548C0791928F0D08349F8
:1080D0000520FBF7E4FE81490520FBF707F88248FD
:1080E000008800280CDD7E48C0793038C3B27E4855
:1080F00002887E49002001F0AFFA00207A4908800A
:10810000FFF763FD9EE07EBB0024002578480078E1
:1081100030BB01207649087000234A466F49009021
:1081200002A802F056FE0446002C19DDB4F5007FCB
:1081300016DA01232246694902A804F088F96D483D
:10814000008800280CDD6648C0793038C3B2694821
:1081500002886949002001F07FFA00206549088003
:108160000020634908706DE0FFE7012E6AD15B488B
:108170000078642865D1012060490870002428E057
:10818000A000401C5549085C484991F86A10884293
:108190001DD1A000801C5149095C444890F86B0037
:1081A000814214D1A000C01C4C49095C3F4890F8A2
:1081B0006C0081420BD1A000001D4849095C3B487E
:1081C00090F86D00814202D100204C490870601C7B
:1081D000C4B209F0FF00C11700EB9171B4EBA10F1D
:1081E000CEDB4648007860B3002001F09DFB002004
:1081F0004349887700214248C17780F8201080F8F1
:10820000211088460AE03F4810F808103C48253005
:1082100000F8081008F1010000F0FF08B8F1140F91
:10822000F1DB374890F83E0040F00200344981F815
:108230003E002B48C0793038C3B24022002001F004
:108240000BFA00BF64209AFBF0F100FB11A0D0B93B
:1082500000F07DFD28B92C480078401C2A490870A0
:1082600005E002201149887100202749087026483E
:108270000078032807DB01200C498871002022497F
:1082800008700D4908705046411C1FFA81FAB0F57C
:10829000967F09DD4FF0000A012000F0B2FF0228AE
:1082A00002D10020044908707CE500008B8A002080
:1082B000F1010020E2010020EE01002041542B4397
:1082C00049504D4F44453D30000000003235352EB9
:1082D0003235352E3235352E323535008B82002041
:1082E0008B86002058600020EC0100209780002041
:1082F000E8010020EA010020A37E00208001002088
:108300005F8D0020C4620020F201002000B58BB018
:1083100001210220F1F753FF2748F1F769FA4FF4E2
:10832000167003901020029000200A9023480190BC
:108330000020079080200590202008902048009081
:108340000020069004904FF48050099069461A4826
:10835000F1F7F0FA0BB000BD10B504460122802100
:108360001748001FF3F730F921461348F1F722FBB5
:1083700001211148F1F709FB00BF1248F1F720FB7A
:108380000028FAD00F48F1F72FFB00210A48F1F737
:10839000FCFA002280210A48001FF3F715F910BDEE
:1083A00070B505460C462246294604480AF0CDF928
:1083B0002046FFF7D1FF70BD58040240078B002014
:1083C000044C004000000210F0B503460D4616466E
:1083D000002729460A2E03D0002008702846F0BD49
:1083E00033B9302001F8010B002008702846F6E769
:1083F000002B03DA2D2001F8010B5B4242F21072D0
:108400000DE093FBF2F404B937B104F1300001F848
:10841000010B04FB123301270A2092FBF0F2002A21
:10842000EFDC002008702846D9E70FB470B586B09D
:1084300006460CA8019073E00B9800785C281CD1CC
:108440000B98401C0B9000786E2809D072280FD131
:108450000D213046F3F7F4F80B98401C0B900BE01D
:108460000A213046F3F7ECF80B98401C0B9003E020
:108470000B98401C0B9000BF4BE00B980078252810
:1084800040D10B98401C0B900078642818D07328BA
:1084900033D1019810C801900BE021783046F3F7F2
:1084A000CFF800BF80213046F3F738F90028F9D023
:1084B000641C20780028F0D10B98401C0B9020E021
:1084C000019820C801900A2202A92846FFF77CFFE4
:1084D00002AC0BE021783046F3F7B2F800BF802100
:1084E0003046F3F71BF90028F9D0641C20780028E7
:1084F000F0D10B98401C0B9003E00B98401C0B90A4
:1085000000BF06E00B9810F8011B0B903046F3F704
:1085100097F800BF80213046F3F700F90028F9D022
:108520000B980078002887D106B070BC5DF814FB6A
:1085300008B54FF4A060F0F7C5FE34208DF80000B8
:1085400000208DF801008DF8020001208DF8030055
:108550006846F0F7BCFE08BD00B585B00121C8042F
:10856000F1F747FE01211020F1F736FE4FF480604D
:10857000ADF8100018208DF8130003208DF81200BC
:1085800004A9FD48F1F74CFB4FF40060ADF8100072
:1085900004208DF8130004A9F748F1F741FB4FF4CC
:1085A000E13000900020ADF80400ADF80600ADF811
:1085B0000800ADF80C000C20ADF80A006946EF4841
:1085C000F2F745FF012240F22551EC48F2F7D7FFC0
:1085D000012240F22441E948F2F7D1FFFFF7A8FF5A
:1085E0000121E648F2F7BFFF05B000BD08B5102035
:1085F0008DF8030003208DF8020001211020F1F70F
:10860000EBFD4FF40070ADF800006946DA48F1F771
:1086100007FB08BD10B5FFF7E9FFFFF79DFFFFF768
:1086200075FE4FF40071D448F1F7A7FB10BD10B5EB
:108630004FF40071D048F1F7A2FB4FF4FA70F7F74E
:1086400044F94FF40071CC48F1F797FB10BD2DE9C8
:10865000F04707460C4615469846DDF820A0C84866
:10866000B0F800046FF30E00C549A1F8000400261D
:108670000CE0B95DC148F2F7E3FF00BF8021BF48BD
:10868000F3F74CF80028F9D0701C86B24645F0DBB1
:10869000BB48B0F800046FF30E00B949A1F800041C
:1086A000084690F8010420F08001B54880F80114D4
:1086B0004FF0000904E03220F7F707F9F1F707FC63
:1086C000AF4890F80104C00928B94846411C1FFA78
:1086D00081F90A28EFDB0020A949B1F80014C1F3A1
:1086E0000E01A74A5054BCB1B5B12146104609F05D
:1086F000ABFF08B1012000E0002040B92946A048A6
:1087000009F0A2FF08B1012000E0002010B1012013
:10871000BDE8F0870020FBE744B12146984809F006
:1087200093FF08B10120F3E70020F1E729469448C0
:1087300009F08AFF08B10120EAE70020E8E72DE907
:10874000F04706460C4615461F4632468DA18B481B
:10875000FFF76BFE1CB915B90120BDE8F08788480A
:10876000B0F800046FF30E008549A1F80004084634
:1087700090F8010420F08001814880F801144FF046
:1087800000093220B7FBF0F01FFA80F804E0322035
:10879000F7F79BF8F1F79BFB794890F80104C009C3
:1087A00028B94846411C1FFA81F94045EFDB0020FB
:1087B0007349B1F80014C1F30E01714A5054B4B1B9
:1087C000ADB12146104609F03FFF08B1012000E09D
:1087D000002040B929466A4809F036FF08B1012057
:1087E00000E0002008B10120B7E70020B5E744B160
:1087F0002146634809F028FF08B10120ADE70020B9
:10880000ABE729465E4809F01FFF08B10120A4E745
:108810000020A2E710B500244FF400715648F1F78C
:10882000ACFA4FF47A70F7F750F80DE04FF4FA73A2
:10883000002256A156A0FFF782FF08B1022010BD0A
:10884000FFF7F5FE601CC4B20A2CEFDB01D100205B
:10885000F5E70120F3E710B5044624B1012C0AD056
:10886000022C18D10FE040F6C4134AA247A14CA035
:10887000FFF765FF10BD40F6C41346A243A14BA00D
:10888000FFF75DFFF6E740F6C41342A23FA14AA0FE
:10889000FFF755FFEEE70020ECE730B59FB0044648
:1088A0000D462B46224647A101A809F04BFC41F298
:1088B0008833002235A101A8FFF741FF1FB030BD6A
:1088C00030B59FB004460D462B46224642A101A872
:1088D00009F038FC41F2883300222CA101A8FFF7EF
:1088E0002EFF1FB030BD10B5CEB0642135A809F001
:1088F000CDFF002409E013AA02EB84013C4A105D7D
:108900000A22FFF761FD601CC4B2042CF3DB0024D3
:108910000AE00FAA02EB8401354A121D105D0A22FB
:10892000FFF752FD601CC4B2042CF2DB00240AE005
:108930000BAA02EB84012E4A0832105D0A22FFF7CF
:1089400043FD601CC4B2042CF2DB12A811A910AACA
:108950000FABCDE90632CDE908100EA80DAA0CA97F
:108960000BABCDE90231CDE9042016A815A914AB53
:1089700013AACDE900103DE000100140004C00407A
:108980009F8D002025730D0A000000004F4B000052
:10899000415400006E6F206368616E6765000000DF
:1089A00041542B43574D4F44453D310041542B43D7
:1089B000574D4F44453D320041542B43574D4F4492
:1089C000453D330041542B43574A41503D222573C6
:1089D000222C22257322000041542B43574A415038
:1089E0005F4445463D222573222C22257322000038
:1089F000F58A0020F0A135A809F0A4FB35AAF9A159
:108A000017A809F09FFB4FF47A630022AFF28401AC
:108A100017A8FFF794FE4EB010BD70B5A0B0044685
:108A20000D4616462B462246F3A102A8009609F0F1
:108A300089FB4FF47A730022AFF2B00102A8FFF76E
:108A40007EFE20B070BD10B586B004460CB101208A
:108A500000E000200246EEA101A809F073FB4FF4EC
:108A6000FA730022AFF2DC0101A8FFF768FE06B03E
:108A700010BDF0B5B9B006460F4614461D46642138
:108A800020A809F003FF16B1012E10D107E03B46E4
:108A9000E3A2E4A120A8009409F054FB08E03B46BF
:108AA000E4A2E0A120A8009409F04CFB00E000BF84
:108AB00000BF052D06DA20AB2A46DFA102A809F087
:108AC00041FB04E020AAE1A102A809F03BFB4FF41E
:108AD0007A63E2A2AFF24C1102A8FFF730FE39B080
:108AE000F0BD2DE9F041BAB004460D461646984651
:108AF000409F642121A809F0C9FE2346CDA2DBA135
:108B000021A88DE8600109F01DFB052F06DA21ABD5
:108B10003A46C9A103A809F015FB04E021AACBA19C
:108B200003A809F00FFB4FF47A63CCA2AFF2A411B3
:108B300003A8FFF704FE3AB0BDE8F08170B59EB01F
:108B400004460D4616467CB12B460122CCA1684650
:108B500009F0F8FA4FF4FA730022AFF2D011684628
:108B6000FFF7EDFD1EB070BD2B460022C4A1684684
:108B700009F0E8FA4FF4FA730022AFF2F0116846F8
:108B8000FFF7DDFDEEE710B54FF4FA730022AFF208
:108B90000421C0A0FFF7D3FDD8B1C2A1C44809F099
:108BA00053FD08B1022010BDC2A1C14809F04CFD1F
:108BB00008B10320F7E7C2A1BD4809F045FD08B19F
:108BC0000420F0E7C1A1BA4809F03EFD08B1052034
:108BD000E9E70620E7E710B500244FF4FA73002216
:108BE000AFF25821ABA0FFF7AAFD002831D0BAA1FF
:108BF000AF4809F029FD10B144F0010401E024F070
:108C00000104B9A1AA4809F01FFD10B144F0020403
:108C100001E024F00204B8A1A54809F015FD10B147
:108C200044F0040401E024F00404B7A1A04809F0D2
:108C30000BFD10B144F0080401E024F00804B6A1D3
:108C40009B4809F001FD10B144F0100401E024F04C
:108C50001004204610BD2DE9FC4180464FF4FA7304
:108C60000022AFF2D821B0A0FFF769FD002600274F
:108C7000B1A18F4809F0E8FC05460DB10B3502E0C3
:108C80000020BDE8FC81002435E0285D3A280DD1A4
:108C9000022F07D19DF801109DF8000001EB001094
:108CA00008F80600701CC6B2002722E0052E03D18A
:108CB000285D222800D120E0285D30280BDB285DCC
:108CC000392808DC285D3038C2B23846791CCFB26A
:108CD0000DF800200DE0285D61280ADB285D66287C
:108CE00007DC285D5738C2B23846791CCFB20DF880
:108CF0000020601CC4B2282CC7DB00BF022F07D1A4
:108D00009DF801109DF8000001EB001008F8060026
:108D10000120B6E730B591B0044660792179E27858
:108D2000A378CDE90032CDE902106378227886A1DC
:108D300004A809F007FA4FF47A730022AFF2B431B5
:108D400004A8FFF7FCFC0546284611B030BDF8B575
:108D50004FF4FA730022AFF2CC3185A0FFF7EFFC9D
:108D60000027002686A1524809F06EFC05460DB189
:108D70000C3509E085A14E4809F066FC05460DB1A9
:108D80000220F8BD0020FCE700240EE0285D222828
:108D900003D1601C0544002609E02A5D3046711CA1
:108DA000CEB27C490A54601CC4B23C2CEEDB00BF3E
:108DB0000DB11535F2E0EFE02225732E25732E2537
:108DC000732E2573222C2225732E25732E25732EA8
:108DD0002573222C2225732E25732E25732E2573A1
:108DE0002200000041542B4349505354415F4445F5
:108DF000463D25730000000041542B43575341501A
:108E00003D222573222C222573222C312C2564002F
:108E100041542B4349504D55583D256400000000F6
:108E200054435000222573222C222573222C2573B3
:108E3000000000005544500041542B434950535406
:108E40004152543D25642C257300000041542B43AE
:108E5000495053544152543D25730000414C5245F2
:108E6000415920434F4E4E45435400002225732262
:108E70002C222573222C25642C25642C25640000CB
:108E800041542B4349505345525645523D25642C7D
:108E90002573000041542B434950535441545553BA
:108EA000000000005354415455533A320D0A00005B
:108EB0009F8D00205354415455533A330D0A0000FE
:108EC0005354415455533A340D0A000053544154FD
:108ED00055533A350D0A00002B4349505354415421
:108EE00055533A302C0000002B4349505354415401
:108EF00055533A312C0000002B43495053544154F0
:108F000055533A322C0000002B43495053544154DE
:108F100055533A332C0000002B43495053544154CD
:108F200055533A342C00000041542B4349505354BC
:108F3000414D41433F0000002B4349505354414DA4
:108F400041433A220000000041542B4349505354FE
:108F5000414D41435F4445463D2225783A25783AC4
:108F600025783A25783A25783A25782200000000BD
:108F700041542B43574A41505F4355523F00000034
:108F80002B43574A41505F4355523A0062757379FB
:108F900000000000958A00200020F2E6002408E08E
:108FA000285D2C2803D1601C0544002603E0601CCA
:108FB000C4B2052CF4DB00BF00270026002417E014
:108FC000285D00B916E0285D2D2801D100260DE0AE
:108FD000285D30280ADB285D392807DC285D303819
:108FE000C2B23046711CCEB20DF80020601CC4B273
:108FF000052CE5DB00BF012E04D19DF80000FE49E1
:1090000008721DE0022E0AD19DF801009DF80010A3
:1090100001EB810100EB4100F749087210E0032EDB
:109020000ED19DF80000642148439DF8011001EB2A
:10903000810100EB41009DF802100844EE490872DE
:1090400001209EE62DE9FE4F8146884692464FF468
:10905000FA730022AFF2CC61E8A0FFF770FB0026A4
:109060000027E9A1EA4809F0EFFA05460DB1ED1D28
:1090700002E00020BDE8FE8F00243BE0285D2E28A2
:1090800028D1012F04D19DF8080008F806001DE042
:10909000022F0AD19DF809009DF8081001EB81010B
:1090A00000EB410008F8060010E0032F0ED19DF8F8
:1090B0000800642148439DF8091001EB810100EB91
:1090C00041009DF80A10084408F80600701CC6B25A
:1090D00000270DE0032E03D1285D222800D10BE0EC
:1090E000285D3038C2B23846791CCFB202A90A5482
:1090F000601CC4B25445C1DB00BF012F04D19DF8F0
:10910000080008F806001DE0022F0AD19DF80900AA
:109110009DF8081001EB810100EB410008F8060002
:1091200010E0032F0ED19DF80800642148439DF8FC
:10913000091001EB810100EB41009DF80A10084481
:1091400008F806004FF4FA730022AFF2C071AFF2D4
:109150002820FFF7F4FA00260027AFF22421AC48BC
:1091600009F072FA05460DB10B3501E0002081E7E8
:10917000002435E0285D3A280DD1022F07D19DF853
:1091800001109DF8000001EB001009F80600701CAA
:10919000C6B2002722E0052E03D1285D222800D187
:1091A00020E0285D30280BDB285D392808DC285DAD
:1091B0003038C2B23846791CCFB20DF800200DE02D
:1091C000285D61280ADB285D662807DC285D5738A2
:1091D000C2B23846791CCFB20DF80020601CC4B270
:1091E0005445C7DB00BF022F07D19DF801109DF841
:1091F000000001EB001009F80600FFF7A8FD0120B0
:1092000038E72DE9FF4180464FF4FA730022AFF6AC
:10921000840180A0FFF793FA0024002581A17C48F7
:1092200009F012FA07460FB17F1D03E0002004B0D9
:10923000BDE8F08100263BE0B85D2E2828D1012D45
:1092400004D19DF80C0002A908551DE0022D0AD199
:109250009DF80D009DF80C1001EB810100EB410021
:1092600002A9085510E0032D0ED19DF80C006421D1
:1092700048439DF80D1001EB810100EB41009DF882
:109280000E10084402A90855601CC4B200250DE068
:10929000032C03D1B85D222800D10BE0B85D303833
:1092A000C2B22846691CCDB203A90A54701CC6B2CA
:1092B000282EC1DB00BF012D04D19DF80C0002A9AE
:1092C00008551DE0022D0AD19DF80D009DF80C10E7
:1092D00001EB810100EB410002A9085510E0032DCC
:1092E0000ED19DF80C00642148439DF80D1001EB50
:1092F000810100EB41009DF80E10084402A90855B9
:10930000B8F1000F04D13C480299C0F86A1021E07E
:109310009DF80800384991F86A10884214D19DF8E8
:109320000910354890F86B0081420DD19DF80A1064
:10933000314890F86C00814206D19DF80B102E4800
:1093400090F86D00814205D02B480299C0F86A1050
:1093500002206CE70024002534A12D4809F074F99F
:1093600007460FB10A3701E0002060E700263BE026
:10937000B85D2E2828D1012D04D19DF80C0001A93B
:1093800008551DE0022D0AD19DF80D009DF80C1026
:1093900001EB810100EB410001A9085510E0032D0C
:1093A0000ED19DF80C00642148439DF80D1001EB8F
:1093B000810100EB41009DF80E10084401A90855F9
:1093C000601CC4B200250DE0032C03D1B85D222837
:1093D00000D10BE0B85D3038C2B22846691CCDB26E
:1093E00003A90A54701CC6B2282EC1DB00BF012D90
:1093F00025D19DF80C001FE08B8A002041542B439F
:10940000494653520000000053544149502C220059
:109410009F8D002041542B4349505354415F435585
:10942000523F00003A69703A220000003A676174C6
:10943000657761793A22000001A908551DE0022DE7
:109440000AD19DF80D009DF80C1001EB810100EB95
:10945000410001A9085510E0032D0ED19DF80C0024
:10946000642148439DF80D1001EB810100EB4100A0
:109470009DF80E10084401A90855B8F1000F04D159
:10948000FE480199C0F8721021E09DF80400FB49E4
:1094900091F87210884214D19DF80510F74890F8A1
:1094A000730081420DD19DF80610F44890F87400C5
:1094B000814206D19DF80710F04890F8750081426E
:1094C00005D0EE480199C0F872100220AFE60024E2
:1094D0000025EBA1ED4809F0B7F807460FB10A37B0
:1094E00001E00020A3E600263DE0B85D2E282AD149
:1094F000012D04D19DF80C000DF804001FE0022D91
:109500000BD19DF80D009DF80C1001EB810100EBD3
:109510004100C0B20DF8040011E0032D0FD19DF8F9
:109520000C00642148439DF80D1001EB810100EB14
:1095300041009DF80E100844C0B20DF80400601CF4
:10954000C4B200250DE0032C03D1B85D222800D160
:109550000BE0B85D3038C2B22846691CCDB203A911
:109560000A54701CC6B2282EBFDB00BF012D04D1E7
:109570009DF80C000DF804001FE0022D0BD19DF8A2
:109580000D009DF80C1001EB810100EB4100C0B211
:109590000DF8040011E0032D0FD19DF80C0064219B
:1095A00048439DF80D1001EB810100EB41009DF84F
:1095B0000E100844C0B20DF80400B8F1000F04D139
:1095C000AE480099C0F86E1021E09DF80000AB494C
:1095D00091F86E10884214D19DF80110A74890F8B8
:1095E0006F0081420DD19DF80210A44890F87000E0
:1095F000814206D19DF80310A04890F87100814285
:1096000005D09E480099C0F86E1002200FE6012098
:109610000DE610B54FF4FA730022AFF690419CA00E
:10962000FFF78DF808B9002010BD4FF4FA739CA223
:10963000AFF6A8419BA0FFF782F8F5E710B54FF40D
:109640007A70F6F742F99AA19A48FEF7EEFE4FF4C7
:10965000FA70F6F73AF910BD2DE9F043ADF5177D34
:1096600080460E4614461F464FF0000940F2262061
:10967000844204D900200DF5177DBDE8F083B8F1D0
:10968000000F08D03246AFF630018A48FEF7CDFE13
:109690004FF0010922E0052F06DA23463A4686A15B
:1096A00001A808F04FFD04E0224688A101A808F0B7
:1096B00049FD01A809F02AF885B215B1B5F5077F73
:1096C00001DD0020D7E7294601A8FEF769FE022048
:1096D000F6F7FBF8A1B23046FEF762FE4846CAE74D
:1096E00070B5044600256948B0F800046FF30E0019
:1096F0006649A1F80004084690F8010420F08001B2
:10970000624880F8011440F2024109F09DF80026F9
:1097100004E00220F6F7D9F8F0F7D9FB5B4890F89F
:109720000104C00920B93046711C8EB26428F0DBF8
:1097300000205649B1F80014C1F30E01534A5054A9
:109740000CB1154605E065A1504808F07DFF00B159
:109750004E4D284670BD70B5002540F22551554844
:10976000F1F7F2FFD8B15348F1F76EFFC4B24748A2
:10977000B0F80004C0F30E0040F2FF3188420EDA68
:109780004249B1F80014C1F30E00411C3F4AB2F83F
:10979000002461F30E023D49A1F800240C5440F26C
:1097A00024414448F1F7D0FF01280CD1374890F804
:1097B000010420F080008030344981F801043D48E4
:1097C000F1F742FFC4B270BD30B502460B4600242B
:1097D000107A2C2850D1907A3A2815D1507A302816
:1097E00012DB507A39280FDC507A303884B20021ED
:1097F00006E001F10B00105C03F8010B481C81B27C
:10980000A142F6DB204630BDD07A3A2821D1507AE9
:10981000302832DB507A39282FDC907A30287FDBF1
:10982000907A39287CDC907A3038557A303D05EBD7
:10983000850500EB450084B2002106E001F10C0033
:10984000105C03F8010B481C81B2A142F6DB2046F4
:10985000D9E7107B3A2863D1507A302860DB507A00
:1098600039285DDC907A30285ADB907A392857DC29
:10987000D07A302854DB35E054E051E08B8A002068
:109880003A6E65746D61736B3A2200009F8D002003
:1098900041542B4349504D4F44453D310000000099
:1098A0003E00000041542B43495053454E440000B4
:1098B0002B2B2B00004C004041542B434950534567
:1098C0004E443D25642C25640D0A000041542B4371
:1098D000495053454E443D25640D0A002B495044E0
:1098E00000000000D07A39281ADC507A303864251C
:1098F0006843957A303D05EB850500EB4505D07A48
:109900003038284484B2002106E001F10D00105CDB
:1099100003F8010B481C81B2A142F6DB204672E736
:10992000002070E700206EE710B50446402144484F
:1099300008F08AFF1CB965204149088004E0012C29
:1099400002D167203E4908801D203D4948803D489E
:10995000007888803B4841783948C180394881780F
:10996000374801813748C17835484181352034492D
:10997000888134480079C881334890F86A000882A9
:10998000314890F86B102E4841822F4890F86C10A7
:109990002B4881822C4890F86D102948C1822A48B2
:1099A000408827490883472048832648007B8883CE
:1099B00026480088C0F307202449097840EA01209E
:1099C0001F4948841F48007981F824001F48006817
:1099D000000C00021D490968090C40EA21201849C1
:1099E000A1F83900002081F83B001748808888875B
:1099F000002081F83E0081F83F00012014490870E2
:109A000010BD0B120370417000238370C3701312DA
:109A100003714271704700B59FB0642106A808F039
:109A200035FF06AA0BA101A808F08CFB4FF47A635E
:109A300000220DA101A8FEF782FE1FB000BD0000AC
:109A40005F8D0020586000208B8A002004000020D9
:109A50008001002041542B4357444843505F444504
:109A6000463D312C310000004F4B0000002801D052
:109A7000D14B036011B1D04808380860002A02D0E9
:109A8000CD48001F10607047412801D20120704767
:109A900000207047C94800787047C949085C401CDD
:109AA0007047C849084410F8010C70472DE9F0418F
:109AB00006460C463046FFF7F4FF00256F1E7CB1CA
:109AC00055212180676025720421A172C2B2002154
:109AD0000120FBF7F9FD206184F87052D4F874423C
:109AE000DCB16F202080676025720820A07204F12D
:109AF0001000074604F0D4FF00221146384604F057
:109B0000D8FF00220121384604F0D3FF00220221B1
:109B1000384604F0CEFF84F870523046BDE8F0417C
:109B2000FCF773BD10B503460C4600221846FFF73C
:109B3000B8FF402B08D2C1B20120FCF712FB01464E
:109B4000204605F076F80246104610BD2DE9F04398
:109B5000ADF51B7D814608469846A39DA29CFFF764
:109B6000A0FF0227FE1E4F2A42D008DC1C2A32D05A
:109B7000242A68D04B2A1BD04D2A08D11EE0512A36
:109B800066D0552A39D06F2A41D0752A6CD02770FB
:109B9000202028703046002806DBB8F1FF3F03D0B4
:109BA00027703220287030460DF51B7DBDE8F0830C
:109BB00002460021484604F0D7FBECE7C1B2012081
:109BC000FCF7CFFA014601A805F033F801A9484691
:109BD00004F087FCDFE7C1B20120FCF702FB01467D
:109BE00001A805F026F801A9484604F07AFCD2E75E
:109BF0000021484604F07BFDCDE7C2B200210120E0
